:104CAD004F787967656E3A202025352E316620259F
:104CBD002520283F29004F787967656E3A202025F9
:104CCD00352E3166202525004F787967656E3A209F
:104CDD0020756E63616C69627261746564004F600A
:104CED003A2073657420746F2025352E316620258A
:104CFD00250048656C69756D3A202020202E2020F6
:104D0D0025250048656C69756D3A205B25352E317A
:104D1D00662025255D0048656C69756D3A20202556
:104D2D00352E31662025250054656D7065726174D0
:104D3D007572653A2025352E3166202573007E4625
:104D4D00007E43007D25362E3166202573204025BB
:104D5D00362E316625730070736900626172005CD6
:104D6D0025362E3166202573204025362E316625B9
:104D7D00730050726573737572653A2025362E3146
:104D8D00662025730000576F726B696E672C20705B
:104D9D006C6561736520776169740048656C697530
:104DAD006D004F787967656E2025352E316620258B
:104DBD0025004169720045414E2025352E31660092
:104DCD00544D582025352E3166202F25352E316630
:104DDD000048656C696F782025352E3166202525B4
:104DED00204F6000466F756C204169722028253573
:104DFD002E3166202525204F6029004572726F7275
:104E0D0000417070726F78696D6174652076616CA8
:104E1D007565733A004D4F4425342E306620257349
:104E2D002C2070704F603D25332E316600667377F0
:104E3D00006D7377004D4F442020202020257300F6
:104E4D00454E4425342E3066202525206F66206181
:104E5D0069720020202020206C6F77202061637400
:104E6D0075616C2068696768002025733A25352EB9
:104E7D0031662025352E31662025352E31660025EB
:104E8D00254F603A25352E31662025352E31662089
:104E9D0025352E316600252548653A25352E316696
:104EAD00202020202E202025352E31660025254856
:104EBD00653A25352E31662025352E31662025356E
:104ECD002E3166007073693A25352E3066202535F2
:104EDD002E30662025352E3066006261723A2535FA
:104EED002E31662025352E31662025352E31660072
:104EFD0042617474657279204C6F772020202052A6
:104F0D00653A253373004F7574206F662072616E9C
:104F1D00676520202052653A25337300202020201C
:104F2D00202020202020202020202052653A2533CB
:104F3D007300202020202020414C41524D204F460F
:104F4D004600202020205B42617474657279204CEC
:104F5D006F775D00202020205B6F7574206F6620B9
:104F6D0072616E67655D00202020202020202020AA
:104F7D0020202020202020202000202020205B2009
:104F8D0020202020202020202020205D002573209F
:104F9D002041637475616C204025352E31662025C6
:104FAD0073004162733A2025362E31662020253656
:104FBD002E31660052656C3A2025362E3166202042
:104FCD0025362E31660054616E6B2074656D702E22
:104FDD003A2025362E31662025730052656C61749A
:104FED006976653A2025362E31662025730041728B
:104FFD00676F6E00436172626F6E2064696F7869CE
:10500D0064650053756C70687572206865786166AB
:0D501D006C756F7269646500487964726F8C
:10502A0067656E00436F6E7461696E732068796498
:10503A00726F67656E00556E6B6E6F776E20676173
:10504A0073005761726E696E6700556E636572749C
:10505A0061696E20646574656374696F6E00556E6C
:10506A0062726561746861626C6520676173004F82
:10507A0025352E316600482020202E20004825356F
:10508A002E3166004865202A2A2A2E2A20004865E1
:10509A002025352E316620004F32202A2A2A2E2A30
:1050AA000D0A004F322025352E31660D0A00787818
:0250BA0078007C
:100026004426E800000000C1154126CF004426D032
:10003600000000004226D400004226DA0000C196E5
:10004600C1124426E0000000004426CB0000000058
:100056004426D6000000004426E400000000C11437
:1000660044274000000000C1134426DC00000000C5
:108DE0009026E0E4FFFE7DC87C42E0F8A3E0F9A312
:108DF000E0FAA3E0FB229025171220459019B8E075
:108E0000FCA3E0FDA3E0FEA3E0FF22121657E4FB63
:108E1000FA79A07840121760E4FBFAF9784202155B
:108E20006690249AE0FBA3E0FAA3E0F92290251BC8
:108E3000EBF0A3EAF0A3E9F02212165790251702EF
:108E400020459024B6E025E025E024ECF582E434CA
:108E500026F583227F917E0F7D687C419026DC225F
:108E60007DC8E4FFFE7C429026CB22EC4D4E4F7B2A
:108E7000FF2212165790251B022045E4FFFE7D10AD
:108E80007C41229026C9E0FFA3E0FD227F0A7ED725
:108E90007DA37C3B9026CB221215627B917A0F79C1
:108EA00068784102165712204590249AE0F9A3E011
:108EB000FAA3E022E4FFFE7C439026D6229024C34E
:108EC000E0FCE4121885A804A905AA06AB072290C5
:108ED000251E12204590197622E0FCA3E0FDE41245
:108EE00018807BE37A38790E783A021657F0A3742B
:108EF00024F0A37460F07BFF2212165790246112B5
:108F000020457BFF227BFF7A4D7992227F0A7ED714
:108F10007D237C3C22E0FCA3E0FDEC021880902441
:108F20005F7401F0227DA17C437F007E809026D675
:108F3000221215667BA47A70797D783F0217FD9026
:108F4000251F1220457BFF22E4FFFE7C439026D69E
:108F5000221215629024B7022045121566E4FBFA2E
:108F6000F978400217607F857EEB7D517C3E90262C
:108F7000E0227FF67E287D5C7C3E9026E022EC4D50
:108F80004E4F90193F22A3F0A37401F0A322E4FBFB
:108F9000FA798078410217609026D4E0FEA3E07849
:0C8FA000022224ECF58274263EF58322A8
:0EDFEF00E49026D4F0A3F09026DAF0A3F022FE
:108287009024A91220459024AD128E3090157912B2
:108297008DFFEC4D4E4F70179024A9128DFFA3123E
:1082A7008E24121F7F9024B3128E24E4021CB190F7
:1082B70024B0128E24121C4970289024A9128DFF15
:1082C700C004C005C006C007128F98C333CE33CE93
:1082D700D8F9128FA2D007D006D005D004122045B6
:1082E7008014128F98C333CE33CED8F9128FA212CF
:1082F7002051BF8000009026D5E004F0700690263C
:10830700D4E004F09026D4128F1590159A128DEAB6
:108317001217FD5007E49026D4F0A3F09026DAE078
:10832700FEA3E0FF9026D4E0B5062BA3E0B5072611
:108337009026DBE004F070069026DAE004F0902641
:10834700DA128F1590159A128DEA1217FD5007E46D
:108357009026DAF0A3F0E49024C3F09024B712201B
:1083670051000000009024BB1220514479C00090B6
:1083770024BF122051C479C0009026DBE002841D7F
:108387009024B6E0FFFD9026D4E07003A3E06D7063
:1083970003028424EF128E46128DFFE4FBFA7980E4
:1083A70078BF1217FD50549024B7128DFF128E42DA
:1083B700128DEA121566128F549024C3E004F0124E
:1083C7008E42128DFF9024BB128DEA1217FD600EAC
:1083D700400C128E42128DFF9024BB122045128E44
:1083E70042128DFF9024BF128DEA1217FD500C1216
:1083F7008E42128DFF9024BF1220459024B6E004D0
:10840700F0E0FCE412188590159A128DEA1217FD18
:108417004003028387E49024B6F0028387128EBD5F
:1084270090159A128DFF1215621218B99024B31283
:108437008E24EF121CB19024C3E0FF70199024B072
:10844700128E247401121CB19024AD128E241220B6
:10845700820000000022EFD3940240239024B71239
:108467008DFFA3128DEA128F519024B7128DFF90C2
:0584770024BF128DEA94
:10847C00128F519024C3E024FEF0128EBD9024B7CD
:10848C00128DFF1217609024AD128E24121F7F22C2
:10753A0090245CEFF0A3EDF0901537128DFFEC4D1F
:10754A004E4F603830150E128DE0128E397BFF7A5D
:10755A004C79AD80339012C4128DFFEC4D4E4F60C2
:10756A000E128DE0128E397BFF7A4C79C380197B1B
:10757A00FF7A4C79D57F0112CFDE8011128DE0128D
:10758A008E397BFF7A4C79EB7F0112D2B590245C5D
:10759A00E0D3940040087BFF7A4C79FF8023902443
:1075AA005DE0D394009026CB128DE3400B128E3906
:1075BA007BFF7A4D79108009128E397BFF7A4D79DB
:1075CA00237F0212D2B5901976128DFFEC4D4E4FE1
:1075DA00600E128E7B9026E4128DEA128E0B8006C4
:1075EA009026E4128DFF128E3C901976128DFF12AE
:1075FA008E6B60067A4D794B80047A4D794E128EE5
:10760A002D7BFF7A4D79357F0312D2B512E077EFE1
:10761A00640960030277A020140302775E12DEE891
:10762A00902462122045902740128DFF9024F01278
:10763A002045902462128DFF9024F4122045902652
:10764A00E0128DFF9024F81220459026CB128DFF70
:10765A009024FC1220459026DC128DFF12D68A90C7
:10766A00245E128DF9EC4D4E4F600B128E54128D22
:10767A00EA12165780069026DC128DFF128DF6123A
:10768A008E6B60067A4D796480047A4D7968128E21
:10769A002D901976128DFFEC4D4E4F600E128E7B97
:1076AA00902740128DEA128E0B8006902740128D89
:1076BA00FF128ECF128DFF128E6B60067A4D794BB8
:1076CA0080047A4D794E902522128E307BFF7A4DB6
:1076DA0079517F0412D2B5128DFCEC4D4E4F6013D6
:1076EA007F917E0F7D687C4190245E128DEA12168E
:1076FA0057800690245E128DFF128DF6128E6B60F3
:10770A00067A4D796480047A4D7968128E2D901923
:10771A0076128DFFEC4D4E4F600E128E7B902462D6
:10772A00128DEA128E0B8006902462128DFF128E41
:10773A00CF128DFF128E6B60067A4D794B80047AD8
:10774A004D794E902522128E307BFF7A4D796C7FCF
:10775A000502D2B5128DFCEC4D4E4F600B128E54C1
:10776A00128DEA12165780069026DC128DFF128DB2
:10777A00F6128E6B60067A4D796480047A4D7968C8
:10778A00128E2D7BFF7A4D797F7F0412D2B5128F2C
:07779A00057F0512CFDE227E
:1072CB00EDD394005005EF9400400B7BFF7A4D7982
:1072DB00937F0202CFDE7F007E507DC37C479015EB
:1072EB00DC128DEA1216579026E0128DEA12176007
:1072FB007B807AE679C578C71215667BF27A84793A
:10730B001D784612176090245C1220457D9A128ED0
:10731B0062128DEA121657128EC6E4FFFE7DC87CF0
:10732B00421215629024601220457FA47E707D7DF1
:10733B007C3F9026CB128DEA1217FD40117A4D79C6
:10734B00A812752F12205141B800000274827FA43D
:10735B007E707D7D7C3F9026E0128DEA1217FD40FA
:10736B000F128DE0128E397BFF7A4D79AF02747D4F
:10737B00128E8C128DEA1217FD5033128F66128DFE
:10738B00EA1217FD4028128F72128DEA1217FD6058
:10739B0002501B7A4D79BF12752F12205142C80033
:1073AB000090245C12205142820000027482128EE3
:1073BB008C128DEA1217FD501C128F72128DEA126D
:1073CB0017FD6011400F128DE0128E397BFF7A4D45
:1073DB0079C302747D128E8C128DEA1217FD402B2D
:1073EB009026E0128DFF9026CB128DEA128F316022
:1073FB001A4018128DE0128E39128E60128DEA121D
:10740B008E727BFF7A4D79CD02747D9026E0128DC2
:10741B00FF9026CB128DEA128F316002502A9026F4
:10742B00E0128DFF9026CB128DEA1215667BAE7A99
:10743B00477981783F1217FD400E128DE0128E397D
:10744B007BFF7A4D79DE802A128E8C128DEA121711
:10745B00FD5019128F66128DEA1217FD500E128D08
:10746B00E0128E397BFF7A4D79F180067BFF7A4EE5
:10747B0079087F0212D2B57BFF7A4E790E7F031209
:10748B00CFDE7F007EE07D797C4490245C128DEA18
:03749B001217FDC8
:10749E005054901997128DFFEC4D4E4F60137F484C
:1074AE007EF97D517C4090245C128DEA1216578035
:1074BE000690245C128DFF128E3C901997128DFF50
:1074CE00128E6B60067A4E793A80047A4E793E12AD
:1074DE008E2D9015DC128DFF90251E1220457BFF00
:1074EE007A4E79228021901997128DFF128E6B6041
:1074FE00067A4E793A80047A4E793E902517128E8E
:10750E00307BFF7A4E79427F0412D2B57BFF7A4EE2
:10751E00794D902460128DFF128E3C7F0512D2B5EC
:0C752E00227BFF7F0212CFDE902460223F
:1050BC0090245CEFF0A3EDF0A3EBF0E4A3F07860A8
:1050CC007C247D017BFF7A5079B8FE7F04121C236F
:1050DC00E4902464F07BFF7A4E79607F0112CFDE7E
:1050EC0090245EE0700302518A20140302518A90CE
:1050FC001976128DFF128E6B60067A4D794B8004F7
:10510C007A4D794E902517128E30901976128DFFAC
:10511C00EC4D4E4F600E128E7B901767128DEA127B
:10512C008E0B8006901767128DFF90251A128ED267
:10513C00128DFFEC4D4E4F600E128E7B902740125D
:10514C008DEA128E0B8006902740128DFF128ECFA7
:10515C00128DFFEC4D4E4F600E128E7B9017041289
:10516C008DEA128E0B8006901704128DFF9025226B
:10517C001220457BFF7A4E79767F0112D2B59015BD
:10518C0037128DFFEC4D4E4F60219016A1128DFF02
:10519C00128E3C128DE0128E729016C2128DFF127E
:1051AC008F3F7A4E798C7F0212D2B590245CE0D37B
:1051BC0094005006A3E09400401A7BFF7A4E79A32A
:1051CC009016E3128DFF128E3C901704128DFF1275
:1051DC008E75801F9016E3128DFF128E3C128E601E
:1051EC00128DEA128E72901704128DFF128F3F7A75
:1051FC004E79BA7F0312D2B590245EE0700812E0AB
:10520C0077EF64097060128DFCEC4D4E4F602C9062
:10521C001725128DFF128E3C128E54128DEA128EAF
:10522C00727F917E0F7D687C41901746128DEA1239
:10523C001657128F3F7A4E79D180247BFF7A4E79A4
:10524C00E7901725128DFF128E3C9026DC128DFFF5
:0C525C00128E75901746128DFF90251FD2
:105268001220457F0412D2B58008128F057F0412E0
:10527800CFDE901537128DFFEC4D4E4F6037128FF1
:105288000C9016A1128DEA1217FD60154013128DAD
:10529800E01216579016A1128DEA1217FD600250FF
:1052A80011128DE01216579016C2128DEA1217FDD0
:1052B8005003128F1E90245CE07041A3E0703D12F1
:1052C8008F0C9016E3128DEA1217FD601840161223
:1052D8008E60128DEA1216579016E3128DEA121795
:1052E800FD60025014128E60128DEA121657901744
:1052F80004128DEA1217FD5003128F1E3014371254
:105308008F0C901767128DEA1217FD6013401190E9
:105318001767128DFF902740128DEA1217FD401370
:10532800901788128DFF902740128DEA1217FD60A2
:10533800054003128F1E128F0C901725128DEA124A
:1053480017FD60134011901725128DFF9026DC126F
:105358008DEA1217FD4013901746128DFF9026DC38
:10536800128DEA1217FD60054003128F1E300D03DF
:10537800128F1E90245EE0700302545CA3E060224A
:10538800201228D212E4FFFE7D207C429017A91239
:105398008DEA1216571218B9901D4FEEF0A3EFF0D0
:1053A8008009C212E4901D4FF0A3F090245FE07BC7
:1053B800017A247964600FE4FD7F0112DA589024A1
:1053C80060742DF0800D7D017F0112DA5890246001
:1053D8007431F0301213901D4FE07002A3E0700991
:1053E800FD12549D742DF080087D0112549D743275
:1053F800F07B017A24796430100FE4FD7F0312DA20
:1054080058902462742DF0800D7D017F0312DA58C4
:105418009024627433F0902464E060077F2C7E014E
:1054280012DE9C90245FE0601A9025177401300DFD
:1054380009128EED7A4E79FD8015128EED7A4F792C
:0654480013800C902517F3
:10544E007401128EED7A4F79297F0502D2B52010A4
:10545E00087BFF7A4F793F803090245FE0602430E4
:10546E0016117BFF300D067A4F794F800C7A4F79EB
:10547E006180067BFF7A4F79747F0512CFDEB216FC
:10548E0002DD7D7BFF7A4F79877F0512CFDE227B8F
:0E549E00017A2479647F0212DA589024612288
:109C910012DEE8902460122045902740128DFF903B
:109CA10024F0122045902460128DFF9024F412209C
:109CB100459024F81220513E570A3D9024FC122071
:109CC10051000000009026DC128DFF12D68A9024EC
:109CD1005C128DF9128E6B60067A4D796480047A7C
:109CE1004D7968902517128E30901976128DFFEC00
:109CF1004D4E4F600E128E7B902460128DEA128EB3
:109D01000B8006902460128DFF90251A128ED212BC
:109D11008DFF128E6B60067A4D794B80047A4D79F6
:109D21004E90251E128E307BFF7A4F799A7F011259
:109D3100D2B5128DFCEC4D4E4F600B128E54128D2C
:109D4100EA12165780069026DC128DFF128DF6EC72
:109D51004D4E4F600B128E54128DEA12165780062B
:109D61009026DC128DFF128E757BFF7A4F79AF7FC3
:109D71000212D2B5128DFC128F7E600E128DEA9006
:109D810026DC128DFF128E98800C128DEA9026DC53
:109D9100128DFF121562128DF6128F7E600E128DDA
:109DA100EA9026DC128DFF128E98800C128DEA90BB
:109DB10026DC128DFF121562128E757BFF7A4F79A8
:109DC100C17F0312D2B5128F057F0412CFDE901925
:109DD10076128DFFEC4D4E4F600E128E7B90274018
:109DE100128DEA128E0B8006902740128DFF128E83
:109DF1003C901976128DFF128E6B60067A4D794B6D
:109E010080047A4D794E128E2D7BFF7A4F79D37F64
:049E11000502D2B5BF
:10C9EE00128F057F0112CFDE128F057F0212CFDE6E
:10C9FE00128DFCEC4D4E4F600B128E54128DEA12BE
:10CA0E00165780069026DC128DFF128DF6128E6B55
:10CA1E0060067A4D796480047A4D7968128E2D7B8A
:10CA2E00FF7A4D797F7F0312D2B5128DFC128F7E65
:10CA3E00600E128DEA9026DC128DFF128E98800CFD
:10CA4E00128DEA9026DC128DFF121562128DF612EF
:10CA5E008E6B60067A4D796480047A4D7968128EF9
:10CA6E002D7BFF7A4F79E87F0412D2B5128F057FA6
:04CA7E000502CFDE00
:10B94D007D9E128EB4128DEA1217FD6016401412F0
:10B95D008F25128DEA1217FD50097BFF7A4F79FB67
:10B96D0002B9F87D7D128EB4128DEA1217FD6018A2
:10B97D0040167D82128F48128DEA1217FD50097BF9
:10B98D00FF7A50790102B9F87D02128F48128DEAC3
:10B99D001217FD601C401AE4FFFE7D097C439026C2
:10B9AD00D6128DEA1217FD50087BFF7A5079108060
:10B9BD003A7DA27C44128F29128DEA1217FD600A7E
:10B9CD0040087BFF7A50792580217F007EC07D80E5
:10B9DD007C449026D6128DEA1217FD7BFF6008403D
:10B9ED00067A50792E80047A5079407F0212CFDE8C
:10B9FD007BFF7A50794C7F0312CFDE7BFF7A507933
:10BA0D00547F0412CFDE7BFF7A5079687F0502CF19
:01BA1D00DE4A
:10D7210090245CEFF0A3EDF0D217128DE0128E3948
:10D731007BFF7A5079797F0112D2B590245CE0D3D6
:10D7410094005006A3E0940040087BFF7A50798052
:10D75100800F128E60128DEA128E397BFF7A50791A
:09D76100877F0212D2B5C2172223
:10D1EB0090245CEFF0A3EDF030195912DF57EF608C
:10D1FB005390245CE07007A3E0D39400400B7BFFBB
:10D20B007A50798E12DBAF8010128E60128DEA127B
:10D21B008EF97A50799812D496901537128DFFECBF
:10D22B004D4E4F600330150C128DE0128EF97A5073
:10D23B0079A2800A128DE0128EF97A5079AD12D450
:05D24B009612DF152220
:1091550090248E128E309024A11220510000000020
:109165009024A512205100000000E4FF12D31990AD
:1091750026E8E07002A3E07008128E217401121C2B
:10918500B19026E8E0FEA3E0FFC39026EBE09FFF49
:109195009026EAE09E90249DF0A3EFF07F0112D384
:1091A500199026E8E07002A3E07008128E21740180
:1091B500121CB19026EAE0FEA3E0FFC39026E9E089
:1091C5009FFF9026E8E09E90249FF0A3EFF0128E7B
:1091D50021121C49703590249D128ED9C004C005FA
:1091E500C006C00790249F128ED99024AD128EA67A
:1091F5009024B1C9128E31D007D006D005D0041203
:10920500CD2E902494128E24121F7F901537128D27
:10921500FFEC4D4E4F601D12D9809024A1122045C0
:1092250012D43B9024AD1220459024A1128DFF123B
:10923500DAC18010E4FBFA79C87842901558128D8E
:10924500FF12176090248E128E24121F7F128E211A
:10925500121C49704112D43BC004C005C006C007AA
:1092650090248E128E24121F2F9024AD122045902B
:109275002494128E24121F2F9024B1128EA69024AE
:10928500B5C9128E31D007D006D005D004128C1482
:109295009024A51220459024A5128DFF128EA99029
:1092A50024B0C9128E31902497128EAC9024B3C984
:1092B500128E31902491128E24128287902491125D
:1092C5008E24121F2FE4FBFAF9F81217FD602540D2
:1092D50023902491128E24121F2F7B507AC2794C31
:1092E50078BD1217FD500D902491128E2412208204
:0592F500000000002252
:10D7FA0090245C12204512D43B7B337A9379887843
:10D80A0043121566C004C005C006C00790245C1206
:10D81A008DFFA804A905AA06FB121657D003D00249
:10D82A00D001D0001217607B337A93799278431231
:06D83A00165712C3242260
:10A5D70090245BEFF0ED600302A6989026C9F0A3E4
:10A5E700F012E077BF0904D2138002C213301303BD
:10A5F70012000712D43B9026E412204512CA82ACFF
:10A6070006AD07EC121880902740122045E4FFFEA4
:10A61700FD7CC7902740128DEA1217FD7004C21403
:10A627008011D214902740128DFF128F8E902740F1
:10A6370012204590245BE0B402097FC87E0012DE39
:10A647009C803F9024917401F0A37426F074CB1280
:10A657008F867426F074D6128F867426F0A374CA78
:10A66700128F877426F0A374C9F07B017A2679E0EC
:10A677001291559026D6128DFF12D7FA9026D61230
:10A68700204530130C12DC369026DC1220451200D0
:10A697000690245BE014602914602E14603824F6B9
:10A6A700603C146040240E7044128F25128DEA120C
:10A6B70017FD500512B94D8034128E831272CB806C
:10A6C7002C128E8312753A8024301405129C9180C7
:10A6D7001C12C9EE8017128E8312D721800F128E9B
:10A6E70083E4FB8005128E837B011250BC9015BB5F
:10A6F700128DFFEC4D4E4F6006128E8312D1EB2266
:10D43B00E49024ECF0A3F09026CFE0D394004002CC
:10D44B00804412C82B9024ECEEF0A3EFF0EE339552
:10D45B00E0FDFC7B007A8079FF78FFC3121F087018
:10D46B000C9026D012205100000000800F9024EC6D
:10D47B00128F15128F8E9026D0122045C2A990269E
:0BD48B00CF7428F0D2A9A3128DFF225D
:10D980009014B3128DFFEC4D4E4F6008E4FFFE7D06
:10D99000207C4122E4FF12DDC4AC06AD07E412187E
:10D9A00080901348128DEA1215667B367A94795767
:06D9B000783C121657221C
:10949B009024D61220459024DA128DEAE4FFFE7D4B
:1094AB00807C3F1215629024DE128DEA12156290B9
:1094BB0024E21220457FFC7EA97DEA7C419024DECC
:1094CB00128DEA121657C004C005C006C0077F48AC
:1094DB007E507DA57C419024DA128DEA121657D06E
:1094EB0003D002D001D000121566C004C005C0061F
:1094FB00C0077F817E957DE87C419024E2128DEA46
:10950B00121657D003D002D001D00012156690244A
:10951B00EA1220457F5E7EBA7DA77C419024DE1245
:10952B008DEA121657C004C005C006C0077F4D7EDA
:10953B00847D577C419024DA128DEA121657D003A2
:10954B00D002D001D000121566C004C005C006C001
:10955B00077F217EB07DA57C419024E2128DEA121B
:10956B001657D003D002D001D0001215669024EE0E
:10957B001220457F8B7EFD7DFF7C419024DE128D7A
:10958B00EA121657C004C005C006C0077F4D7E15F2
:10959B007D807C409024DA128DEA121657D003D0CE
:1095AB0002D001D000121566C004C005C006C0076A
:1095BB007FB87E407DE17C419024E2128DEA121649
:1095CB0057D003D002D001D000121566AB07AA0604
:1095DB00A905A804E4FFFE7D7A7C441217607B1476
:1095EB007A08790578411216579024E61220459097
:1095FB0024EE128DEA9024EA128DFF12176090244C
:10960B00E6128DEA121657C004C005C006C0077FCC
:10961B00337E937D887C439024D6128DEA12156697
:0F962B00D003D002D001D00012165712C3242250
:108C14009024A91220459024B8122051BD23D70ACC
:108C24009024BC1220513F851EB89024C0122051BC
:108C34003C23D70A9024C0128DEA9024B8128DFFE9
:108C44001215629024C41220459024C0128DFF9006
:108C540024BC128DEA1215669024C8122045902473
:108C6400CC122051BF8000009024D012205100006B
:108C74000000E49024D4F0A3F09024B5128E24E4F0
:108C8400121CB19024C8128DEA9024C4128DFF12D4
:108C94001562E4FBFAF9F81217FD9024C86013403A
:108CA40011128DEA9024C4128DFF12156212186AF3
:108CB400800C128DEA9024C4128DFF1215627B176A
:108CC4007AB779D178381217FD4003028D53902476
:108CD400D5E004F070069024D4E004F0D39024D5B9
:108CE400E094199024D4E094004003028D779024FA
:108CF400C8128DFF9024C4128DEA128F5A9024CC8E
:108D04001220459024CC128DFF9024DA1220459035
:108D140024AD128DFF9024DE1220459024A9128DDB
:108D2400FF12949B9024D01220459024B1128DFF01
:108D34009024D0128DEA1217FD9024CC128DFF508E
:108D4400059024C480039024C8122045028C879087
:108D540024B8128DFF9024CC128DEA1217FD401313
:108D64009024BC128DFF9024CC128DEA1217FD6062
:108D74001340119024B5128E247401121CB1E4FF27
:108D8400FEFDFC22E4FFFEFD7C3F9024CC128DEA24
:108D94001217FD9024CC600F400D128DFF7B6F7A6B
:108DA400127903783C8025128DEAC000C001C0020C
:108DB400C0037F6F7E127D837C3C9024CCA3A3A34D
:108DC400E0121657D003D002D001D00012156690DD
:0C8DD40024CC1220459024CC128DFF22EC
:10D9B6009024BC1220459024DA1220510000000069
:10D9C6009024DE1220513E570A3D9013AB128DFF74
:10D9D60012949B901369128DEA1216579024BC126A
:06D9E6008DEA1217602219
:10D9EC009024BC1220459024DA1220510000000033
:10D9FC009024DE1220513E570A3D9013AB128DFF3E
:10DA0C0012949B90138A128DEA1216579024BC1212
:06DA1C008DEA12176022E2
:10CD2E0012D9B69024B41220459024AD128DFF1264
:10CD3E00D9EC9024B81220457FCD7ECC7D8C7C3FE3
:10CD4E009024B4128DEA1216579024B8128DEA125E
:10CD5E0017FD6002501E7FCD7ECC7D8C7C3F9024D3
:10CD6E00B8128DEA1216579024B4128DEA1217FDDE
:10CD7E00600C400A9024B1128E2474018007902416
:10CD8E00B1128E24E4121CB19024B8128DFF90249F
:08CD9E00B4128DEA128F5A2233
:10DAC1009024A9122045901327128DFF9024A912AA
:10DAD1008DEA121657901306128DEA1215669024DC
:10DAE100A9128DEA1216579012E5128DEA121566E7
:01DAF1002212
:10DC36007F0312DDC4AC06AD07E4121880901471A0
:10DC4600128DEA121562901492128DEA1216577B03
:0BDC5600007A5079C378471217602253
:10DC8B000000000000000000000000000000000089
:10DC9B000000000000000000000000000000000079
:0ADCAB00000000000000000000006F
:10007600C117C118647408340000000000000000B5
:10008600000000000000BE000000000000000000AC
:1000960000181800000000000000000028FE28FEDE
:1000A60028000000000000000854FE542000000054
:1000B60000000000C62610C8C600000000000000B0
:1000C6006C92AC40A00000000000000000000E0092
:1000D600000000000000000000384482000000001C
:1000E600000000000082443800000000000000000C
:1000F60054381038540000000000000010107C1026
:1001060010000000000000000000C04000000001D8
:100116000000000010101010100000000000000089
:1001260000C0C0000000000000000000C020100851
:1001360006000000000000007CA2928A7C000000FD
:10014600000000008884FE8080000000000000009F
:10015600C4A292928C000000000000004282929A93
:100166006600000000000000302824FE2000000089
:10017600000000005E928A8A720000000000000003
:1001860078A49292600000000000000002C2221AC9
:1001960006000000000000006C9292926C000000C5
:1001A600000000000C92924A3C0000000000000093
:1001B60000CCCC0000000000000000000008DC4875
:1001C600000000010000000000102844820000002A
:1001D6000000000028282828280000000000000051
:1001E6000082442810000000000000000402B20A49
:1001F60004000000000000007C82B2AA1C0000007F
:1002060000000000F8242224F8000000000000008E
:1002160082FE92926C000000000000007C828282C6
:10022600440000000000000082FE82827C00000084
:1002360000000000FE929292820000000000000082
:10024600FE12121202000000000000007C8282A250
:100256006400000000000000FE101010FE00000008
:10026600000000000082FE82000000000000000086
:100276004080827E0200000000000000FE1028443C
:100286008200000000000000FE80808080000000E8
:1002960000000000FE081008FE000000000000003C
:1002A600FE081020FE000000000000007C82828212
:1002B6007C00000000000000FE1212120C0000007C
:1002C600000000007C82C2827C0000000000010069
:1002D600FE1232528C000000000000004C929292F6
:1002E60064000000000000000202FE02020000009E
:1002F600000000007E8080807E000000000000007C
:100306000E7080700E00000000000000FE403040BD
:10031600FE00000000000000C6281028C6000000ED
:10032600000000000608F0080600000000000000BB
:10033600C2A2928A860000000000000000FE8282AF
:100346000000000000000000040890A0C0F00000BB
:1003560000000000008282FE000000000000000095
:10036600080402040800000000000000000000006D
:10037600000002020202020020905020000001014B
:100386000101000040A8A8A8F0000000000000003D
:10039600FE50888870000000000000007088888881
:1003A600500000000000000070888850FE00000029
:1003B6000000000070A8A8A830000000000000009F
:1003C60010FC1212040000000000000030484848EB
:1003D600F800010202020100FE100808F000000009
:0D03E600000000000088FA80000000000008
:1003F30000000000800008FA00000102020100FE74
:1004030020205088000000000000000082FE8000D1
:1004130000000000000000F8087008F00000000071
:10042300000000F8100808F0000000000000007051
:100433008888887000000000000000F850888870E9
:100443000003000000000070888850F800000000DE
:10045300000300F8100808100000000000000090DE
:10046300A8A8A84000000000000000087E8888407B
:100473000000000000000078808040F800000000C9
:100483000000001860806018000000000000007881
:1004930080608078000000000000008850205088B1
:1004A3000000000000000038404020F80001020274
:1004B30002010088C8A8988800000000000000BC62
:1004C300C202C2BC000000000000000000FE0000E9
:1004D3000000000000000000FC0303FC0000030414
:1004E300040300000C12120C000000000000006066
:1004F300D202F8F0FCFE0E0707070707070EFEFC03
:10050300F00080C0E0F0783C1E0FFFFFFF0000709A
:100513007C7E0E0707070707070EFEFCF0707C7E44
:100523000E0707070707070EFEFCF0000000008018
:10053300E0F87E1F0701000000FFFFFF0707070722
:1005430007070707070707F0FCFE0E07070707075C
:10055300070E7E7C7007070707070707070787E76C
:10056300FF7F1FF0FCFE0E0707070707070EFEFCC1
:10057300F0F0FCFE0E0707070707070EFEFCF0006E
:100583000000000000000000000000000000000068
:100593000000000000000000000000000000000058
:1005A3000000000000000000000000000000000048
:1005B3000000000000000000000000000000000038
:1005C300000000000060D20226FFFFFF00000000D1
:1005D30000000000FFFFFF00070301000000000010
:1005E300FFFFFF00000000000080C0E0F0783C1E29
:1005F3000F070300000000001C1C1C1C1C3EFFF71F
:10060300C180E0F87E1F070100F0F0F00000001F3A
:100613001F1F1C0E0E0E0E0E0E1CFCF8E0FFFFFF3C
:10062300381C1C1C1C1C1C38F8F0C0000000000007
:1006330080E0F87E1F07010000C1F7FF3E1C1C1C71
:100643001C1C1C3EFFF7C1070F1F1C3838383838F5
:10065300381CFFFFFF000000000000000000000046
:100663000000001C1C1C1C1C1C1C1C1C1C1C1C1C1B
:100673001C00000000000000000000000000003E1D
:100683004141413E0090C8A890000000007F080847
:10069300087F00385454541800000060D201540FEE
:1006A3003F7F70E0E0E0E0E0E0707F3F0F0000009C
:1006B300000000000000FFFFFF0000F8FCFEEFE772
:1006C300E3E1E0E0E0E0E0E0E00E3E7E70E0E0E069
:1006D300E0E0E0707F3F0F0707070707070707FF03
:1006E300FFFF0707070E3E7E70E0E0E0E0E0E0700A
:1006F3007F3F0F0F3F7F70E0E0E0E0E0E0707F3F7F
:100703000F0000E0F8FE1F07010000000000000FCB
:100713003F7F70E0E0E0E0E0E0707F3F0F0E3E7E61
:1007230070E0E0E0E0E0E0707F3F0F0000000000D9
:10073300F0F0F0F0000000000000000000000000F6
:1007430000000000000000000000000000000000A6
:100753000000000000000000000000000000000096
:0D0763000000000000000000000000000089
:10077000000000004103CA014100810041008000E7
:0407800041111C0007
:10A36900121C49FF902521E0FBA3E475F001121DA1
:10A3790043A9F0FA22E0FF902513E0FD75F015A43A
:10A3890024CBF582E43403F583E5822FF582E435A5
:10A3990083F583E0FC902515F0ED75F015A424EB09
:10A3A900F582E43400F583E5822FF582E43583F5FF
:10A3B90083227401F0A3EAF0A3E9F0902517E004E1
:10A3C900F090251675F080A42434F9740435F0FA58
:10A3D900E07E0029F9EE3AFA227E007F697D207B32
:10A3E900017A0379CB1221BB7A0079EB7E007F6970
:10A3F9007D207B010221BB3EFA9025217401F0A347
:10A40900EAF0A3E9F022E0FB902577E0FEA3E0FF64
:10A419007C007D08021CF77D017B017E007F6912AB
:10A429001C239003CA7401F022902515E0FF9025A2
:10A4390014E0FE902513E075F015A424EBF582E4F1
:10A449003400F583E5822E2290256DE0FBA3E0FA26
:10A45900A3E0F922EF121CB1902524E004F0E022D8
:10A46900902518E4F0A32290256CE075F015A4243A
:10A47900B6F9740335F02274342DF58274083CF56D
:10A4890083E0C4222434F58274043EF583229025A6
:08A4990015E0FFEEFB7A002242
:10A95D00902516EDF0EB75F006A4A3F0ED75F00C57
:10A96D00A4131313541FA3F0EF3395E0FE74002FBF
:10A97D00F58274003EF583E0FF7E00902519EEF020
:10A98D00A3EFF07C007D0C121CE5902519EEF0A3D1
:10A99D00EFF0902518E090251712A3CD90251B12EE
:10A9AD00A405902518E004F075F080A42434F97402
:10A9BD000435F0FA90251712A3D990251E12A4057F
:10A9CD00902516E030E058902519E0FEA3E024A86C
:10A9DD00F9740C12A400E4A3F090251B12A45412D8
:10A9ED001C49540F121CB190251B12A370C003C03B
:10A9FD0002C00112A369121C494FD001D002D0032D
:10AA0D0012A45EB406D3E4902524F012A36D121C9B
:10AA1D0049FF90251E12A37012A45DB406ED22907D
:10AA2D002519E0FEA3E02434F9740812A400E4A370
:10AA3D00F012A36D121C49FF90251B12A37012A4D6
:10AA4D005DB406EDE4902524F090251E12A4541259
:10AA5D001C4954F0121CB190251E12A370C003C0E6
:10AA6D0002C00112A369121C494FD001D002D003BC
:07AA7D0012A45EB406D3220F
:10B5C700EB75F014A4902516F0ED7004A3F0800637
:10B5D7009025177404F0EFB42E0812A469748CF048
:10B5E700804CEFB42D0812A469749AF08040EFB430
:10B5F700200812A46974A8F08034EFB44F0812A48D
:10B607006974B6F08028EFB4480812A46974C4F0CE
:10B61700801CEF3395E0FEEF24D0FFEE34FFFE7C75
:10B62700007D0E121CE5902518EEF0A3EFF0902593
:10B6370017E012A3CA90251A12A3BB90251D12A3C7
:10B64700BB90252012A405E4FF902519E024F8F506
:10B6570082E43402F583E0FE90251A12A370EE12FD
:10B667001CB1902519E02426F582E43402F583E025
:10B67700FE90251D12A370EE121CB1902518E475DB
:10B68700F001121D43FC745425F0F58274013CF55A
:10B6970083E0FE90252012A370EE121CB10FEF6419
:04B6A7000E70A62259
:06E09000EF908000F02279
:10CC2C00902576EFF0A3ECF0A3EDF0EB603812A4B6
:10CC3C0011EF7807C333CE33CED8F912A48DC0834D
:10CC4C00C082902576E0D082D083258212A3B3C017
:10CC5C0083C08212A40FAF057401A807088002C319
:10CC6C0033D8FC4B803712A411EF7807C333CE3383
:10CC7C00CED8F912A48DC083C082902576E0D082E4
:10CC8C00D083258212A3B3C083C08212A40FAF0538
:10CC9C007401A807088002C333D8FCF45BD082D09F
:03CCAC0083F022F0
:10DC610005A290043405A27B007C0890800074B06A
:10DC71002B0BF07410F07400F07D8090800105A2F0
:0ADC8100E0A305A2F0DDF7DCE222CB
:10D88500E4FFE4FE75F080EFA42434F582E5F0347E
:10D8950004F583E5822E12A3B3E4F00EEEB480E422
:10D8A5000FEFB408DD7B007C0890800074B02B0B73
:10D8B500F07410F07400F07D809080017400F0DD4C
:04D8C500FDDCE6227E
:10C1BF007FE212E0907F2F12E0907F2412E0907FB9
:10C1CF00AF12E0907FA612E0907FC812E0907F81BF
:10C1DF0012E0907F3812E09012D88512A3E27E0011
:10C1EF007F207DFF7B017A0079001221BB7F20EF3A
:10C1FF0024E0FE74002FF582E43400F583EEF00F97
:10C20F00EFD3947F40E990007F74FFF0E4FDFCE4EE
:10C21F00FF12A48054F0FE74A82DF582740C3CF527
:10C22F0083EEF0743A2DF58274083CF583E0C45424
:10C23F00F0FE12A480540F4EFE74AE2DF582740CD6
:10C24F003CF583EEF00DBD00010C0FEFB406C27488
:10C25F00062DFDE43CFCC3ED9474EC6480948440A3
:02C26F00AE22FD
:10DFDF00C3EE648094814003C29422D2948FFB22BB
:0AE063007FAE12E0907FA502E0906E
:10C47700AA07900080E075F006A4FF902570E5F00C
:10C48700F0A3EFF0900081E075F00CA4240AFFE41C
:10C4970035F0FE902572F0FCA3EFF0FD902571E0DA
:10C4A700FFAB0212CC2C902571E02405A312C50E18
:10C4B700902573E004F07006902572E004F0902553
:10C4C70070E0FFA3E0902574CFF0A3EFF090257103
:10C4D700E02406FF902570E03400FEC3902575E048
:10C4E7009FEE6480F8902574E06480985018A3E06C
:10C4F70090257212C50E902575E004F070CF902537
:10C5070074E004F080C722FFE0FCA3E0FDAB021259
:03C51700CC2C2207
:10C51A009003CAE0700302C5B8301841E4902513AD
:10C52A00F0E4902514F0902514E0FEC39406501E02
:10C53A0012A37EE06C600E12A49712B5C712A43241
:10C54A0012A3B3EFF0902514E004F002C530902551
:10C55A0013E004F0E0C3940240C702C5A5E49025A5
:10C56A0013F0E4902514F0902514E0FEC3941550BE
:10C57A001E12A37EE06C600E12A49712A95D12A48B
:10C58A003212A3B3EFF0902514E004F002C57190C3
:10C59A002513E004F0E0C3940540C790111CE06045
:0FC5AA00057F0112C47712DC61E49003CAF0220E
:10CFDE0090256CEFF0A3EB12A407A217301801B343
:10CFEE00500D12A3E212DF8112D885A21792187E7D
:10CFFE00007F15C006C0077D2012A470FA7B01D0F9
:10D00E0007D0061221BB12A45112DF6CD3EF941578
:10D01E00EE6480948040067E007F15800612A45137
:10D02E0012DF6CC006C00712A470A801FC7D01A31C
:0BD03E0012A454D007D00612A4282230
:10D2B500902513EFF0A3EB12A407783F7C257D01A1
:10D2C5007BFF7ADC798B7E007F2A121C23902569EF
:10D2D5007401F0A37425F0A37417F0902514E0F9F8
:10D2E500A3E0FAA3E090258CC912A407902569E074
:10D2F500F9A3E0FAA3E090258FC912A4077B017A70
:10D3050025793F12D6D7902513E0FF7B017A257941
:04D315003F02CFDE26
:10DAF2009024DBECF0A3EDF0A90790111CE0600587
:10DB0200E4FF12C47790111C7401F09024DCE0143D
:10DB1200900080F0E914A3F07F0112C47712A42BC5
:01DB220022E0
:10DF810090111CE06008E4FF12C47712A42BE49006
:04DF9100111CF0224D
:0EDFFD007A0379CB12A3F512DF8112A42B2236
:0CE0340078827C007A0379CB12A42022B1
:0CE0400078CB7C037A00798212A42022A5
:10B2F0002573002530352E31662025252020257325
:10B30000002530352E3166202525002043616C69EB
:10B3100062726174696F6E2061626F72746564201D
:10B3200000252D3037732025352E3166206D5600CF
:10B330002025352E316625732020253673007E4664
:10B34000007E4300535441424C45002025352E31A8
:10B35000662573202025332E316600506F696E7488
:10B360002031004149520043414C3100506F696E19
:10B370007420320043414C3200506F696E742033A8
:10B380000043414C330025362E3366206D73202553
:10B39000362E3366206D730025352E3266257300F8
:10B3A00025362E336620574149540000000000C95D
:10B3B0007423F000000000000000000000C97423A6
:10B3C000F000000000000000000000C97423F0003D
:10B3D000000000000000000000C97423F00000001D
:03B3E0000000006A
:100784004228150000602827ED3120706F696E74CF
:100794002063616C2E003220706F696E7420636177
:1007A4006C2E003320706F696E742063616C2E00B0
:0107B4000044
:108FAC00902470E0F8A3E0F9A3E0FAA3E0FB121719
:108FBC006090130612204590245CE0FCA3E0FDA316
:108FCC00E0FEA3E0FF22E0F8A3E0F9A3E0FAA3E0BF
:108FDC00FB12165790246CE0F8A3E0F9A3E0FAA377
:108FEC00E0FB22902815E0FEA3E0FFE4FCFD9024BA
:108FFC0088E0FBA3E0FAA3E0F922902815E0FEA399
:10900C00E0FFC3EF9BFFEE9AFEE499FDE498FCE4CD
:10901C007B19FAF9F8121DDDE412187BE4FBFA79DE
:10902C007A7844121760A804A905AA06AB0722F0A7
:10903C00902457E0FCA3E0FDE41218807BE37A381F
:10904C00790E783A021657E4FBFA79107841121629
:10905C0057E4FBFA79A07840121760E4FBFAF97830
:10906C0042021566EB90251BF0A3EAF0A3E9F0226F
:10907C0090247CE0FCA3E0FDA3E0FEA3E0FBAA06A9
:10908C00A905A80422121FF5902815E0FEA3E0FF05
:10909C00C322C2A9D211901CA77428F0D2A9227D98
:1090AC00017BFF7E007F0E021C23902517022045BA
:1090BC00122045E4FBFA79C8784222900004122071
:1090CC001590248422EF9BFFEE9AFEE499FDE49820
:1090DC00FCE422EF9BFFEE9AFEE499FDE498FCE49D
:1090EC0022C2A9C211D2A922902462E4F0A3F0A357
:1090FC00F022E0F9A3E0FAA3E022121562E4FBFAF5
:10910C00F9F80217FDC2A9E4902815F0A3F0D2A932
:10911C002290245B74FFF0A32290245B7401F0A3D3
:10912C0022A3F0A37401F0A322C3902457E064801F
:10913C0022EFF0901CA8E022EC4D4E4F7BFF2290CA
:09914C00247012204590247022C9
:106DDA00902458EB129074121F2F902465122045AC
:106DEA009024691220513DCCCCCD90246D7409F0C9
:106DFA00E4A3F0A3F0A312205100000000E49024C1
:106E0A0074F0A3F0601390246FE024FEFF90246EC8
:106E1A00E034FFFEFCAD0780087EFF7FFF7CFF7D2C
:106E2A00FF12703D12204590245B1290FE902517A8
:106E3A00C91290747BFF7AB279F07F0112D2B53011
:106E4A000F0302703912C51A1292FA12C2719024F3
:106E5A006D12913D7004A3E06401701220110512B5
:106E6A00909E800D901CA7E07007D20F80031290AD
:106E7A00ED90246DE024FEB407004003026FC49035
:106E8A006E9775F003A4C58325F0C58373026F5E00
:106E9A00026F8A026F39026F65026F0F026EAC02CF
:106EAA006F7390246FE004F0700690246EE004F093
:106EBA0090246EE07004A3E06401700E90246FE0E9
:106ECA0004F0700690246EE004F0D390246FE094EE
:106EDA000390246EE0648094804004E4F0A3F09070
:106EEA00246EE0FEA3E0FF4E600DEF24FEFFEE34B9
:106EFA00FFFEFCAD0780087EFF7FFF7CFF7DFF124F
:106F0A00703D026F6E902465128FC6A3128FE31232
:106F1A0015661290BF1217FD5003026FC4902465C4
:106F2A00128FC6A3128FE3121566902465803590DE
:106F3A002469128FE3902465128FC61291066002AB
:106F4A005078902465128FC6A3128FE312156290AF
:106F5A002465801012DFFDE4FEFF2290245E128F6A
:106F6A00C69024651220458051902465128FC690E0
:106F7A002458128FFD121F7F12DFFD7E007F01222F
:106F8A00902474E0FAA3E0FB4A6005902470800F15
:106F9A00902465128FC690247012204590245E12A8
:106FAA008FC6902465122045EB4A70047F01800247
:106FBA007F00902474E4F0A3EFF0902462E0FBA336
:106FCA00E0FAA3E04A4B603E90245E128FE39024DD
:106FDA0065128FC6121562E4FBFA792078411216FF
:106FEA00571218B912DFCDEF4E701B902465128F1D
:106FFA00C61290B69024621290FEC91290717BFF5D
:10700A007AB279F3800F7BFF7AB379019024651203
:10701A008FC61290B67F0312D2B590246E12909743
:10702A0074059FFDE49EFC7F0312DAF2026E491298
:10703A00DFFD22EC12188090247A1220457F007E10
:0C704A00007D207C41129F84902469226C
:10963A00902484122045902488EB129074C20190E1
:10964A0024971220510000000090249B1220510000
:10965A00000000128FFA900004121F4F7BF07A2349
:10966A00797478C91217FD701BC201128FEF121F8D
:10967A007F902484128FC6A3128FFD900004121FBC
:10968A00990297BF128FFA1290911290D17B19FA10
:10969A00F9F8121DDDE412187B902493128FE3125D
:1096AA0017FD60144012128FFA90000C121D5945D2
:1096BA00F024FF92010297BFE4FFFEFDFC90248B89
:1096CA00128FE31217FD7003029799128FFA129004
:1096DA00C7128FC612910690248860134011128F08
:1096EA00FD1290C7128FC612156212186A800C12E8
:1096FA008FFD1290C7128FC6121562C004C005C032
:10970A0006C007128FFA1290911290D112187B128A
:10971A009032D007D006D005D00412176090249753
:10972A00122045E4FFFEFDFC90248B128FE31217F2
:10973A00FD90248B128FC6500512186A8000E4FB34
:10974A00FA79C87841121657C004C005C006C00786
:10975A00E4FFFE7D7A7C4490248F128FE312165721
:10976A00129032D007D006D005D004121760902488
:10977A009B12204590249B128FC6902497128FE348
:10978A001217FD60025003D38001C392018002D2F6
:10979A0001128FEF121F7F902484128FC6A3128F9B
:1097AA00FD900004121F99A201E4FF3390000CCF30
:1097BA008FF0121DB020010D128FEF900008121FBA
:0A97CA0099E4FEFF227E007F0122D9
:10DF950012DFFD7BFF7AB3790B7F0312CFDE12C54B
:04DFA5001A02D90D76
:107C2400902458EB129074C20078667C247AB3795D
:107C3400AB1290AB78747C247AB379B91290AB12FE
:107C44009111300F03027E3D12D9809024611220DD
:107C54004512D43BC004C005C006C0077B017A248A
:107C6400796690248B1220513F80000090248F125B
:107C740020513F800000902493122051447A000048
:107C8400D007D006D005D00412963AEF4E60627B3E
:107C9400017A24797490248B1220514120000090A1
:107CA400248F1220513F80000090249312205142CF
:107CB400C80000902461128FC612963AEF4E6031CC
:107CC40090247C128FC690246E128FE3D3121F1E51
:107CD400400990246EE0FCA804800312907C12906A
:107CE400941290DF7BC8FAF9F8D3121F1E50028059
:107CF40001C392009024581290FE902517C9129047
:107D040074902461128FC690251A1220457BFF7A45
:107D1400B379217F0112D2B5300047901976128FC2
:107D2400C6EC4D4E4F600812D43B129053800312A0
:107D3400D43B1290B6901976128FC6129144600605
:107D44007AB3793E80047AB37941129070A374FFB8
:107D5400F0A374B3F0A37444F07BFF7AB3793002D8
:107D64007DCF901976128FC6EC4D4E4F600812D419
:107D74003B129053800312D43B1290B690197612A2
:107D84008FC612914460067AB3793E80047AB3793F
:107D94004112907090247C128FC690246E128FE34F
:107DA400D3121F1E400990246EE0FCA80480031225
:107DB400907C129006E4FFFE7DA07C401215629038
:107DC400251E1220457BFF7AB3794B7F0212D2B570
:107DD40012C51A1292FA12C27190246512913D7062
:107DE40004A3E06401701220110512909E800D908E
:107DF4001CA7E07007D20F80031290ED902465E079
:107E0400B4020A12DF9512DFFDE4FEFF229024651E
:107E1400E064086003027C46200003027C46902450
:107E240061128FC690245B128FFD121F7F12D43B08
:107E340090245E128FFD121F7F12DFFD7E007F01F2
:017E4400221B
:10705600E4902455F0A3F0FFFE7D807CBF90117A6A
:10706600128FE31215661218B9902457EFF0300FFD
:10707600030272B5902455E0B4070040030271E79D
:1070860090708DF82828730270A202710702715F52
:107096000271BF0270D40271370271929024971266
:1070A60090F77B01A304F0A37424F0A37456F0A315
:1070B600EBF0A37424F0A37457F07A2779ED7D03DF
:1070C6007C00129B069024557404F00271ED129117
:1070D6001D74B3F0A3745BF0A312205141A8000005
:1070E60090246274FFF0A374B3F0A37463F07A1172
:1070F600799B1272B87004F00271ED7401F002719E
:10710600ED1291257411F074BC12912D7411F0A337
:1071160074DDF07AB379671272C3700280561291E9
:1071260035948190245540067405F00271ED027184
:10713600EA12911D74B3F0A3746CF0A312205142AD
:10714600C800001290F47A1179FE1272B87004F039
:107156000271ED7402F00271ED1291257412F07451
:107166001F12912D7412F0A37440F07AB379741241
:1071760072C37007902455F00271ED129135948216
:1071860090245540057406F0805D805812911D7458
:10719600B3F0A37479F0A3122051000000001290FE
:1071A600F47B017A127961126DDAEF4E90245570F4
:1071B60003F080337403F0802E1291257412F0A32D
:1071C600748212912E7412F0A374A3F07BFF7AB32B
:1071D6007981127C24EF4E9024557003F08008804C
:1071E600039024557407F012C51A1292FA12C2714E
:1071F600901CA8E07004A3E064017012201105122F
:10720600909E800D901CA7E07007D20F800312900D
:10721600EDEF640270030272B5902457E0FFC36479
:1072260080948050030272B5902455E06407600391
:10723600027074EF701490121F12205100000000AB
:1072460090124012205100000000D3129136948112
:107256005014901282122051000000009012A312C6
:10726600205100000000902457E0FF3395E0FEEF28
:107276002401FDE43EFC12188090117A12204590FC
:10728600119F7401F09011C0F09011E1F09012027C
:10729600F0901223F0901244F0901265F09012864E
:1072A600F09012A7F090117EF0123F6E12DFBB0233
:1072B600DFFD7B01126DDAEF4E902455227BFF1223
:0572C6007C24EF4E22C4
:106B270090245B7409F0C200A312205100000000FA
:106B37009024601220510000000078647C247D01BD
:106B47007BFF7AB379C71290AF78727C247D017B83
:106B5700FF7AB379D51290AF12911190245BE0645C
:106B6700027003026DD9300F03026DD9E4FF12D30F
:106B7700199026E81290979026EBE09FFF9026EA5F
:106B8700E09E902457F0A3EFF07F0112D3199026CF
:106B9700EA1290979026E9E09FFF9026E8E09E9002
:106BA7002459F0A3EF12903B1290B69024591290FB
:106BB7003F90251B1220457BFF7AB379867F011210
:106BC700D2B5901976128FC6EC4D4E4F600812D48D
:106BD7003B129053800312D43B1290B69019761251
:106BE7008FC612914460067AB3793E80047AB379EE
:106BF700411290707BFF7AB379987F0212D2B51257
:106C0700D43BC004C005C006C0077B017A24796461
:106C170090248B1220513F80000090248F12205126
:106C27003F800000902493122051447A0000D0073F
:106C3700D006D005D00412963AEF4E7003026CE2EC
:106C4700902459E0FEA3E0FF902458E02FFF902402
:106C570057E03EC313FCEF13FDE4121880C004C0D5
:106C670005C006C0077B017A24797290248B122015
:106C7700510000000090248F1220513F80000090A7
:106C8700249312205141200000D007D006D005D010
:106C97000412963AEF4E604390247A128FC69024DE
:106CA7006C128FE3D3121F1E400990246CE0FCA8DE
:106CB70004800690247A12907F1290941290DF7BC2
:106CC700407A01F9F8D3121F1E5010D2007BFF7AC9
:106CD700B379447F0312CFDE026D2B90247A128F93
:106CE700C690246C128FE3D3121F1E400990246CA8
:106CF700E0FCA804800690247A12907F129006E4A4
:106D0700FFFEFD7C41121562902480122045C200CF
:106D17007BFF7AB379A0902480128FC61290B67F3A
:106D27000312D2B512C51A1292FA12C27190245BDD
:106D370012913D7004A3E0640170122011051290B6
:106D47009E800D901CA7E07007D20F80031290ED74
:106D570090245BE0FF64026079EF640870453000BF
:106D6700429013CC1220513F8000009013D0740141
:106D770012903B90136912204590136D7401F090A7
:106D8700245912903F90138A12204590138E740154
:106D9700F012D43B9013AB1220459013AF7401F05F
:106DA70002DFBB90245BE064056003026B629028FE
:106DB70015E0FAA3E0FBFFAE02E4FCFD90247A1293
:106DC7002045AF03AE02E4FCFD90246C122045027F
:036DD7006B6222CA
:103F6E001290BF90119B128FC61217609024581298
:103F7E0020459011BC128FC690245C1290BC9011FB
:103F8E00FE128FC612176090246012204590121FE9
:103F9E00128FC69024641290BC901261128FC612BA
:103FAE001760902468122045901282128FC69024BA
:103FBE006C1220459012E512205100000000901363
:103FCE00061220510000000090132712205100000D
:103FDE0000009012C4122051000000009012E974EB
:103FEE0001F090130AF090132BF09012C8F090117C
:103FFE007A128FC61218B9EE60030243E4EF24FE64
:10400E00603A14700302409F240260030243E47F6F
:10401E00CD7ECC7DCC7C3D90245C128FE31217FDBF
:10402E00600250030243E490245C128FE390245804
:10403E00128FC61217609013060243D790245C129B
:10404E008FE3902464128FC612156212914B128F59
:10405E00C612E0277BCD7ACC79CC783D1217FD4085
:10406E00030243E4902458128FE3902460128FC60B
:10407E00121562128FAC901306128FE3121657129E
:10408E009032902458128FC61215629012E5024398
:10409E00D7128FE0128FC3121562C004C005C0067E
:1040AE00C007902464128FE3128FC3121562D003DF
:1040BE00D002D001D000121657C004C005C006C0F1
:1040CE0007128FE0902464128FC6121562D003D0AF
:1040DE0002D001D00012165712914B128FC612E069
:1040EE00277B6F7A127983783A1217FD40030243C9
:1040FE00E4128FC312E04CC004C005C006C0079086
:10410E002468128FC612186AD003D002D001D000D4
:10411E00121657902464128FE3121657C004C0056E
:10412E00C006C007902464128FC612E04CC004C0B3
:10413E0005C006C007128FC3902468128FE31216B3
:10414E0057D003D002D001D000121657D003D002A0
:10415E00D001D000121566C004C005C006C00712FB
:10416E008FC312E04C902460128FD2121657D003D8
:10417E00D002D001D000121566C004C005C006C022
:10418E0007902464128FC61243E5128FD21216576F
:10419E00129032D007D006D005D004121562C0049A
:1041AE00C005C006C00790246C128FC612E04CC02A
:1041BE0004C005C006C007128FC3A3128FE31216E8
:1041CE0057D003D002D001D000121657129032D021
:1041DE0007D006D005D004121562C004C005C00673
:1041EE00C00790246C128FC612E04CC004C005C0EC
:1041FE0006C007902464128FC6902458128FE312C3
:10420E001657D003D002D001D000121657D003D0CB
:10421E0002D001D00012156612186A902470128F07
:10422E00E31217609012E5128FC012E04CC004C06A
:10423E0005C006C007902460128FC612186AD003FC
:10424E00D002D001D000121657C004C005C006C05F
:10425E0007128FC312E04C902468128FE312165788
:10426E00D003D002D001D000121566C004C005C024
:10427E0006C007902464128FC61243E5128FE31214
:10428E001657D003D002D001D000121566C004C05C
:10429E0005C006C007902464128FC612E04C90240D
:1042AE0068128FE3121657129032D007D006D0053F
:1042BE00D004121562C004C005C006C00790246C5D
:1042CE00128FC612E04C902458128FE3121657121A
:1042DE009032D007D006D005D004121562C004C0AB
:1042EE0005C006C00790246C128FC612E04C9024B5
:1042FE0060128FE3121657D003D002D001D00012F5
:10430E00156612186A128FAC902468128FE312167B
:10431E0057C004C005C006C007128FC3A3128FE397
:10432E00121657D003D002D001D000121562C0046D
:10433E00C005C006C007902464128FC69024581280
:10434E008FE3121657129032D007D006D005D00444
:10435E00121562C004C005C006C007902464128FF7
:10436E00C6A3128FE3121657D003D002D001D0008D
:10437E00121566C004C005C006C00790246C128FCB
:10438E00C6902458128FE3121657D003D002D001D4
:10439E00D000121566C004C005C006C00790246C7C
:1043AE00128FC6902460128FE3121657129032D0DD
:1043BE0007D006D005D00412156212186A90247028
:1043CE00128FE31217609013271220459012C41219
:0E43DE0020513F8000002212E04C9024582213
:10ADC9000025303258253032582530325825303256
:10ADD90058253032582530325825303258004572BE
:10ADE900726F7220202020004169722020202020CB
:10ADF90020004F60202020202020200048652020AE
:10AE090020202020200025342E31662020202020DB
:10AE19000025342E31662F25342E31660045727295
:10AE29006F72004169722020004F60202020004885
:10AE3900652020200025322E306620202000253272
:10AE49002E30662F25322E3066004572726F7220C1
:10AE5900360045787465726E616C20706F77657223
:10AE6900006F766572766F6C746167652E002535A3
:10AE79002E31662056005761726E696E6700426115
:10AE89007474657279206C6F77005265706C6163B8
:10AE9900652039205620416C6B616C696E650062D2
:10AEA900617474657279206F72207573650031322F
:10AEB900205620444320706F776572206164617069
:10AEC900746F720000000000000000000000000024
:04AED9000000000075
:0507B5004228170000BE
:10B1F400A3F0902491E4FFFE7DC87C42E0F8A3E034
:10B20400F9A3E0FAA3E0FB2290259574FFF0A322B2
:10B21400E0902598FFE4F0A3EFF022902516E0FBE0
:10B22400A3E0FAA3E0F922E0FCA3E0A3FDE0FEA37F
:10B23400E0FF22E090259CFFE4F0A3EFF022E090F1
:10B2440025A0FFE4F0A3EFF022FFE4F0A3EFF02247
:10B25400EBF0A3EAF0A3E9F0221216579025980226
:10B264002045E09025A4FFE4F0A3EFF022FFE4F0F2
:10B27400A3EFF0227F0A7ED77DA37C3B227FF67E5C
:10B28400287D5C7C3E227FA47E707D7D7C3F2212E3
:10B2940015667BAE7A477981783F0217FDA3F0E407
:10B2A400FFFE7DC87C42228F82AF058F8375D20258
:10B2B40075A22022C2A9D211901CA77428F0D2A989
:10B2C40022901D51E04410F0908002F022901D5114
:10B2D400E054EFF0908002F0227D017BFFFE7F08B6
:0CB2E400021C2312165790259C022045E6
:0EE00B00E5D220E0FB12B2ABEBF0E4F5D2223E
:0EE01900E5D220E0FB12B2ABE0FFE4F5D2222C
:10DDC400901D51E054FBF0908002F0EF128B6DAF88
:10DDD400F0FD901D51E04404F0908002F0EFFEED60
:02DDE400FF221C
:10DE4400901D51E04410FFF0908002F0EF7F96DFC8
:0EDE5400FEFFEF54EF901D51F0908002F0227F
:10DD7D00E4902465F012B2C5128B22128B22128B05
:10DD8D002212B2D1128B22902465E004F0E0C394EC
:04DD9D00C040E2227E
:10DE6200E4902454F012B2C5128B2212B2D1128B5A
:0EDE720035902454E004F0E0C3943240E822DE
:10D8400090251612B254A3EDF0902519E0D3940060
:10D85000402F12B21F12DF6CEF2401FFE43E90252F
:10D86000178FF0121D2D902519E014F012B21F74BD
:10D87000FF90ADC96B7008E965827003EA6583703B
:05D88000C812B21F22D6
:10D94900FDE0FAA3E0FBEF4CFEEDFFEEA2E713FECC
:10D95900EF13C4F8540FC868FFEEC454F048FEEF43
:10D9690024FCFFEE34FFFEAD03C374109BCDE49A93
:07D97900CD2FFFED3EFE2261
:10C82B00128A4630D702805D74CC128A5E74441231
:10C83B008A5EC2D7128A4630D702804974CC128ADC
:10C84B005E74BE128A5E128B27E4F5F0128A779023
:10C85B0024EE12B24D128A779024F012B24D12C808
:10C86B00BC12C8BC128A779024F212B271128A776A
:10C87B009024F412B271A3E5F0F0128A779024F6AB
:10C88B00E0FF6F60057E807F0022C2B49024F0E051
:10C89B00FEA3E0FF9024EEE0FCA3E09024F212D97B
:10C8AB0049300B0CEF7803CEA2E713CE13D8F8FF69
:08C8BB0022128A77128A77220B
:10CA8200128A9330D702806374CC128AAD74441236
:10CA92008AADC2D7128A9330D702804F74CC128AE1
:10CAA200AD74BE128AAD128B27E4F5F0128AC690DD
:10CAB20024EC12CB0A9024EE12CB0A128AC6128AF6
:10CAC200C6128AC6128AC6FF9024F0E4F0A3EFF0E1
:10CAD200128AC6FF9024F2E4F0A3EFF0A3E5F0F08F
:10CAE200128AC69024F4E0FF6F60057E807F0022E8
:10CAF200D2B59024EEE0FEA3E0FF9024ECE0FCA38C
:10CB0200E09024F012D94922FFE4F0A3EFF0128A58
:02CB1200C62239
:10D5ED00E490244AF0A3F0A3F0128A46B3500F74CE
:10D5FD0033128A5EE4F5F0128A7790244CF0902471
:10D60D004CE064287026D20B901E3E7402F0128AF4
:10D61D004674CC128A5E744E128A5EE4128A5EE4FF
:0FD62D00128A5EE4128A5EC2D7128A46C2B42203
:0100060022D7
:0100070022D6
:10C8C30090246C12B254E4A3F0A3F078717C247A20
:10C8D300AE79CD12B2DD128A46B350317433128A67
:10C8E3005EE4F5F090246FE0C394085020128A7739
:10C8F300902470F0E0FF90246FE02471F582E4341B
:10C9030024F583EFF090246FE004F080D712B20C8B
:10C9130074ADF0A374CAF090247712B21490247605
:10C92300E090259A12B21890247512B237902474AD
:10C93300E090259E12B23B90247312B2429024726F
:10C94300E09025A212B24690247112B26690246C34
:06C9530012B222023B506B
:10C6F50090246C12B254E4A3F0A3F078717C247AF0
:10C70500AE79D512B2DD128A93B350317433128AE1
:10C71500ADE4F5F090246FE0C394085020128AC66A
:10C72500902470F0E0FF90246FE02471F582E434EA
:10C7350024F583EFF090246FE004F080D712B20C5B
:10C7450074ADF0A374CAF090247712B214902476D5
:10C75500E090259A12B26A90247512B2379024742B
:10C76500E0FF90259EE4F0A3EFF090247312B2420F
:10C77500902472E0FF9025A2E4F0A3EFF0902471DD
:0CC7850012B26690246C12B222023B50EB
:0BE05800EF7003C29322D2938FFA22D4
:10D31900E49024A9F0A3F07E01F5CDF5CCD2CAC2E0
:10D32900A8C2AA04A807088002C333D8FCFE901D2E
:10D3390051E04EFFF0908002F0EF7F32DFFEFFEE0A
:10D34900F45F901D51F0908002F0C289C28BD2AA7D
:10D35900D2A820A80330AA16E5CDC3944040F3C251
:10D36900A8C2AAE49026E8F0A3F0A3F0A3F0C2CAE9
:03D37900028B66BE
:10DE8000EFD3940440037F00221F908002E0FEA89D
:0CDE900007088002C313D8FC5401FF22D5
:09E07700908002E0F4540FFF2236
:10DA58007410A807088002C333D8FCFF901D51E05A
:10DA6800FEED6005E04FF0800B901D51E0FDEFF4F6
:10DA7800FFED5FF0901D51E0908002F06E6005743C
:05DA880001121CB12297
:10B6AB0090248E12B254A312204590249112B22BE7
:10B6BB00A312B20012B293500C12B20C74ADF0A3E1
:10B6CB0074E702B73C12B27890249512B2001217AD
:10B6DB00FD502E7F857EEB7D517C3E90249112B2E6
:10B6EB00001217FD401B12B28190249112B200126E
:10B6FB0017FD6002500B12B20C74ADF0A374F18005
:10B70B003012B28A90249112B2001217FD400B1224
:10B71B00B20C74ADF0A374FB801712B28A9024950F
:10B72B0012B2001217FD400D12B20C74AEF0A374DE
:10B73B0005F002B78512B27890249512B200121759
:10B74B00FD502012B28190249112B2001217FD60AD
:10B75B0012401012B20C74AEF0740F12B1F412B29C
:10B76B005D801712B20C74AEF0741A12B1F412B2EF
:10B77B005D90249512B1F912B2E790248E12B22289
:04B78B00123B5022FB
:10B3E3009024EC12B254A31220459024EF12B22BF6
:10B3F300A312B20012B293500C12B20C74AEF0A3AB
:10B40300742602B47412B2789024F312B2001217A5
:10B41300FD502E7F857EEB7D517C3E9024EF12B252
:10B42300001217FD401B12B2819024EF12B20012DA
:10B4330017FD6002500B12B20C74AEF0A3742C8093
:10B443003012B28A9024EF12B2001217FD400B1291
:10B45300B20C74AEF0A37432801712B28A9024F344
:10B4630012B2001217FD400D12B20C74AEF0A374A9
:10B4730038F002B4CC12B2789024F312B20012174F
:10B48300FD502612B2819024EF12B2001217FD6014
:10B4930018401612B20C74AEF0743E12B2A190248E
:10B4A300EF12B20012B25D802012B20C74AEF074CF
:10B4B3004712B2A19024EF12B20012B25D12B2A3EE
:10B4C3009024F312B20012B2E79024EC12B22212CB
:03B4D3003B5022C9
:10D90D007F09200F3612C51A1292FA12C271901C9D
:10D91D00A8E07004A3E06401701220110512B2B8E2
:10D92D008010901CA7E0700AD20F8006C2A9C21108
:0CD93D00D2A9EF64086004EFB402C72216
:10DA22007F09200F3012C271901CA8E07004A3E09D
:10DA32006401701220110512B2B88010901CA7E088
:10DA4200700AD20F8006C2A9C211D2A9EF6408607F
:06DA520004EFB402CD2236
:1092FA00E4902511F0A3F07F0612DDC490250DEE4F
:10930A00F0A3EFF07F0712DDC490250FEEF0A3EF74
:10931A00F0D390250EE094F790250DE0940A405280
:10932A0012DFFD7AAE79531294917AAE795B7F029D
:10933A0012D2B57BFF7AAE796A7F0312D2B5902535
:10934A000DE0FCA3E0FDE41218807B117AC779BA1C
:10935A00783B1216579025171220457BFF7AAE7973
:10936A00777F0412D2B512C51A7FD07E0712DE9C0F
:10937A00D290E4FFFE7D807C3F9014F512B2001279
:10938A0017FD700A902511F0A37404F08019E4FF08
:10939A00FEFD7C409014F512B2001217FD70089081
:1093AA002511F0A37410F0D390250EE09482902535
:1093BA000DE094064028C20DD3902512E094009047
:1093CA002511E064809480401590151612B22BEC9A
:1093DA004D4E4F6009902511E4F0A37480F0300AD5
:1093EA0014901CA8E07004A3E0640670089025118C
:1093FA00F0A37480F0902817E0FCA3E090251112E6
:10940A00B2306D7002EE6C601212DFDF902511E04F
:10941A00FFA3E0902817CFF0A3EFF0901CAAE0700A
:10942A0002A3E07061200D5EC3902510E0945C9069
:10943A00250FE09403504FD20D20104A12E0341247
:10944A00DFFD7AAE797F1294917AAE79877F021224
:10945A00CFDE7BFF7AAE79937F0312CFDE7BFF7A72
:10946A00AE79A87F0412CFDE7BFF7AAE79B77F058B
:10947A0012CFDE12C51A7FE87E0312DE9C12DA22B0
:10948A0012E04012C51A227BFF7F0112CFDE7BFF5A
:01949A0022AF
:0CE04C00A804A905AA06AB07121657226B
:10DEE8009015FD12B22BEC4D4E4F600790161E1286
:07DEF800B22B2212D43B22E1
:10D68A009024EC1220457F337E937D887C4390243E
:10D69A00F412B2001215669024EC12B20012165758
:10D6AA00C004C005C006C0077F337E937D887C43D3
:10D6BA009024F012B200121566A804A905AA06ABB6
:0DD6CA0007D007D006D005D004121760224B
:1022F100536F756E642028636F6D70757465642902
:10230100000025362E3366206D732020756E6361C3
:102311006C2E0025362E3366206D732025362E3126
:1023210066206D2F7300636F6D703A2025332E3058
:1023310066202070756C73653D2025332E30660054
:10234100636F6D703D2025332E3066202070756CD3
:1023510073653A2025332E3066004F602063656C2B
:102361006C00412F443A202535690041646A757338
:10237100743A2025352E306600526573756C743AB7
:102381002025362E3366206D5600536F756E6420FE
:102391002872617729006677643A253575202535DD
:1023A100752025352E3066006277643A2535752013
:1023B1002535752025352E306600496E707574738C
:1023C10000584920343A2531627520333A2531626B
:1023D1007520323A2531627520313A253162750016
:1023E100494420496E742025313473004944204505
:1023F1007874202531347300412F4420302D33006F
:102401004F6020202025356925382E3366206D56F2
:1024110000566F6C742025356925382E3366205699
:10242100004F686D202025356925382E33662056EA
:1024310000417578312025356925382E33662056BF
:1024410000412F4420342D37004175783220253545
:102451006925382E336620560050574D30202535DA
:102461006925382E336620560055652020202535F4
:102471006925382E336620560055722020202535D7
:102481006925382E336620560054656D706572617A
:102491007475726500496E743A206E6F20646174C0
:1024A1006100496E743A20253469202020202534AA
:1024B1002E3166202573007E46007E4300457874E8
:1024C1003A206E6F7420636F6E6E6563746564008D
:1024D1004578743A202534692020202025342E3176
:1024E10066202573004F787967656E2073656E737A
:1024F1006F72206E6F740063616C696272617465E2
:10250100642E0043616E277420636F6E74696E756B
:10251100652E004F787967656E2073656E736F72F3
:102521002064616D61676564006D697373696E67CD
:10253100206F7220657870697265642E005B257367
:102541005D00202573200025342E30660025352EB0
:102551003166002020202020202020200025633A01
:1025610020536F6C76696E670025633A2563257386
:1025710020256325730025632563257320256325A5
:10258100730025332E3066002020202020002534C2
:102591002E306622002020200025322E30664C008D
:1025A100456D707479202020200025633A2563252C
:1025B100732025732025730025632563257320254A
:1025C10073257300536176696E672073657474694E
:1025D1006E677300706C6561736520776169742043
:1025E1002000526573657420746F2064656661759F
:1025F1006C74733F00526563616C696272617465EA
:102601003F002020202020206F7665726C6F61646E
:1026110000282B29202020202020202020202020BD
:10262100202020282D2900282D292020202020208D
:10263100202020202020202020282B290025362E74
:1026410032662056204443002820292020202020C3
:10265100202020202020202020202820290025366D
:102661002E326620562041430025362E32662056F2
:102671002041432025332E306620487A0020202037
:102681004D61782E20343020562041432F444300A1
:102691002020202020202020202E2020207B0025EB
:1026A10031312E316620207B0020202052616E675F
:1026B100652030202D2031303030207B002020203B
:1026C10020205B636F6E6E65637465645D0020201E
:1026D1002020205B2020202020202020205D0020A1
:1026E1002020426565702062656C6F772032303042
:1026F100207B0054656D70657261747572653A2551
:10270100362E3166202573004D696E696D756D3AFF
:102711002020202025362E3166202573004D61783A
:10272100696D756D3A2020202025362E31662025D1
:102731007300417665726167653A20202020253655
:102741002E3166202573004572726F722031004868
:10275100656C69756D2073656E736F7220646F654A
:10276100736E277400776F726B20636F727265638B
:10277100746C79004572726F722032006F72206D35
:10278100697373696E672028796F75206D617900AF
:10279100737769746368206974206F666620696E57
:1027A100004D454E55202D20707265666572656E2F
:1027B10063657329005761726E696E670052756EA9
:1027C1006E696E6720696E2064656D6F206D6F6440
:1027D1006500446F206E6F742075736520666F729B
:1027E100006D6561737572656D656E74005377690F
:1027F1007463682064656D6F206D6F6465206F661A
:10280100663F004F787967656E2073656E736F72EE
:10281100007377697463686564206F666620287940
:102821006F75206D617900737769746368206974CD
:10283100206F6E20696E004572726F722033004FF7
:10284100787967656E2073656E736F722065787035
:1028510069726564005265706C616365206F787997
:1028610067656E2073656E736F7200286F722073D7
:102871007769746368206974206F666620696E00E9
:102881004572726F72203400446576696365206910
:102891007320746F6F20636F6C64004D61792077D2
:1028A1006F726B20696E636F72726563746C79000D
:1028B10025352E3166202573004572726F722035E1
:1028C1000044657669636520697320746F6F2077B2
:1028D10061726D0048652F4F6020616E616C797A7D
:1028E10065720044697665736F66740048572032DB
:1028F1002E2531626400465720257320257300324E
:102901002E313200323030392F30362F31310053F1
:102911004E20256C75002020202053776974636850
:10292100696E67206F66662020202000000000008D
:102931000000000000000000000000000000000096
:10294100303132334D004131323344000000000058
:1007BA00411E3E01C10FC111411CA700421CA500E8
:1007CA0000421CA80009421E3F0000421CA1000171
:1007DA00421C9F0000421D7A0000421CA3000042F6
:1007EA001CAA0190C10D421D4F0000C110C10B414E
:1007FA001D5100C10CC10AC10E60281D524D6574FD
:10080A0072696320756E69747300552E532E2075B4
:10081A006E697473005365742073657061726174D4
:10082A00656C79000060A31CAC476173206D697820
:10083A0020736F6C76657200476173206D6978204A
:10084A0073696D756C61746F7200436F6E74696E53
:10085A0075616C20616E616C7973697300507265A1
:10086A00666572656E636573004D65617375726561
:10087A006D656E7420756E69747300526573657464
:10088A0020746F2064656661756C740050726F62C3
:10089A00652063616C6962726174696F6E00496E8A
:1008AA007465726E616C2076616C75657300526551
:1008BA0063616C63756C617465204C534D005365BC
:1008CA007276696365206D6F64650000605C1D80E7
:1008DA0052656C6F61642076616C7565730055733F
:1008EA00652031206D6978747572650055736520CD
:1008FA0032206D697874757265730055736520339B
:10090A00206D69787475726573004D6561737572CF
:10091A00656D656E7420756E697473004761732026
:10092A0070726F70657274696573000060621DDCB5
:10093A00536F6C76650052656C6F61642076616CEA
:10094A00756573005573652031206D697874757209
:10095A0065005573652032206D6978747572657308
:10096A00005573652033206D69787475726573005C
:10097A004D6561737572656D656E7420756E697407
:10098A0073004761732070726F7065727469657362
:10099A000000481C934E6F005965730000441E41C5
:1009AA004479C000442445C479C000441C9B00001B
:0909BA000000441D7C0000000057
:1043EC00A3F0902457E075F018A42448F582E43427
:1043FC0027F583E0FCA3E0FDA3E0FEA3E0FF229001
:10440C002452E4FFFE7D107C41E0F8A3E0F9A3E028
:10441C00FAA3E0FB22902478E025E0FF902477E0DB
:10442C0033FE74452FF582741E3EF58322F09024E2
:10443C009DE0FBA3E0FAA3E0F922121657E4FBFA85
:10444C0079A07840121760E4FBFAF97842021566FD
:10445C0004FF902461E0902517F090245AE09025F9
:10446C0018F0A37401F0A37424F0A3746AF0A3747D
:10447C0001F0A37424F07476A3F0A37401F0A322CA
:10448C00902477E0FEA3E0FFC322902517EEF0A363
:10449C00EFF0FDAC06E41218807923783B7B0A7AA6
:1044AC00D71216579025191220457BFF22E0FEA348
:1044BC00E0FF90247FE0FCA3C3E0FDEF9DEC648063
:1044CC00F8EE64809822E0FCA3E0FDEC02188090EA
:1044DC00251BEBF0A3EAF0A3E9F022E0FB75F01842
:1044EC00A42450F582E43427F583122045EB75F0B3
:1044FC0018A4244CF582E4342722C2A9D211901CB2
:10450C00A77428F0D2A9227BFFE0FFA3E0CF90256F
:10451C0017F0A3EFF0221216579025170220451220
:10452C00156690248D122045902478E004F022909A
:10453C002459E075F018A42454F582E43427F5834B
:10454C00022045121657797A7844E4FBFA02176078
:10455C00902517EEF0A3EFF0FDAC06E4021880A353
:10456C00F0902457E075F018A42444F582E4342725
:10457C00227B01E075F018A42450F582E434272244
:10458C00E4FFFE7D807C3F021562E075F018A424E8
:10459C0058F582E43427F583022045902477E00413
:1045AC00F022E0FB75F018A42448F582E43427F5DA
:1045BC0083022045902497E4F0A3F0A3F07B01A3A1
:1045CC0004F0A322E0FEA3E0FFEE3395E0FDFC7BBC
:1045DC00007A8079FF78FFC3021F087B007A50793C
:1045EC00C3784722CFF0A3EFF0902477E475F00165
:1045FC00121D43AFF02290251B1220457FE37E381D
:10460C007D0E7C3A9024582279C87842E4FBFA0259
:10461C001760EF04FF7BFF7A237902229026EBE0F0
:10462C009026EA9FFDE09EFCE4021880EFF0901CBF
:10463C00A8E022C2A9C211D2A922EC4D4E4F7BFF99
:10464C0022121C49FF3395E0FE902496E024FFFDD6
:10465C00902495E034FFFC227424F0A37455F0A34D
:10466C00EBF0A37424F0A37456F07A1C79AC22EC12
:10467C0012187BA804A905AA06AB07227D017BFFB3
:10468C007E007F06021C23121566902489022045A9
:10469C00901CA1E0FEA3E0FF64054E2290251912A8
:1046AC00204590197622E4FBFAF9F80217FDE00494
:1046BC00FF902461E0902517F090245AE090251883
:1046CC0022E4902477F0A3F022902452122045E4A7
:1046DC00FFFEFD22E4F090248704F022902517744D
:1046EC0001F0A37424F0A37458F07BFF22E0FFA325
:1046FC00E0902519CFF0A3EFF090245A22E4FFFEAE
:10470C007D107C412212165790259802204590244A
:10471C0077E0FFA3E0229EF9E0FBA3E0FAA3E0C957
:10472C008FF0021D919024ABE0F9A3E0FAA3E022F4
:10473C001215627B5D7AF9797C783F021657121557
:10474C00627BAC7AA87941783C0216571217607BD1
:10475C00917A0F796878410216577424F0A3746B20
:10476C00F0902462E090251C22E490247FF09019B4
:10477C003CE0FEEF229D7480F8E064809822902546
:10478C001B02204590193EE0FF902459E022E0FFE7
:10479C00A3E0902477CFF0A3EFF022E4FBFA79802A
:1047AC0078BF22E4FBFA7980783F221220457F5DA6
:1047BC007EF97D7C7C3F226480F8E0648098227DC9
:1047CC0004FE7C00021CF7E0FEA3E0C39BEA22E09F
:1047DC00FEA3E0D39BEA22E0FEA3E0FF90247DE061
:1047EC00FCA322F58312204575F084EBA4227409F6
:1047FC00F0E4A3F0A37420F022902478E09F90249E
:10480C0077E09E22902484E09FFF902483E0229006
:10481C0024581220459013CC22A3F0A3EBF0A32232
:10482C001216579024922212165790248D227D0432
:10483C007C00E4FF227424F0A37463F07BFF2274E9
:10484C0024F0A37462F07BFF22E0FCA3E0FDC32202
:09485C007B0A7AD779230217FDCB
:03000B0002BED062
:10BED000C0E0C083C082C0D0758C4C758A009028A9
:10BEE00016E004F07006902815E004F0901E3FE084
:10BEF0007002A3E0600E901E40E024FFF0901E3F11
:10BF0000E034FFF0901C9FE07002A3E0600E901CF4
:10BF1000A0E024FFF0901C9FE034FFF0901D7BE038
:10BF200004F07006901D7AE004F09026CFE06002E5
:10BF300014F0901CA3E07002A3E0600E901CA4E03B
:10BF400024FFF0901CA3E034FFF0301108901CA7F0
:10BF5000E0600214F0901CAAE07002A3E0600E9072
:10BF60001CABE024FFF0901CAAE034FFF0901D4FC2
:10BF7000E07002A3E0600E901D50E024FFF0901DE1
:10BF80004FE034FFF0C28DD0D0D082D083D0E032E9
:0300030002DE0614
:10DE0600C0E0C083C082C2CA9026E9E5CCF0902665
:0FDE1600E8E5CDF0D2CAC2A8D082D083D0E032E6
:0300130002DE25E5
:10DE2500C0E0C083C082C2CA9026EBE5CCF0902644
:0FDE3500EAE5CDF0D2CAC2AAD082D083D0E032C3
:0300230002D76A97
:10D76A00C0E0C0F0C083C082C0D075D000C000C085
:10D77A0001C002C003C004C005C006C00730990535
:10D78A0012DFA9C29930980512E089C298D007D051
:10D79A0006D005D004D003D002D001D000D0D0D01A
:08D7AA0082D083D0F0D0E03200
:10BA1E007BFF7A2279F17F0112CFDE1246217F025F
:10BA2E0012CFDEE4FF12D3199026E812448F12468D
:10BA3E002812481B1243FFEC4D4E4F124608700E53
:10BA4E001244151245227BFF7A2379038018124483
:10BA5E001512165712D9B612460212441512452265
:10BA6E007BFF7A2379147F0312D2B57F0112D3198B
:10BA7E009026EA12448F9026E9E09026E812462F8F
:10BA8E0012481B1243FFEC4D4E4F124608700E1219
:10BA9E0044151245227BFF7A237903801812441530
:10BAAE0012165712D9EC1246021244151245227B79
:10BABE00FF7A2379147F0412D2B57BFF300E067AFB
:10BACE0023792780047A2379419011591243FF126A
:10BADE0045259014D41243FF12478A7F0512D2B522
:01BAEE002235
:10CF04007BFF7A23795B7F0112CFDE1246217F02F9
:10CF140012CFDEE4FF12DDC4902458EEF0A3EFF04C
:10CF24007A2379639024581245137F0312D2B57B78
:10CF3400FF7A23796C9013481243FF1245257F042E
:10CF440012D2B5902458E0FCA3E0FDE412188090BE
:10CF540013481244151215667B367A947957783C37
:0ECF64001245227BFF7A23797A7F0502D2B52F
:10C10800E4902458F0A3F07BFF7A23798B7F011207
:10C11800CFDE1246217F0212CFDEE4FF12D3199040
:10C1280026E812448F12462890245A1220457A2372
:10C1380079979026E81245139026EA1246F9124399
:10C14800FF12478A7F0312D2B57F0A7E0012DE9C57
:10C158007F0112D3199026EA12448F9026E9E09FB6
:10C16800FD9026E812463190245A1220457BFF7A2A
:10C178002379A99026EA1245159026E81246F91265
:10C1880043FF12478A7F0412D2B57BFF300E067A2E
:10C1980023792780047A2379419011591243FF1299
:10C1A80045259014D41243FF12478A7F0512D2B551
:07C1B8007F0A7E0002DE9CFD
:10CB140078587C247D017BFF7A29792D7E007F144F
:10CB2400121C237BFF7A2379BB7F0112D2B57F04C9
:10CB340012DE80C0077F0312DE80C0077F0212DE90
:10CB440080C0077F0112DE8090251AEFF09025192E
:10CB5400D0E0F0902518D0E0F0902517D0E0F07BDD
:10CB6400FF7A2379C27F0212D2B51246217F0312C3
:10CB7400CFDE7B017A24795812C8C31246E87A239F
:10CB840079E17F0412D2B57B017A24795812C6F573
:0CCB94001246E87A2379ED7F0502D2B545
:10CDA6007BFF7A2379F97F0112D2B5E4FF12DDC445
:10CDB600EE12451A1245647B367A947957783C12FE
:10CDC60044AD7A2479017F0212D2B57F0112DDC407
:10CDD60012455C79A3783C1244A97A2479127F0320
:10CDE60012D2B57F0212DDC412455C7B6F7A1279CE
:10CDF60083783A1244AD7A2479227F0412D2B57F21
:10CE06000312DDC41244967A2479327F0512D2B514
:07CE16007FC87E0002DE9CD4
:10CE1D007BFF7A2479427F0112D2B57F0412DDC4E3
:10CE2D001244967A24794A7F0212D2B57F0512DD1B
:10CE3D00C412455C7B6F7A127983783A1244AD7ACD
:10CE4D0024795A7F0312D2B57F0612DDC412455CD8
:10CE5D007B117AC779BA783B1244AD7A24796A7F0F
:10CE6D000412D2B57F0712DDC412455C7B117AC75F
:10CE7D0079BA783B1244AD7A24797A7F0512D2B50E
:07CE8D007FC87E0002DE9C5D
:10AEDD0012C82B902460EEF0A3EFF012CA829024DA
:10AEED0062EEF0A3EFF09024601244D279807841A5
:10AEFD001245569024581220459024621244D2795E
:10AF0D0080784112461890245C1220457BFF7A24EC
:10AF1D00798A7F0112D2B51246217F0212CFDE90BF
:10AF2D0024601245D070097BFF7A24799602AF8197
:10AF3D009024601245159019761243FFEC4D4E4F3B
:10AF4D00600B90245812440E1244468006902458EB
:10AF5D001243FF1246A81243FF12464660067A249A
:10AF6D0079B880047A2479BB90251D1244DE7BFFCD
:10AF7D007A2479A37F0312D2B59024621245D07042
:10AF8D00097BFF7A2479BE02AFDE9024621245154B
:10AF9D009019761243FFEC4D4E4F600E12470990FB
:10AFAD00245C124415124446800690245C1243FF23
:10AFBD001246A81243FF12464660067A2479B880DD
:10AFCD00047A2479BB90251D1244DE7BFF7A247907
:0EAFDD00D17F0412D2B51246217F0502CFDECD
:1079F2009024577409F0902457E0FF640270030248
:107A02007C23EF64037003027C23300F03027C2388
:107A1200901CA1E0FEA3E0FFEE704BEF14B4070050
:107A22005044907A3275F003A4C58325F0C5837360
:107A3200027A47027A4C027A51027A56027A5B0241
:107A42007A60027A6512AEDD801C12CDA680171212
:107A5200CE1D801212CB14800D12C108800812BAFA
:107A62001E800312CF0412C51A1292FA12C271902A
:107A720024571246387004A3E064017012201105E5
:107A8200124506800D901CA7E07007D20F800312EA
:107A9200463F902457E024FC605124FE7003027B91
:107AA2006E14601D240260030279F812469C60097C
:107AB200EF64064E60030279F8A20EB3920E0279C9
:107AC200F8901CA2E004F07006901CA1E004F0D330
:107AD200901CA2E09407901CA1E064809480500363
:107AE2000279F8E4F0A304F00279F812469C6006E9
:107AF200EF64064E7045300E21E4FFFEFDFC90144B
:107B0200D41244151217FD600250030279F8901442
:107B1200D41243FF1247A7027B9AE4FFFEFDFC90BA
:107B220011591244151217FD600250030279F890A0
:107B320011591243FF1247A7027BC7901CA1E070A4
:107B420004A3E0640760030279F89013381243FF3C
:107B52009013481244151217FD600250030279F87F
:107B62009013481243FF1247A7027C1112469C60F1
:107B720006EF64064E706C300E2DE4FFFE7D8C7CA9
:107B8200429014D41244151217FD40030279F89062
:107B920014D41243FF1247AF1215669014D4122068
:107BA200459014D8027C1DE4FFFE7D7F7C4390113A
:107BB200591244151217FD40030279F89011591217
:107BC20043FF1247AF1215669011591220459011CA
:107BD2005D7401F09011591243FF1218B912E05866
:107BE2000279F8901CA1E07004A3E064076003022C
:107BF20079F890133C1243FF901348124415121760
:107C0200FD40030279F89013481243FF1247AF1266
:107C1200156690134812204590134C7401F00279B6
:027C2200F82246
:10A0EA00902457EFF0A37409F09012C41243FFECC6
:10A0FA004D4E4F700D7A2479E612A2227A2479F80D
:10A10A00800E30151E7A25791412A2227A25792A10
:10A11A007F0212CFDE7BFF7A2579047F0312CFDE1E
:10A12A0002D90D902457E06004D2108002C21012A6
:10A13A00DFEF300F0302A1F6902457E0600B12E024
:10A14A0077EF6406600302A1F6902457E060047F6B
:10A15A000E80027F0DE4FD12A5D712C51A1292FADB
:10A16A0012C2719024581246387004A3E064017038
:10A17A0012201105124506800D901CA7E07007D227
:10A18A000F800312463F902458E024FE604E24FBC1
:10A19A0060552404709C12DFFD902457E0600890FB
:10A1AA00245A7409F0802112CA821245D560089097
:10A1BA00245A7408F0801112E07790245ABF0905D6
:10A1CA007406F080037404F07B017A167985902472
:10A1DA005AE0FD12BBBA12DFFD02A13C902457E0FF
:10A1EA00600302A13C8005B21002A13CC210902477
:10A1FA0057E060177F0112A2167F0212A2167B0196
:10A20A007A247959E4FD7F0312DA58227B017A24F1
:10A21A007959E4FD12DA58227BFF7F0112CFDE7BE7
:02A22A00FF2211
:10BE0D009024A6ECF0A3EDF0E49024AEF09024ABDA
:10BE1D001244DE9024A8E09024AFF09024AEE0FD13
:10BE2D007C00D39024A7E09024A6124781407990FE
:10BE3D0024AFE0FFD39405506F9024A9E0FB339518
:10BE4D00E0FAC3ED9BEA6480F8748098403AA3E071
:10BE5D00FE9024AEE0B50612124731902517C91297
:10BE6D0044DF7BFF7A25793E80159024AFE0FF12E9
:10BE7D004731902517C91244DF7BFF7A257943128C
:10BE8D00D2B59024AFE004F09024AB12443D12DF04
:10BE9D006CEF2401FFE43E9024AC8FF0121D2D9029
:10BEAD0024AEE004F002BE289024AFE0FFD3940549
:10BEBD00500E12462112CFDE9024AFE004F080E840
:03BECD0002C51A91
:109B06009024921244DEA3ECF0A3EDF09024A1740D
:109B160001F0A3124439121C49C364809480500496
:109B2600E4121CB112443A12464DD31244C7400601
:109B3600A3E014121CB1902497E0FBA3E0FAA3E083
:109B46004A4B6012902497A3A3E0F97F0112CFDE5F
:109B56009024A27402F0300F03029C9090249A1273
:109B6600443D121C49FF12443A121C49FEC3EF122F
:109B760044CA500A90249A12443DEE121CB1902415
:109B86009A12443D121C49FF3395E0FE9024A2E050
:109B9600FD3395E0FCC3EF9DFFEE9CCF2406CF344A
:109BA60000FE12443A121C49FDFB3395E0FAC3EB62
:109BB6009FEE6480F8EA6480984014ED24FBFF90E1
:109BC60024A2E02FFF90249A12443DEF121CB1907C
:109BD60024A1E0602F902495E0FCA3E0FD9024A250
:109BE600E09024A8F090249A12443D121C49902437
:109BF600A9124439121C499024AAF09024921244C6
:109C06003D12BE0DE49024A1F012C51A1292FA126A
:109C1600C2719024A01246387004A3E06401701249
:109C2600201105124506800D901CA7E07007D20F83
:109C3600800312463F9024A0E024FD604A14601978
:109C460024FE602824FE603F24066003029B5C120B
:109C5600443A74FF121CB1802E12443A12464DC388
:109C66001244C750197401121C8F801212443A1202
:109C76001C49D364809480400574FF121C8F902485
:0B9C8600A17401F0029B5C12DFFD22C4
:10D548009024571244DEA3EDF0E4A3F0A3EDF0908D
:10D558002457124734902497C9F0A3EAF0E91244FB
:10D56800847424F0A3745B1244857424F0A3745C5F
:10D57800F07B017A1C79937D027C00129B06902433
:10D588005CE0FE7002FF22EEB401037F01229024CA
:04D598005AE0FF2234
:10CCAF00E4902490F0A3F0902491E0F46070200FB2
:10CCBF006D1245C07424F074901248257424F0A3AB
:10CCCF007491F07A1D79527D037C00129B0690249B
:10CCDF0091E0FC14600714603A240270CAEC121839
:10CCEF00859019FA1220459019D91220459019B83C
:10CCFF001220459019971246AB1220459019FE74D9
:10CD0F0001F09019DDF09019BCF090199BF090197B
:0FCD1F007AF0227B017A19795A7D0512BBBA226C
:10BAEF00902490ECF0A3EDF0A3EFF0902492E0FF00
:10BAFF00FDC3902491E0902490124781500302BB24
:10BB0F00B975F084EFA4243CF582E5F0341A1243A2
:10BB1F00FD124552902492E0FB1245711247EF241B
:10BB2F001BF582E5F0341A1243FD1245E712482C3B
:10BB3F001245AE75F084EBA4245DF582E5F0341A5E
:10BB4F001243FD124614902492E0FB1244FA12475E
:10BB5F00EF247EF582E5F0341A1243FD124614905D
:10BB6F0024921244E7F58312441512458C902492C7
:10BB7F0012457FF5831244151215629024931247D4
:10BB8F00B790249312441512482C12453E7FAC7E79
:10BB9F00A87D417C3C90249312441512482C1245E9
:0BBBAF0096902492E004F002BAFA2203
:10BF900090248BECF0A3EDF0A3EFF090248DE0FF64
:10BFA000FDC390248CE09D7480F890248BE0648025
:10BFB00098500302C04D75F063EFA424CAF582E5E2
:10BFC000F034171243FD1245E71248331245AE759F
:10BFD000F063EBA424EBF582E5F034171243FD1275
:10BFE000461490248DE0FB1244FAF5831220457527
:10BFF000F063EBA4240CF582E5F034181243FD1233
:10C00000461490248D1244E7F58312441512458C92
:10C0100090248D12457FF5831244151215629024E9
:10C020008E1247B790248E12441512483312453EA3
:10C030007FAC7EA87D417C3C90248E124415124832
:0EC040003312459690248DE004F002BF9B223F
:10D37C00E4902489F0A3F090248AE0F46053200F09
:10D38C00501245C07424F074891248257424F0A3FB
:10D39C00748AF07A1D79807D067C00129B0690249D
:10D3AC008AE01424FD500F6016146018240570C711
:10D3BC0012483A02BF9090248AE090193EF0221253
:10D3CC00CCAF80B37B017A1679237D0212BBBA8075
:02D3DC00A62287
:105890009024581247FA785B7C247A297941124681
:1058A000889024777401F0E4A31246E1E4A3F01297
:1058B000DFEF9019D91243FFEC4D4E4F6005E49095
:1058C0002477F07D037C00E4FF12BF90300F0302C9
:1058D0005C2C902478E0700302598EE4902486F0CA
:1058E000902479F012E077BF090312000790249109
:1058F0007401F0A37424F0A3747E1244857424F020
:10590000A374821244857424F0A3748612448574AF
:1059100024F0A37479F07B017A24797A129155905E
:105920002479E07069A31243FF902459E0FB1244EC
:10593000FAF58312204590247E1243FFEB12458036
:10594000F58312204590247A12441512458C902438
:105950007E12441512473C90245912453E90247AF9
:1059600012441512458C90247E12441512474A9019
:10597000245912459612E077BF091312DC361245FE
:10598000E7121657902459E01245B0120006E49031
:105990002457F0902457E0FFC394054003025B05B1
:1059A00090193EE0FEEF9E400E902457E094045084
:1059B0000612461E025AF99024571247936F702A16
:1059C000902478E0601C902486E0700E902479E0AA
:1059D000700890245A743EF0801690245A743FF058
:1059E000800E90245A742AF0800690245A7420F075
:1059F0009019B81243FFEC4D4E4F902595601474EA
:105A0000FFF0A37425F074481243EC1245E71247E7
:105A100058801274FFF0A37425F0744E1243EC12F8
:105A200045E71217601247147B017A247963123B11
:105A3000501243EE1246B25032902457E01244FA0C
:105A40001243FDC004C005C006C0077A24796B90DC
:105A5000245712457D1243FD902495122045D0070E
:105A6000D006D005D00412B6AB801790259574FFF0
:105A7000F0A37425F0A37454F07B017A24796B129F
:105A80003B50902457E0FF245BF582E43424F583F7
:105A9000E0902461F0EF6003B40408902462742065
:105AA000F08006902462742BF0902488E0701990A6
:105AB0002457E0B4041204FF7BFF7A25795E90241A
:105AC00061E0902517F08031902477E090245760B2
:105AD000151246BA1244851247661244851248418F
:105AE0007A25796A80131246BA12448512476612E3
:105AF00044851248417A25797712D2B5902457E02F
:105B000004F002599312C51A1292FA12C27190242B
:105B1000581246387004A3E0640170122011051277
:105B20004506800D901CA7E07007D20F8003124637
:105B30003F902487E0601090193EE0FF125F54E42C
:105B4000902487F0A304F0902458E024FE70030210
:105B50005C2C24FE7003025C101460381470030285
:105B60005BF224FE6068240560030258CC12D37CEB
:105B7000124790D39F4002EFF09019D91243FFECE7
:105B80004D4E4F6007E4902477F08038902477746E
:105B900001F08030E4902478F012DFFD902459E089
:105BA00075F063A424AEF9741735F0FA7B017D0318
:105BB00012BBBA12DFFD12DFBB902459E0FFFD7C5F
:105BC0000012BF90E49024881246E10258CC902441
:105BD00078E060091246E012DFBB0258CC902478CE
:105BE0007401F0E4902488F0902487F012DFEF0233
:105BF00058CC902459E0D3940050030258CC902400
:105C000078E060031246E0902459E014F00258CC8A
:105C1000124790C39F40030258CC902478E0600361
:0D5C20001246E0902459E004F00258CC2216
:10CE9400E490248EF0A3F090248FE0F46061200FDE
:10CEA4005E1245C07424F0A3748EF0A3EBF0A37457
:10CEB40024F0A3748FF07A1D79DC7D077C00129B2B
:10CEC4000690248FE014601524FC5017601F146032
:10CED40021240670C290193CE0FF02ACB412483A17
:10CEE40002BAEF90248FE01490193CF02212CCAFD8
:10CEF40080A57B017A1679237D0212BBBA80982221
:1054AC009024581247FA785B7C247A297947124663
:1054BC008890247E7401F0E4A3F012DFEF9019D9E8
:1054CC001243FFEC4D4E4F6005E490247EF01248E1
:1054DC003A02582A300F0302588F90247FE0700351
:1054EC000255B4E490248DF0902480F012E077BF44
:1054FC0009031200079024917401F0A37424F0A303
:10550C0074851244857424F0A37489124485742420
:10551C00F0A3748D1244857424F0A37480F07B0185
:10552C007A247981129155902480E0707BA31243E8
:10553C00FF902459E0FB1244FAF583122045902485
:10554C00851243FFEB124580F58312204590248190
:10555C0012441512458C90248512441512473C12A6
:10556C00453B90248112441512458C90248512449D
:10557C001512474A902459124596902481124415CD
:10558C0012458C90248512441512156212453B125B
:10559C00E077BF091312DC361245E7121657902438
:1055AC0059E01245B0120006E4902457F0902457AD
:1055BC00E0FFC39405400302577612477A9E400ED3
:1055CC00902457E09404500612461E02576A902409
:1055DC0057E0FF902459E06F702A90247FE0601C04
:1055EC0090248DE0700E902480E0700890245A7402
:1055FC003EF0801690245A743FF0800E90245A741A
:10560C002AF0800690245A7420F09019B81243FFA7
:10561C00EC4D4E4F902595601974FFF0A37425F056
:10562C00A37448F09024571243F11245E7124758DF
:10563C00801774FFF0A37425F0A37483F0902457A3
:10564C001243F11245E71217601247147B017A24BA
:10565C007962123B509019D91243FFEC4D4E4F60BA
:10566C003812456D1243FD1246B2902595700E749A
:10567C00FFF0A37425F0A37489F00256D974FFF0DF
:10568C00A37425F0748F12456B1243FD7BBE7A5FB9
:10569C00796E7847124711803412456D1243FD1212
:1056AC0046B2902595700D74FFF0A37425F0A37489
:1056BC0096F0801974FFF0A37425F0749A12456B60
:1056CC001243FDE4FBFA797A78441247117B017A94
:1056DC00247976123B509024571243F11246B25063
:1056EC0032902457E01244FA1243FDC004C005C0A6
:1056FC0006C0077A24796A90245712457D1243FD1F
:10570C00902495122045D007D006D005D00412B6AF
:10571C00AB801790259574FFF0A37425F0A374A1AA
:10572C00F07B017A24796A123B50902457E0FF24D5
:10573C005BF582E43424F583E0902461F090247EC0
:10574C00E0600DEF12445C12484B7A2579AB800E69
:10575C00902457E012445C12484B7A2579B912D246
:10576C00B5902457E004F00255B912C51A1292FAFA
:10577C0012C2719024581246387004A3E064017070
:10578C0012201105124506800D901CA7E07007D25F
:10579C000F800312463F902458E024FE70030258F9
:1057AC008F24FE700302586C146046147003025868
:1057BC004A24FE606F240560030254E012CE9490DC
:1057CC00193CE0FF902459E0FED39F4007EE64059E
:1057DC006002EFF09019D91243FFEC4D4E4F600868
:1057EC00E490247EF00254E090247E7401F0025484
:1057FC00E0E490247FF012DFFD902459E075F084F2
:10580C00A424FFF9741935F0FA7B017D0412BBBA9C
:10581C0012DFFD12DFBB902459E0FFFD7C0012BAB1
:10582C00EF0254E090247FE06008E4F012DFBB024A
:10583C0054E090247F7401F012DFEF0254E09024C6
:10584C0059E0FFD3940050030254E0124775D39EE5
:10585C009024594005EEF00254E0E014F00254E0BC
:10586C00902459E0FFD3940540030254E01247758D
:10587C00C39E90245940067404F00254E0E004F0F6
:04588C000254E022C0
:10AFEB00E4902455F0A3F0902456E0F4700302B0E3
:10AFFB00F3300F0302B0F3902497E4300C0A1245A0
:10B00B00C41246647D0A80081245C41246647D064C
:10B01B007C00129B06300F0302B0F3902456E00421
:10B02B00602B14B40A0050BF90B03AF82828730272
:10B03B00B07D02B08302B08902B09102B09B02B026
:10B04B00A102B0B802B0D902B0E702B0ED7BFF7A33
:10B05B002579C57F0112CFDE7BFF7A2579D57F025B
:10B06B0012CFDE12C51A12D7B212E06D12DFFD023B
:10B07B00AFF21254AC02AFF212589002AFF2E4FFEF
:10B08B0012A0EA02AFF27B017A1479D97D0A8046CD
:10B09B0012CCAF02AFF27BFF7A2579E3E4FD12D538
:10B0AB0048EF700302AFF212DB8102AFF27BFF7A43
:10B0BB002579F6E4FD12D548EF700302AFF2901339
:10B0CB00CC12205100000000126B2702AFF27B0163
:10B0DB007A11793D7D1C12BBBA02AFF2123F6E02A0
:09B0EB00AFF21279F202AFF22279
:102FA8009024621244DE90246E12443DE4121CB157
:102FB80090246212443DE4121CB190246812443DEE
:102FC800E4F5F0121D9190246B12443DE4F5F012E3
:102FD8001D9190247112443D12208200000000903F
:102FE800247412443D12208200000000C2A9124637
:102FF800CD7F0112DDC4AC06AD07124421ECF0A36D
:10300800EDF012453470031245A7C3902477E0947D
:103018000340DED2A990247B74F0F0A3E4F090245E
:10302800797410F0A3E4F01246CE12448CEE9403A7
:1030380040030230D3EF25E0FFEE12442CE0FEA35C
:10304800E0FF902495EEF0A3EFF04E600C902495ED
:10305800E0B40F10A3E0B4FF0B90246212443D7457
:1030680001021CB19024951244D212467F9013EDB0
:103078001243FF1215621218B9902495EEF0A3EFCF
:10308800F0D390247AE09FEE9024791247C3400F42
:10309800902495E0FFA3E0902479CFF0A3EFF0907F
:1030A800249512485590247CE09DEC90247B12478F
:1030B800C35005ECF0A3EDF0124421ECF0A3EDF0C1
:1030C80012453470031245A702303290247B124413
:1030D800D2783C12485C6002500D9024791244D298
:1030E80078BC12485C50047F0180027F0090246EF7
:1030F80012443DEF121CB190246E12443D121C493B
:1031080070030231C790248D1220510000000090F6
:103118002489122051000000001246CD9024891203
:103128004415C000C001C002C0031244211244D299
:10313800D003D002D001D00012469390248D1244BF
:1031480015C000C001C002C0031244211244D2C0FD
:1031580004C005C006C0071244211244D2D003D0CF
:1031680002D001D000121657D003D002D001D000EF
:1031780012452B70031245A7902477E06403700270
:10318800A3E07098E4FBFA794078449024891243CC
:10319800FF12176090140E12441512454F124696EE
:1031A800E4FBFA7940784490248D1243FF1235925B
:1031B80012441512454F90248D1220450235739004
:1031C8002479E0FAA3E0FBC390247CE09BFF9024E1
:1031D8007BE09A1247CBEB2FFFEA3E90247DF0A3C9
:1031E800EFF090247BE0FEA3E0FF90247AE02FFF2D
:1031F800902479E03E7D021247CDAB07AA0612441F
:103208008F90247CE09FFF90247BE09E1247CBC3E5
:10321800A3E09FFF90247BE09E90247FF0A3EFF033
:10322800C3901E46E09BEA6480F8901E45E06480E7
:1032380098400302330C1246CD12448CEE9403508E
:103248001AEF25E0FFEE12442C1247D31244CA505D
:103258000A12453470E31245A780DE1245F5902422
:1032680081F0A3EFF012448CEE94035017EF25E0A1
:10327800FFEE12442C1244B9500A12453470E6127B
:1032880045A780E112448CEE9403501AEF25E0FF25
:10329800EE12442C1247DB1244CA400A124534701D
:1032A800E31245A780DE12471A9024831245F09056
:1032B8002485F0A3EFF012448CEE9403501BEF2505
:1032C800E0FFEE12442C1247E3D31244C5400A1221
:1032D800453470E21245A780DD12448CEE94035009
:1032E8001AEF25E0FFEE12442C1247D31244CA50BD
:1032F8000A12453470E31245A780DE12471A90245B
:10330800870233D91246CD12448CEE9403501AEF3B
:1033180025E0FFEE12442C1247DB1244CA400A1281
:10332800453470E31245A780DE1245F5902485F0F8
:10333800A3EFF012448CEE9403501DEF25E0FFEE4E
:1033480012442C1247E3E0FDD31244C7400A124549
:103358003470E01245A780DB12448CEE9403501AB7
:10336800EF25E0FFEE12442C1247D31244CA500A4C
:1033780012453470E31245A780DE12471A9024875D
:103388001245F0902481F0A3EFF012448CEE9403E0
:103398005017EF25E0FFEE12442C1244B9500A12E0
:1033A800453470E61245A780E112448CEE94035030
:1033B8001AEF25E0FFEE12442C1247DB1244CA40F4
:1033C8000A12453470E31245A780DE12471A90248A
:1033D80083CFF0A3EFF0C3902477E0940340047FF9
:1033E8000180027F0090246512443DEF121CB190C9
:1033F800248D1220510000000090248912205100D1
:1034080000000090248112479A90248312448F125E
:103418004805505F902489124415C000C001C002BD
:10342800C0031244211244D2D003D002D001D000EC
:1034380012469390248D124415C000C001C002C0EA
:10344800031244211244D2C004C005C006C00712AA
:1034580044211244D2D003D002D001D00012165712
:10346800D003D002D001D00012452B70031245A71B
:1034780002341190248512479A90248712448F129F
:103488004805505F902489124415C000C001C0024D
:10349800C0031244211244D2D003D002D001D0007C
:1034A80012469390248D124415C000C001C002C07A
:1034B800031244211244D2C004C005C006C007123A
:1034C80044211244D2D003D002D001D000121657A2
:1034D800D003D002D001D00012452B70031245A7AB
:1034E80002348190248112448F1248109EFE902449
:1034F80088E02FFF902487E03EFE902485124855EF
:10350800EF9DFDEE9CFCE41218809024911220455A
:103518009024911244159024891243FF1217609049
:10352800140E12441512454F1246969024911244D7
:103538001590248D1243FF12359212441512454FEF
:1035480090248D12204590248112448F12481090A7
:10355800246812472290248512448F902488E09F83
:10356800FF902487E090246B12472290248912430D
:10357800FF90247112443D121F7F90248D1243FF47
:1035880090247412443D121F7F2212176012C32424
:0435980090140E225B
:10AA84009024657401F0A37424F0A37450124485D7
:10AA94007424F0A374511244857424F0A3745312E3
:10AAA40044857424F0A3745D1244857424F0A37463
:10AAB400551244857424F0A37459F07B017A2479E7
:10AAC4004F122FA890244FE0601112DFFD7BFF7A14
:10AAD4002679037F0212CFDE02C51A90245DE0605E
:10AAE4002E7F0A7ED77D237CBC90245512441512F8
:10AAF40017FD7BFF600840067A26791280047A26C7
:10AB040079287F0112CFDE7BFF7A26793E8053902D
:10AB14002453E0FEA3E0FF902452E02FFD90245143
:10AB2400E03EFCE412188012467F7F007E487D8A56
:10AB34007C4612176090245E1220457BFF7A2679AA
:10AB4400497F0112CFDE902450E07010FFFEFD7C9F
:10AB54003F9024591244151217FD50117BFF7A2699
:10AB6400795F9024591243FF90251780187BFF7A50
:10AB740026796A9024591243FF12452590245E12C7
:10AB840043FF90251B1220457F0312D2B57BFF7A29
:09AB940026797E7F0512D2B5225C
:10B78F00E4902453F012B86090244F1220457F00AC
:10B79F007EF07D7F7C4590244F1244151217FD706B
:10B7AF000590245304F012B86090142F1244151210
:10B7BF00156690145012441512165790244F1246C6
:10B7CF00D8FC90244F1244151217FD500A90244FA5
:10B7DF001220510000000090193BE0603790245375
:10B7EF00E07BFF600B7A2679917F0312CFDE801208
:10B7FF007A2679A090244F1243FF1245257F03121A
:10B80F00D2B57BFF7A2679AA7F0512D2B57FC87E83
:10B81F000002DE9CE4FFFE7D487C4390244F1244DF
:10B82F00151217FD7BFF50117A2679BE7F0312CFB9
:10B83F00DE12C51A12DE62800C7A2679CF7F0312D0
:10B84F00CFDE12C51A7BFF7A2679E07F0512D2B5BB
:0FB85F00227F0212DDC4AC06AD07E4121880226E
:1088750012CA82AC06AD07EC12188090245012463D
:10888500D87CC79024501244151217FD7003028A34
:10889500459024501243FFE4FBFA79807841121782
:1088A500609024501246AB1243FFEC4D4E4F600EC4
:1088B500124709902450124415124446800690240C
:1088C500501243FF1245259019761243FF12464672
:1088D50060067A2479B880047A2479BB1244DB7B5C
:1088E500FF7A2679F47F0112D2B59024501243FF06
:1088F500901E411244151217FD600E400C90245035
:108905001243FF901E411220459024501243FF90C0
:1089150024451244151217FD500C9024501243FFA4
:10892500902445122045901C9B1243FF9024501221
:108935004415121566901C9B122045901D7C124310
:10894500FFE4FAF9F8EF2401FFEA3EFEE93DFDE810
:108955003CFC901D7C1246AB1243FFEC4D4E4F6024
:108965000E124709901E4112441512444680069086
:108975001E411243FF1245259019761243FF1246F8
:108985004660067A2479B880047A2479BB1244DBE0
:108995007BFF7A2779097F0312D2B59019761243A6
:1089A500FFEC4D4E4F600E124709902445124415B9
:1089B50012444680069024451243FF12452590191E
:1089C500761243FF12464660067A2479B880047A07
:1089D5002479BB1244DB7BFF7A27791E7F0412D2F0
:1089E500B59019761243FFEC4D4E4F901D7C601BE0
:1089F5001243FF12467B901C9B1243FF121760E443
:108A0500FBFA79107841124446800F1243FF124653
:108A15007B901C9B1243FF12176012452590197617
:108A25001243FF12464660067A2479B880047A24F8
:108A350079BB1244DB7BFF7A2779337F0512D2B5E8
:018A4500220E
:1068480090245212205100000000E4FF126B1270D5
:106858000890244EF0A3F08013C39026EBE09FFF2E
:106868009026EAE09E90244EF0A3EFF07F01126B91
:10687800127008902450F0A3F080129026EA124873
:1068880055EF9DFFEE9C902450F0A3EFF090244E1E
:1068980012448F9464EE9400401DD3EF9470EE94EC
:1068A800175014124404C39464EE94004009D3EFC3
:1068B8009470EE9417401A12DFFD7A277948126B0C
:1068C8001F7A277950126AB17A2779667F03126B8B
:1068D8000812D9801246D57C3F90245212441512D2
:1068E80017FD50329015371243FFEC4D4E4F60267E
:1068F80012DFFD7A277975126B1F7A257914126ACF
:10690800B17A27797D7F0312CFDE7A277991126ACF
:10691800C5D21512D90D9014B31243FFEC4D4E4F4A
:10692800603A126AA07A2779BE7F0212CFDE7A27F0
:1069380079D3126ABB7A2779E27F04126B087BFF4E
:106948007A2779EEE4FD12D548EF60109014B3125F
:106958002051000000009014B77401F09015371210
:1069680043FFEC4D4E4F702D126AA07A2879047FB0
:106978000212CFDE7A287912126ABB7A2879287F28
:106988000412CFDE7BFF7A2779A27F0512CFDE12B1
:10699800C51A12D90DE4FFFE7DA07C409024521246
:1069A80044151217FD50369015371243FFEC4D4E23
:1069B8004F602A12DFFD7A287938126AED7A287931
:1069C800407F0212CFDE7BFF7A2879567F0312CFF1
:1069D800DE7A28796C126AC5D21512D90D12D43B09
:1069E8001246D5FC9024521244151217FD50467ACF
:1069F800287981126AED7A287989126AF7901976CE
:106A08001243FFEC4D4E4F600812440B124446806F
:106A1800069024521243FF1245259019761243FF1F
:106A280012464660067A2479B880047A2479BB1223
:106A380044DB126ADBE4FFFE7D207C429024521284
:106A480044151217FD604E404C7BFF7A2879BA7FB7
:106A58000112CFDE7BFF7A2879C2126AF790197685
:106A68001243FFEC4D4E4F600812440B124446800F
:106A7800069024521243FF1245259019761243FFBF
:106A880012464660067A2479B880047A2479BB12C3
:106A980044DB126ADB7F002212DFFD7BFF7A277955
:106AA800B67F0112CFDE7BFF227BFF7F0212CFDE93
:106AB8007BFF227BFF7F0312CFDE7BFF227BFF7FE2
:106AC8000412CFDE7BFF7A2779A27F0512CFDE1270
:106AD800C51A227BFF7A2879B17F0412D2B512C574
:106AE8001A12D90D227BFF7F0112CFDE7BFF227F96
:106AF8000212CFDE7BFF7A28799C7F0312CFDE2239
:106B080012CFDE12C51A12D90D2212D3199026E817
:0F6B1800E0FEA3E0FF4E227BFF7F0112CFDE22C3
:10D63C0090244E7409F0200F4412E077EF640570CB
:10D64C003C12AA8412C51A1292FA12C27190244E7C
:10D65C001246387004A3E0640170122011051245C3
:10D66C0006800D901CA7E07007D20F800312463F76
:0ED67C0090244EE024FD70BE12AFEB80B92268
:10D2500090244E7409F0200F5B12E077EF640370A6
:10D260005312B78F12C51A1292FA12C27190244E3D
:10D270001246387004A3E0640170122011051245B3
:10D2800006800D901CA7E07007D20F800312463F66
:10D2900090244EE024FD601724FC70BA90193BE006
:10D2A00070047F0180027F0090193BEFF080A7128D
:05D2B000AFEB80A2229B
:10DCDF00901E411220514479C000902445122051CA
:10DCEF00C479C000901C9B12205100000000901DB1
:09DCFF007C1220510000000022FB
:10CF720090244E7409F0E4A3F090244FE0FF04F0F3
:10CF8200EFC39432504B12CA8280EE200F4D12E052
:10CF920077EF640A704512887512C51A1292FA1256
:10CFA200C27190244E1246387004A3E064017012DC
:10CFB200201105124506800D901CA7E07007D20FC4
:10CFC200800312463F90244EE024FD600924FE7047
:0CCFD200BA12DCDF80B512AFEB80B02299
:10A22C0090244E7409F0E4902450F078517C247DF5
:10A23C00017BFF7A29794DFE7F04121C2312E077F3
:10A24C0090244FEFF012DFEFD20A300F0302A36815
:10A25C0012E07790244FE06F600302A3687F0490B4
:10A26C0024517401F0A3DFFC9015371243FFEC4D21
:10A27C004E4F600F9012C41243FFEC4D4E4F6003D3
:10A28C00301509E4902451F0902454F090244FE0C0
:10A29C0064096005E4902453F090193AE0D39403D8
:10A2AC004002E4F090193AE0FF2451F582E43424A2
:10A2BC00F583E0700890193AE004F080DC902450AB
:10A2CC00E0FD12A5D712C51A1292FA12C27190248F
:10A2DC004E1246387004A3E064017012201105126E
:10A2EC004506800D901CA7E07007D20F8003124624
:10A2FC003F90244EE024FD605B24FE602A24FE6027
:10A30C001A14600302A254902450E070047F018060
:10A31C00027F00902450EFF002A25490193AE0040E
:10A32C00F012DFFD02A25490193AE0B4020F90260D
:10A33C00DC1243FF90193F12204502A254901537AE
:10A34C001243FFEC4D4E4F700302A254C20A12701E
:0DA35C005602A254C20A12AFEB02A2542214
:10B4D60090244A7409F07BFF7A2879D57F0112CF30
:10B4E600DE7BFF7A2879E47F0212CFDE7BFF7A28A3
:10B4F60079ED901E3EE0902517F07F0312D2B590AD
:10B50600251774FFF0A37429F0A37400F0A374FF49
:10B51600F0A37429F0A37405F07BFF7A2879F77FEE
:10B526000412D2B57BFF7A2979109016691243FF6F
:10B536001245257F0512D2B512C51A908004E0F493
:10B5460030E6047F0180027F0090244BEFF0E4A3F5
:10B55600F0A3F0908004E0F4FF20E01790244CE480
:10B5660075F001121D43FCC3E5F09432EC6480943F
:10B5760080501190244BE07006EF30E602D20C1298
:10B58600C82B80CF12DFFD126848200F3312DFFD73
:10B5960012E077EF24FB601014601224FC6015247F
:10B5A60007701612D25080E212D63C80DD7F01125F
:10B5B600A0EA80D612CF7280D112A22CC20A80CA0B
:01B5C6002262
:10C3CC007581807590E775B0FFC290C293E4FFFE53
:10C3DC0012DFDF901D517404F0908002F07597FF0E
:10C3EC00758F7FE4F5AFF5D975D84075DA8275FA9B
:10C3FC00FF75EAFF75DB82F5FB75EBFFF5DCF5DD10
:10C40C00F5DE75985043892112E06DD28E758C4CF7
:10C41C00E4F58A75A892D28CF5C8D288D28A75B701
:10C42C000575B80712996E12C1BF1292FA90115984
:10C43C001243FF1218B912E05812D5ED90166DE0A8
:10C44C0070051277A1D20C12B4D612DFFD7BFF7AE5
:10C45C002979177F0312CFDE12C51A12D7B2E4FF67
:0BC46C00FE12DFDF12E063D29080FEC2
:10C27100901C9FE07002A3E0600A901CA9E0902549
:10C2810013F0801512DEFF902513EFF0C2A9901C68
:10C291009FE4F0A37402F0D2A9902513E0F9FD7C8C
:10C2A10000901CA8E0FAA3E0FBB50513ECB5020F62
:10C2B100901E3FE07002A3E060057E007F0922EB43
:10C2C100B5050EEAB5040A901CA5E4F0A304F080BC
:10C2D10007E4901CA5F0A3F0E9FF901CA8E4F0A3EB
:10C2E100EFF0C2A9901CA5E07002A3E0901E3F7080
:10C2F10007F0A37414F08006E4F0A3740AF0D2A945
:10C30100901CA8E0FEA3E0FF64094E6009EF640100
:0FC311004E600312DE44901CA8E0FEA3E0FF2262
:10DEFF007F09908004E0F4FEEED394004007EE25F6
:06DF0F00E0FE1F80F3227A
:10DE9C007C007D19121CF7E4901D7AF0A3F0D3904E
:0CDEAC001D7BE09F901D7AE09E40F32259
:10B0F400000000000000000000000000000000004C
:10B10400000000000000000000000000000000003B
:10B11400000000000000000000000000000000002B
:10B12400000000000000000000000000000000001B
:10B13400000000000000000000000000000000000B
:10B1440000000000000000000000000000000000FB
:10B1540000000000000000000000000000000000EB
:10B1640000000000000000000000000000000000DB
:10B1740000000000000000000000000000000000CB
:10B1840000000000000000000000000000000000BB
:10B1940000000000000000000000000000000000AB
:10B1A400000000000000000000000000000000009B
:10B1B400000000000000000000000000000000008B
:10B1C400000000000000000000000000000000007B
:10B1D400000000000000000000000000000000006B
:10B1E400000000000000000000000000000000005B
:0A09C3004126C8004125C700C19974
:09E08000EBF0A3EAF0A3E9F022A1
:0D0016009026C8E0FF9025C7E0C39FFF22A1
:10DDA1009025C7E0FF9026C8E0B507037F002290C9
:10DDB10026C8E0FF04F074C82FF582E43425F5830A
:03DDC100E0FF225E
:10DD08009025C7E02401FDE433FC9026C8E06D703F
:10DD180001EC60139025C7E0FE04F074C82EF5826C
:08DD2800E43425F583EFF0223D
:10DFA900120016EFD39400400612DDA18F9922D2F8
:02DFB90019222B
:10DF1500301905C21912DFA9C2A9901CA3E4F0A308
:06DF25007428F0D2A922CD
:10DF5700C2A9901CA3E07002A3E070047F018002B5
:05DF67007F00D2A92299
:07E08900902449E599F02203
:10DBAF0090258C12E080E4A3F090258CE0FBA3E09D
:10DBBF00FAA3E0F9A3E0F582758300121C62FF60FF
:0DDBCF000B12DD0890258FE004F080DD22B0
:10D4960090245E12E08078897C247D017BFF7AB03F
:10D4A60079F47E017F00121C239025897401F0A374
:10D4B6007424F0A37461F090245EE0F9A3E0FAA36B
:10D4C600E090258CC912E081902589E0F9A3E0FA65
:10D4D600A3E090258FC912E0817B017A2479891215
:0BD4E600D6D77B017A24798902DBAFE6
:102951004261636B6C6967687400005377697463E3
:1029610068206F666620696E6372656173650062D7
:10297100617474657279206C6966652062792033AF
:1029810030202500486569676874656E206261635F
:102991006B6C696768740000486569676874656E87
:1029A100206261636B6C6967687420696600776F88
:1029B100726B206F6E206578742E20706F77657250
:1029C100004F602063656C6C207573656400005373
:1029D1007769746368206F6666206966204F60209E
:1029E10063656C6C0069732064616D616765642067
:1029F1006F72206D697373696E67004F6020737524
:102A010062737469747574650041646A7573746185
:102A1100626C652076616C7565206966004F602087
:102A210063656C6C206E6F7420696E207573650030
:102A3100417665726167696E670000436F6D7075FD
:102A4100746520617665726167652076616C756574
:102A5100006F66206D65617375726564204865203D
:102A6100250056616C75657320746F206176672E41
:102A7100004E756D626572206F662076616C7565BA
:102A81007320666F7200617665726167696E672097
:102A91002869662075736564290053656E64206436
:102AA10061746120746F2055534200555342207266
:102AB100617465203131353230302062707300002D
:102AC1005061727469616C2070726573737572659F
:102AD100204F6000626172005573656420666F72F9
:102AE100204D4F440063616C63756C6174696F6E56
:102AF100005265662E2074656D702E20736F75729D
:102B010063650054656D70657261747572652066E8
:102B11006F72007072657373757265206573746985
:102B21006D6174696F6E005265662E2074656D70FB
:102B3100657261747572650054656D70657261745A
:102B410075726500446570746800446973706C61E6
:102B51007973206173206D6574657273206F7200E3
:102B610066656574206F662073616C74207761748B
:102B710065720050726573737572650000566F6CF3
:102B8100756D65000057656967687400436F6D7006
:102B91002E206C6576656C0043616C6962726174AC
:102BA100696F6E20707473004F602052454631008A
:102BB10025204F6000006D5600004F6020524546B1
:102BC10032004F602052454633004F602063616CF4
:102BD10069627261746564004F6020613020286110
:102BE10062736F6C75746529004F60206131202814
:102BF1006C696E65617229004F6020613220287115
:102C0100756164726174696329004F60207A65722D
:102C11006F2061646A7573740064697600004465AD
:102C21006C61792061697220667764006D730000C0
:102C310044656C6179206169722062776400446542
:102C41006C61792061742074656D702E0044656C2F
:102C510061792063616C6962726174656400566FA9
:102C61006C74207A65726F20706F730064697600EE
:102C7100566F6C7420636F656666696369656E740F
:102C8100006D562F646976004F686D207A65726F0A
:102C91002061646A75737400646976004F686D2001
:102CA100636F656666696369656E74007B2F64692D
:102CB1007600005072657373757265207A65726F64
:102CC1002061646A0064697600507265737375727D
:102CD1006520636F65660050612F64697600446505
:102CE1006D6F206D6F64650050756C736520776939
:102CF10064746800757300416C61726D204F6020CF
:102D01006C6F770025204F6000416C61726D204F20
:102D110060206869676800416C61726D20486520B8
:102D21006C6F77002520486500416C61726D204809
:102D310065206869676800416C61726D2070726519
:102D41007373206C6F770000496620657874657233
:102D51006E616C0073656E736F7220697320757399
:102D6100656400416C61726D2070726573732068D7
:102D71006967680049662065787465726E616C00E8
:102D810073656E736F72206973207573656400419A
:102D91006C61726D2054206C6F77004966206578F4
:102DA1007465726E616C00416C61726D20542068B3
:102DB1006967680049662065787465726E616C00A8
:102DC10044656C617920526531202D3E2052653277
:102DD10000730000507265737375726500496E74FB
:102DE10065726E616C20766F6C756D6500004F7851
:102DF1007967656E0025204F600048656C69756DC7
:102E01000025204865005072657373757265005521
:102E11007365203020666F7220756E6C696D697400
:102E2100656400736F757263652028636F6D7072DE
:102E31006573736F7229004F787967656E00486515
:102E41006C69756D00507265737375726500496EBA
:102E51007465726E616C20766F6C756D65004F786C
:102E61007967656E0048656C69756D0053746174AE
:102E710065206571756174696F6E00005265662E1B
:102E81002074656D706572617475726500257300DB
:102E91004E6F0059657300004F6666004F6E00006B
:102EA10043656C736975730046616872656E686528
:102EB100697400006D657465727300666565740000
:102EC100004F6666004C6F770048696768000049EB
:102ED1006465616C20676173005265616C20676194
:102EE1007300006261720070736900006C6974653F
:102EF1007200637562696320696E636800006B67C5
:102F0100006C620000416D6269656E740044656623
:102F1100696E65640000252E3066002531302E3043
:102F21006620257300252E3166002531302E31664D
:102F310020257300252E3266002531302E32662081
:102F41002573002531302E3366202573002531305D
:102F51002E3466202573002531302E3566202573E9
:102F6100002531322E3966202573002A0052616E08
:102F710067653A202573202D2025730043686F6F04
:102F810073652076616C7565007E46007E43006640
:102F91007377006D73770070736900637569004C16
:072FA100006C62006B670089
:1009CD00614A14D9FF2951FF295B0007400000003F
:1009DD0000000000400000000001FF295CFF2970AD
:1009ED000000000000FF2985FF299800003F8000CE
:1009FD0000000000003F8000000002FF2999FF2940
:100A0D00AF0000000000FF29C2FF29CF00013F8089
:100A1D000000000000003F8000000003FF29D0FF10
:100A2D0029E60000000000FF29FCFF29CF000B4143
:100A3D00A800000000000042C800000004FF2A0AC0
:100A4D00FF2A1E0000000000FF2A31FF2A3B000094
:100A5D003F800000000000003F8000000005FF2ADD
:100A6D003CFF2A520000000000FF2A63FF295B00B3
:100A7D000A412000004000000041A000000006FFD8
:100A8D002A72FF2A870000000000FF2A9BFF299889
:100A9D00000100000000000000003F800000000782
:100AAD00FF2AACFF2AC00000000000FF2AC1FF2A68
:100ABD00D5000B3FCCCCCD3E4CCCCD3FCCCCCD00DE
:100ACD0008FF2AD9FF2AE60000000000FF2AF2FFE6
:100ADD002998000900000000000000003F80000080
:100AED000009FF2B04FF2B140000000000FF2B2832
:100AFD00FF2998010B41A00000C1A0000042480051
:100B0D0000000AFF2998FF2998000000000060A549
:100B1D00195AFF2B39FF2998000200000000000030
:100B2D0000003F8000000014FF2998FF2998000065
:100B3D00000000FF2B45FF29980003000000000076
:100B4D000000003F8000000015FF2B4BFF2B6100C4
:100B5D0000000000FF2B74FF2B7D0004000000003F
:100B6D00000000003F8000000016FF2B7DFF2B7D55
:100B7D000000000000FF2B7EFF2B8500050000000C
:100B8D0000000000003F8000000017FF2B85FF2BA9
:100B9D00850000000000FF2B86FF2998000600004D
:100BAD000000000000003F8000000018FF2998FFA2
:100BBD0029980000000000639C113DFF2B8DFF2B39
:100BCD0085000A433E000000000000437F00000046
:100BDD001EFF2B85FF2B850000000000FF2B99FFCA
:100BED00295B000A3F8000003F800000404000006C
:100BFD00001FFF295BFF295B0000000000FF2BA9F0
:100C0D00FF2BB1000B41A800000000000042C800FE
:100C1D00000020FF2BB6FF2BB60000000000FF2BBD
:100C2D00A9FF2BB7000C410800000000000042573F
:100C3D00851F0021FF2BBAFF2BBA0000000000FF1B
:100C4D002BA9FF29CF010B41A0000000000000429D
:100C5D004800000022FF29CFFF29CF00000000002F
:100C6D00FF2BBBFF2BB1000B42C8000000000000A2
:100C7D0042C800000023FF2BB6FF2BB6000000007A
:100C8D0000FF2BBBFF2BB7000C420C000000000037
:100C9D00004257851F0024FF2BBAFF2BBA0000001E
:100CAD000000FF2BBBFF29CF010B41A0000000006E
:100CBD000000424800000025FF29CFFF29CF00008A
:100CCD00000000FF2BC3FF2BB1000B000000000044
:100CDD0000000042C800000026FF2BB6FF2BB60017
:100CED0000000000FF2BC3FF2BB7000C3F33333345
:100CFD00000000004257851F0027FF2BBAFF2BBABB
:100D0D000000000000FF2BC3FF29CF010B41A00005
:100D1D000000000000424800000028FF29CFFF29F5
:100D2D00CF0000000000FF2BCBFF29CF00000000FB
:100D3D000000000000003F8000000029FF29CFFFC8
:100D4D0029CF0000000000FF2BD9FF29CF00100094
:100D5D00000000C120000041200000002AFF29CF23
:100D6D00FF29CF0000000000FF2BEAFF29CF001064
:100D7D0000000000C120000041200000002BFF29D1
:100D8D00CFFF29CF0000000000FF2BF9FF29CF0076
:100D9D001000000000C120000041200000002CFFC9
:100DAD0029CFFF29CF0000000000FF2C0BFF2C1ACC
:100DBD00000A00000000C500000045000000002DE5
:100DCD00FF2C1EFF2C1E0000000000FF2C1FFF2C0F
:100DDD002D000D4026666600000000412000000039
:100DED002EFF2C30FF2C300000000000FF2C31FFB7
:100DFD002C2D000D402666660000000041200000ED
:100E0D00002FFF2C30FF2C300000000000FF2C3F86
:100E1D00FF2998010C41A00000000000004248008D
:100E2D00000030FF2998FF29980000000000FF2CDA
:100E3D004EFF2998000000000000000000003F80D8
:100E4D0000000031FF2998FF29980000000000FFE5
:100E5D002C5FFF2C6D000A450000000000000045CE
:100E6D007FF0000032FF2C1EFF2C1E000000000042
:100E7D00FF2C71FF2C82000D41A00000000000002E
:100E8D0042C800000033FF2BBAFF2BBA0000000050
:100E9D0000FF2C89FF2C99000AC5000000C57FF0CA
:100EAD0000000000000034FF2C1EFF2C1E0000006F
:100EBD000000FF2C9DFF2CAD000F3F028F5C00004A
:100ECD000000400000000035FF2CB3FF2CB30000E4
:100EDD00000000FF2CB4FF2CC6000A00000000002B
:100EED00000000457FF0000036FF2C1EFF2C1E0079
:100EFD0000000000FF2CCAFF2CD8000B4618966688
:100F0D000000000047C350000037FF295BFF295B3D
:100F1D000000000000FF2CDFFF29980000000000FA
:100F2D000000000000400000000038FF2998FF2954
:100F3D00980000000000FF2CE9FF2CF5000A41701D
:100F4D00000000000000428C00000039FF2C30FF33
:100F5D002C30000000000061291685FF2CF8FF2DB4
:100F6D0005000B41A000000000000042C800000079
:100F7D0046FF2BB6FF2BB60000000000FF2D0AFF29
:100F8D002D05000B421400000000000042C80000B7
:100F9D000047FF2BB6FF2BB60000000000FF2D18F9
:100FAD00FF2D25000B000000000000000042C800CE
:100FBD00000048FF2BB6FF2BB60000000000FF2DF0
:100FCD002AFF2D25000B42C800000000000042C87A
:100FDD0000000049FF2BB6FF2BB60000000000FFFC
:100FED002D38FF2D48030B000000000000000043CA
:100FFD00FA0000004DFF2D49FF2D550000000000A7
:10100D00FF2D64FF2D48030B434800000000000036
:10101D0043FA0000004EFF2D75FF2D8100000000EA
:10102D0000FF2D90FF2D48010B00000000C25C0059
:10103D000042FA0000004AFF2D9CFF2D81000000A8
:10104D000000FF2DA8FF2D48010B42480000C25C97
:10105D00000042FA0000004BFF2DB5FF2D8100006E
:10106D00000000FF2DC1FF2DD2000A41F00000004D
:10107D0000000044160000004CFF2DD4FF2DD400BD
:10108D0000000000629419FFFF2DD5FF2B7D030B8F
:10109D00000000000000000043FA00000064FF2B78
:1010AD007DFF2B7D0000000000FF2DDEFF2DEE04E7
:1010BD000B41C000000000000042C600000065FFAB
:1010CD002DEEFF2DEE0000000000FF2DEFFF2DF6A1
:1010DD00000B41A800000000000042C8000000669F
:1010ED00FF2BB6FF2BB60000000000FF2DFBFF2EDF
:1010FD0002000B000000000000000042C8000000CC
:10110D0067FF2BB6FF2BB60000000000FF2E07FF78
:10111D002B7D030B434800000000000043FA000044
:10112D000068FF2B7DFF2B7D0000000000FF2DDEF2
:10113D00FF2DEE040B424800000000000042C600E7
:10114D00000069FF2E10FF2E240000000000FF2E6E
:10115D0038FF2DF6000B000000000000000042C813
:10116D000000006AFF2BB6FF2BB60000000000FF49
:10117D002E3FFF2E02000B42C8000000000000426F
:10118D00C80000006BFF2BB6FF2BB600000000005F
:10119D00FF2E46FF2B7D030B43480000000000008F
:1011AD0043FA0000006CFF2B7DFF2B7D000000003B
:1011BD0000FF2E4FFF2DEE040B42480000000000F3
:1011CD000042C60000006DFF2E10FF2E240000000F
:1011DD000000FF2E38FF2DF6000B42C80000000066
:1011ED00000042C80000006EFF2BB6FF2BB60000BA
:1011FD00000000FF2E3FFF2E02000B00000000003C
:10120D0000000042C80000006FFF2BB6FF2BB60098
:10121D0000000000FF2E46FF2B7D030B43A50000B1
:10122D000000000043FA00000070FF2B7DFF2B7DB6
:10123D000000000000FF2E4FFF2DEE040B000000FC
:10124D00000000000042C600000071FF2E10FF2EAE
:10125D00240000000000FF2E38FF2DF6000B41A8E2
:10126D0000000000000042C800000072FF2BB6FF16
:10127D002BB60000000000FF2E3FFF2E02000B00DA
:10128D000000000000000042C800000073FF2BB6F4
:10129D00FF2BB60000000000FF2E46FF2B7D030B39
:1012AD00434800000000000043FA00000074FF2BCB
:1012BD007DFF2B7D0000000000FF2E4FFF2DEE0463
:1012CD000B41C000000000000042C600000075FF89
:1012DD002DEEFF2DEE0000000000FF2DEFFF2DF68F
:1012ED00000B419000000000000042C80000007695
:1012FD00FF2BB6FF2BB60000000000FF2DFBFF2ECD
:10130D0002000B422000000000000042C800000057
:10131D0077FF2BB6FF2BB60000000000618C17AED7
:10132D00FF2E07FF2B7D030B42480000000000003D
:10133D0043FA00000082FF2B7DFF2B7D0000000093
:10134D0000FF2E5FFF2DF6000B41A80000000000EE
:10135D000042C800000083FF2BB6FF2BB600000033
:10136D000000FF2E66FF2E02000B000000000000A3
:10137D00000042C800000084FF2BB6FF2BB6000012
:10138D00000000FF2E07FF2B7D030B4248000000DD
:10139D0000000043FA00000085FF2B7DFF2B7D0030
:1013AD0000000000FF2E5FFF2DF6000B0000000077
:1013BD000000000042C800000086FF2BB6FF2BB6D0
:1013CD000000000000FF2E66FF2E02000B42C80039
:1013DD00000000000042C800000087FF2BB6FF2B65
:1013ED00B60000000000FF2E07FF2B7D030B4248C7
:1013FD0000000000000043FA00000088FF2B7DFF75
:10140D002B7D0000000000FF2E5FFF2DF6000B422C
:10141D00C800000000000042C800000089FF2BB684
:10142D00FF2BB60000000000FF2E66FF2E02000B02
:10143D00000000000000000042C80000008AFF2BE1
:10144D00B6FF2BB60000000000FF2E07FF2B7D031B
:10145D000B424800000000000043FA0000008BFF23
:10146D002B7DFF2B7D0000000000FF2E5FFF2DF672
:10147D00000B41A800000000000042C80000008CD5
:10148D00FF2BB6FF2BB60000000000FF2E66FF2ECF
:10149D0002000B000000000000000042C800000028
:1014AD008DFF2BB6FF2BB600000000006042162307
:1014BD00FF2E6DFF2E7C00080000000000000000D4
:1014CD003F8000000096FF2E7CFF2E7C0000000068
:1014DD0000FF2E7DFF2998010B41A00000C25C008A
:1014ED000042FA00000097FF2998FF29980000009C
:1014FD0000006020111D010003000300000000002A
:10150D0000000000000000000000000000000000CE
:08151D00000000000000C11AEB
:107E4500A3F090250FE0FCA3E0FDA3E0FEA3E0FF77
:107E550090259812204590250BE0FBA3E0FAA3E0BE
:107E6500F92274FFF0A3742FF07435A3F090250F59
:107E7500E0FCA3E0FDA3E0FEA3E0FF2290000C12CE
:107E85001F4F9024CCE0F8A3E0F9A3E0FAA3E0FBB0
:107E95001215629024D7E0F8A3E0F9A3E0FAA3E075
:107EA500FB2290000312210C90259CEBF0A3EAF035
:107EB500A3E9F02290244FE090244A75F021A4FF15
:107EC500E0FBA3E0FAA3E02FF9EA35F0FA229000EF
:107ED5001C021F4F9024BCE0FBA3E0FAA3E0241C86
:107EE500F9E43AFA2290000C121F99900010021F33
:107EF5004F90001C121F9990000C021F4F1218B9C9
:107F0500AD077BFF2290250F1220459025137401A4
:107F1500F0A37424F0A374DFF02290166EE0648061
:107F25009480227B017A1979FF7D147C00227B01E4
:107F35007A1679857D097C0022E0FF3395E0FE7C89
:107F4500007D21121CE5902492E0FBA3E0FAA3E05A
:107F55002FF9EA3EFA2290250EE0902595229024ED
:107F6500C9F09024C5227B017A1779AE7D0C7C007F
:107F750022902598022045EEF0A3EFF0A3ECF0A3A4
:107F8500EDF0229024C9F09024C522E4FBFAF9F81B
:107F95000217FD7E007F207D007B017A1679652220
:107FA50090245CE075F021A4FF9024572274019081
:107FB5000020021CC37B017A1479D97D0A22783A04
:107FC5007C197D017B017A11791D7E007F2022902D
:107FD500001C021F99EC4D4E4F7BFF227B017A243A
:107FE5007998227B017A19795A7D057C00227B01DB
:107FF5007A11793D7D1C7C0022FFFDD3E09D7480C4
:10800500F8229024C1022045C2A9D211901CA77460
:1080150028F0D2A9229024D70220457A19793A7DF1
:10802500207C007F807E01227401F0A37424F0A3DC
:1080350074F5F0229024C9F09024C5227B017A16AC
:1080450079237D0222900014121D59AEF078022288
:1080550075F003A4C58325F0C58322900007021C93
:0180650062B8
:10D04900902494127F7CA3127EB0E4A3F0A3F09005
:10D05900249BF0A3F0902496E0FEA3E0FFC3902464
:10D069009CE09F90249BE09E503E902495E0FF9089
:10D079002494E0FD902498127E5EA3E0F8A3E0F5E5
:10D08900828883121C62FB12E00B902495E004F065
:10D099007006902494E004F090249CE004F070B5AC
:09D0A90090249BE004F080AD220C
:10D0B200902450127F7CA3127EB0E4A3F0A3F090E0
:10D0C2002457F0A3F0902452E0FEA3E0FFC3902483
:10D0D20058E09F902457E09E503E902451E0FF90EC
:10D0E2002450E0FD12E019902454127E5EA3E0FC6D
:10D0F200A3E0F5828C83EF121CC3902451E004F06C
:10D102007006902450E004F0902458E004F070B5CA
:09D11200902457E004F080AD22E6
:10D1840090248E127EB0127F81E4A3F0902493E069
:10D19400902492127FFE902491E06480984047EF9F
:10D1A40090248E127EC0900020121C62602F128088
:10D1B4004AC333CE33CED8F92400FDEE3402FC90BA
:10D1C4002493E075F021A4FF90248E127EC5E91209
:10D1D4007EE3AF05AE047D047C0012D04990249315
:07D1E400E004F002D19022EB
:10D4F10090244A127EB0127F81E4A3F090244FE081
:10D5010090244E127FFE90244DE06480984037EFC6
:10D51100127EBD12804AC333CE33CED8F92400FD2A
:10D52100EE3402FC127EB9E9127EE3AF05AE047D52
:10D53100047C0012D0B2127EB9E4127FB490244F61
:07D54100E004F002D4FD221A
:10D3DE00902457127EB0127F81E4A3F090245CE07B
:10D3EE00FFFDD390245BE09D7480F890245AE06496
:10D3FE0080984038EF127FA9127EC5E92408F9E41F
:10D40E003AFA121F2FC006C007127FA5127EC7E977
:10D41E00127EE3D007D006121F7F127FA5127EC5A3
:0DD42E00127FB290245CE004F002D3EA22E9
:1086890090250EEDF090250B127EB0128060B4118A
:1086990000400302885D9086A6F82828730286D9CF
:1086A9000286E60286F302870002872602873202E3
:1086B900873E02870D02871A02874A02876D028761
:1086C900960287BF0287DF0287FF02881F02883E62
:1086D900127E72127F027A2E7991028754127E726B
:1086E900127F027A2E7999028754127E72127F02C2
:1086F9007A2E79A1028754127E72127F027A2E791C
:10870900B5028754127E72127F027A2E79C20287CD
:1087190054127E72127F027A2E79D0802E127E72C6
:10872900127F027A2E79E48022127E72127F027AF7
:108739002E79ED8016127E72127F027A2E79FF80D1
:108749000A127E72127F027A2F790612D84090257A
:1087590098127EB090259574FFF0A3742EF0A3743F
:108769008E02886A127F5B601274FFF0A3742FF087
:108779007417127E70127F7602886B74FFF0A374EF
:108789002FF0741C127E45127EA702886B127F5B44
:10879900601274FFF0A3742FF0A37426127E711275
:1087A9007F76800F74FFF0A3742FF0742B127E452F
:1087B900127EA702886B127F5B6008127E67127FA8
:1087C90076801074FFF0A3742FF0A3743A127E46DA
:1087D900127EA702886B127F5B6008127E67127F88
:1087E90076801074FFF0A3742FF0A37444127E46B0
:1087F900127EA702886B127F5B6008127E67127F68
:1088090076801074FFF0A3742FF0A3744E127E4685
:10881900127EA702886B127F5B6008127E67127F47
:1088290076801074FFF0A3742FF0A37458127E465B
:10883900127EA7802D127F5B6008127E67127F76F9
:10884900801074FFF0A3742FF0A37462127E461295
:108859007EA7800E90259574FFF0A3742FF0A37462
:0C8869006CF0902513127E5E123B502232
:10B86E009024DEEDF09024DB127EB01220EC7F01EE
:10B87E0012CFDE9024DB127E5E127ED3127F0A90F0
:10B88E0024DB127E5EE4FD1286899024DEE0902594
:10B89E0017127F137BFF7A2E798E7F0212D2B5900C
:10B8AE0024DEE0606A9024DB127E5E128060C39418
:10B8BE000A404FC003C002C0019024DBA3A3E012D4
:10B8CE007EFC127F0AD001D002D0037D0112868940
:10B8DE009024DB127E5E127EF090250F1220459092
:10B8EE00251312802D9024DB127E5E7D0112868937
:10B8FE00902517127F13A312802D7BFF7A2F796E5E
:10B90E0080067BFF7A2F797D7F0312D2B5800B7B69
:10B91E00FF7A29795B7F0312CFDE9024DB127E5EE5
:10B92E0090001612210C7F0412CFDE9024DB127EC3
:0FB93E005E90001912210C7F0512CFDE02C51A90
:104865009024B9127EB0127ED39024BD122045E467
:104875009024CAF09024D004F0A304F012806024A0
:10488500F6B407004003024910904895128055730D
:104895000248AA0248B80248C60248D40248E202C1
:1048A50048F00248FE74FF127F631220513F8000DA
:1048B5000080677401127F631220513DCCCCCD80FE
:1048C500597402127F881220513C23D70A804B74F9
:1048D50003127F881220513A83126F803D740412AF
:1048E500803912205138D1B717802F7405128039BD
:1048F5001220513727C5AC80219024C97409F09046
:1049050024C51220513089705F800F9024C5122074
:10491500513F800000E49024D0F0E4FBFA79407820
:10492500409024C5127E751217609024CC12204544
:104935009024CB740AF09024C5127E7512800790DE
:1049450024B9127E5E124C996003024B1C300F0392
:10495500024C9812C51A1292FA12C2719024BCEF39
:10496500F0901CA8E07004A3E0640170122011050A
:1049750012800D8010901CA7E0700AD20F8006C22D
:10498500A9C211D2A99024BCE024FEB4070050BDF1
:1049950090499C128055730249B1024C3D0249FB76
:1049A500024AF7024A70024B200249C89024BD1200
:1049B5007E759024B9127E5E127FD47D0112B86E89
:1049C500024C959024B9127E5E127ED312E0279098
:1049D50024CC127E9B1217FD40109024B9127E5EE6
:1049E50090001C12209C000000009024B9127E5EED
:1049F500127FB2024C959024B9127E5E127ED312BC
:104A05007F9050249024B9127E5E127ED39024C1EB
:104A1500127E9B1217FD6010400E9024B9127E5E27
:104A2500127ED312186A80129024B9127E5E127E0D
:104A3500D39024C1127E9B12156212801A9024B95C
:104A4500127E5E127E811217FD400F9024D7127ED2
:104A5500759024B9127E5E127FD49024B9127E5EC1
:104A6500124C997003024952024B1C9024B9127ED4
:104A75005E127ED3127F90602940279024B9127E62
:104A85005E127ED312186A9024C1127E9B1217FD06
:104A95006010400E9024B9127E5E127ED312186A01
:104AA50080129024B9127E5E127ED39024C1127EAC
:104AB5009B12156612801A9024B9127E5E127EF042
:104AC5009024CC127E9B121566127E981217FD60FB
:104AD50002500F9024D7127E759024B9127E5E1273
:104AE5007FD49024B9127E5E124CA3700302495202
:104AF50080259024B9127E5E900008121F4F127F08
:104B0500D4E49024CAF09024C5127E751280071251
:104B15004CA37003024952A3024C769024D0E07056
:104B250003024952E4FFFE7D207C419024C1127EA0
:104B35009B1216579024D3122045E49024D2F0906E
:104B450024B9127E5E127ED3127F9050249024B930
:104B5500127E5E127ED39024D3127E9B1217FD60C7
:104B650010400E9024B9127E5E127ED312186A8010
:104B7500129024B9127E5E127ED39024D3127E9BAE
:104B850012156212801A9024B9127E5E127E81126D
:104B950017FD40069024D27401F09024B9127E5E70
:104BA500127ED3127F90602940279024B9127E5E31
:104BB500127ED312186A9024D3127E9B1217FD60C1
:104BC50010400E9024B9127E5E127ED312186A80B0
:104BD500129024B9127E5E127ED39024D3127E9B4E
:104BE50012156612801A9024B9127E5E127EF0901C
:104BF50024CC127E9B121566127E981217FD600258
:104C050050069024D27401F09024D2E060179024CD
:104C1500CAE004F09024C9E0FFA3E0B5070204F060
:104C25009024D38008E49024CAF09024C5127E75A0
:104C35001280079024D180399024D0E07003024976
:104C4500529024CAE0D3648094804022E014F0900E
:104C550024C9E0FFA3E0B5070214F09024C1127E39
:104C650075E4FBFA792078411217601280079024C9
:104C7500D1E0FF9024CAE0FD3395E0FCA3E0FB33CF
:104C850095E0FAC3EB9DFDEA9CFC12DAF20249526B
:104C950012DF81227D0112B86E9024D0E0227D01C1
:084CA50012B86E9024D0E02249
:10849C009024B9127EB09024B9E0FBA3E0FAA3E0DB
:1084AC00F8AC02AD03A3127E5E7E007F21121C236A
:1084BC009024B9127E5E900006121C6224FE606845
:1084CC001470030285831470030285D214700302A6
:1084DC00862124046003028688901976127E751218
:1084EC007FDA603D7A2F798AC003C002C0019024E4
:1084FC00B9127E5E90000312213C9024B9127E5E6C
:10850C00127ED312DCB59024B9127E5E127EF61266
:10851C00DCB59024B9127E5E127EEA12DCB50286BE
:10852C00667A2F798D028676901997127E75127F56
:10853C00DA603D7A2F7990C003C002C0019024B953
:10854C00127E5E90000312213C9024B9127E5E12C2
:10855C007ED312DF2B9024B9127E5E127EF612DFD0
:10856C002B9024B9127E5E127EEA12DF2B028666F5
:10857C007A2F79940286769019B8127E75127FDA6A
:10858C00603D7A2F7998C003C002C0019024B912C3
:10859C007E5E90000312213C9024B9127E5E127E06
:1085AC00D312DEB89024B9127E5E127EF612DEB8BB
:1085BC009024B9127E5E127EEA12DEB80286667ACA
:1085CC002A79D50286769019D9127E75127FDA60D7
:1085DC003D7A2F799CC003C002C0019024B9127E51
:1085EC005E90000312213C9024B9127E5E127ED361
:1085FC0012DED09024B9127E5E127EF612DED0907E
:10860C0024B9127E5E127EEA12DED00286667A2FC2
:10861C0079A00286769019FA127E75127FDA60467E
:10862C007A2F79A2C003C002C0019024B9127E5ED9
:10863C0090000312213C9024B9127E5E127ED3125C
:10864C00DF419024B9127E5E127EF612DF41902437
:10865C00B9127E5E127EEA12DF419024B9127E5E60
:10866C00900010021F997A2F79A5C003C002C00197
:0D867C009024B9127E5E90000312213C2272
:10A707009024B9127EB09024B9127E5E9000201278
:10A717001C62700302A833900006121C6224FE60BC
:10A727004014606A14700302A7C214700302A7EDF5
:10A737002404600302A818901976127E75EC4D4E1A
:10A747004F6048127ED9C003C002C0019024B912DD
:10A757007E5E127ED3D001D002D00312D8C902A8E0
:10A767002A901997127E75EC4D4E4F601E127ED9B6
:10A77700C003C002C0019024B9127E5E127ED3D0FE
:10A7870001D002D00312DBDC02A82A02A818901914
:10A79700B8127E75EC4D4E4F601E127ED9C003C0B5
:10A7A70002C0019024B9127E5E127ED3D001D0027E
:10A7B700D00312DB2302A82A02A8189019D9127E07
:10A7C70075EC4D4E4F601D127ED9C003C002C0010B
:10A7D7009024B9127E5E127ED3D001D002D003122C
:10A7E700DB52803F802B9019FA127E75EC4D4E4F4D
:10A7F700601D127ED9C003C002C0019024B9127E29
:10A807005E127ED3D001D002D00312DC09801480FF
:10A81700009024B9127E5E127ED39024BC127E5E15
:0DA82700127FD49024BC127E5E127FB222FC
:10BBBA00902492127EB0A3EDF0E490249702BC6622
:10BBCA00300F0302BC8412C51A1292FA12C2719083
:10BBDA002496EFF0901CA8E07004A3E064017012B0
:10BBEA0020110512800D8010901CA7E0700AD20F58
:10BBFA008006C2A9C211D2A9902496E024FE6077D9
:10BC0A0024FE602B24FE604424FE70B4127FE112ED
:10BC1A004865127FE1E4FD12B86E902497127F3EC8
:10BC2A009024BC127EB0127FE112A70702BBCA9011
:10BC3A002495E014FF902497E0FEC3EF6480F8EEA9
:10BC4A00648098400302BBCAE0048010902497E005
:10BC5A00D364809480500302BBCAE014F0127F3E82
:10BC6A009024BC127EB0127FE112849C127FE1E420
:0BBC7A00FD12B86E02BBCA12DFFD22F3
:10996E00127F981221BB127F9E7D207C00E4FFFEA9
:10997E0012D0B27F067E8C7DE37C49901665127EF6
:10998E009BC3121F1E6003029A89127FBAFC12D467
:10999E00F17A19795A7D05129AFC127FF512D4F1DB
:1099AE00127F3312D4F1127F2812D4F1127F6B1270
:1099BE00D4F1128043129AFC12802012D0B2C390BE
:1099CE00166FE09407127F1F50097A17798D129A3D
:1099DE00BFD21AC390166FE09408127F1F500E125A
:1099EE007F6B12D3DE90193E7403F0D21AC3901619
:1099FE006FE09409127F1F501E7A147955129ABF88
:109A0E007A147976129AC97A177909129AC97A173D
:109A1E00792A129AE8D21AC390166FE0940A127F2E
:109A2E001F500B7A1579C07D01129AD3D21AC390AA
:109A3E00166FE0940B127F1F50097A147997129AC1
:109A4E00E8D21AC390166FE0940D127F1F50097A58
:109A5E001479B8129AF2D21AC390166FE0940E12BD
:109A6E007F1F504C7A1579E1129AF27B017A1679A2
:109A7E00027D017C0012D3DED21A22127F981221AF
:109A8E00BB127FBA7C0012D3DE127FE812D3DE1235
:109A9E007FF312D3DE127F3312D3DE127F2812D35E
:109AAE00DE7A1779AE7D0C129AD3127FC3121C2365
:109ABE00227B017D017C0012D3DE227B017D017CA5
:109ACE000012D3DE227B017C0012D3DE7B017A16DC
:109ADE0079237D027C0012D3DE227B017D017C0086
:109AEE0012D3DE227B017D017C0012D3DE227B01AC
:089AFE007C0012D4F17B01226F
:10D7B200127FBC12D7F0127FEA12D1847A11793D1E
:10D7C2007D1C12D7F0127F3512D184127F2812D11C
:10D7D20084127F6B12D1841280417C0012D1847B2F
:10D7E2000112802012D049301A0312DDE6227B0199
:08D7F2007C0012D1847B0122AE
:10DDE60090166512205149E38C0690166EE4F0A356
:10DDF600740EF0127F9E7D207C00E4FFFE02D04967
:10DB8100127FBA7C0012D3DE127FE812D3DE127F3D
:10DB91003312D3DE127F2812D3DE127F6B12D3DE53
:0EDBA1001280417C0012D3DE127FC3021C23CF
:10DFBB00127FF312D184127F3312D184127F280285
:02DFCB00D184FF
:0AE06D00758DFF758BFF438780223D
:10AB9D00532F4E3A202530396C7500556E706C75FB
:10ABAD006720534554555000446973636F6E6E654D
:10ABBD0063742074657374206361626C65005072F8
:10ABCD0065737320456E74657200506C7567205304
:10ABDD004554555020636F6E6E6563746F720043FC
:10ABED006F6E6E6563742074657374206361626C3F
:10ABFD006500412F442030206F70656E202020208D
:10AC0D00202025352E3064002020202020203435B2
:10AC1D002E323030206D562025352E306400202008
:10AC2D002020202020382E343830206D5620253518
:10AC3D002E30640020202020202020312E37353565
:10AC4D00206D562025352E3064004F4B3D456E74DA
:10AC5D0065722020202041626F72743D4573630040
:10AC6D00412F442030004C696E6561726974792002
:10AC7D00313A2025362E3266202525004C696E6529
:10AC8D00617269747920323A2025362E326620257C
:10AC9D002500436F6D70656E736174696F6E3A2038
:07ACAD00252B352E30660057
:10C9590090246CE0FCA3E0FDA3E0FEA3E0FF22E04D
:10C96900FCA3E0FDEC121880901348E0F8A3E0F96D
:10C97900A3E0FAA3E0227BFFE0FFA3E0902517CF15
:10C98900F0A3EFF022121760E4FBFA79C87842129B
:10C999001657E4FBFA79C878C2021566EEF0A3EFE0
:10C9A900F07B017A24794A22E0FCA3E0FDEC12181D
:10C9B90080A804A905AA06AB0722FB1215667B36D7
:10C9C9007A947957783C021657C2A9D211901CA7BC
:10C9D9007428F0D2A922902517022045E0FCA3E093
:05C9E900FDEC021880C6
:109E150090246512205105F5E1009024697408F03D
:109E2500A3740EF0A37403F090166912C95C029F27
:109E35001C300F03029F6312C51A1292FA12C271E7
:109E4500902464EFF0901CA8E07004A3E064017016
:109E55001220110512C9D28010901CA7E0700AD2F9
:109E65000F8006C2A9C211D2A97BFF7AAB799D12D8
:109E7500C95912C9DF90246BE0FF12D2B5129F6455
:109E850012C51A902464E024FE7003029F6024FE2C
:109E9500601924FE6043147003029F25147092120A
:109EA500C959901669122045029F6090246512C910
:109EB5005C90246C12C974FBC3121F1E5003029ED2
:109EC5003612C95990246512C974FBEF9BFFEE9AAF
:109ED500FEED99FDEC98FC803E90246512C95C90DE
:109EE500246C12C9742FFFEA3EFEE93DFDE83CFCF7
:109EF5007BFF7AC9799A783BC3121F1E5003029ED5
:109F05003612C95990246512C974FBEF2BFFEE3A3E
:109F1500FEED39FDEC38FC90246C122045029E368E
:109F2500902469E0D364809480401AE014F0902472
:109F35006512C95CE47B0AFAF9F8121E689024657B
:109F450012204580109024697408F0902465122031
:109F55005105F5E100129F64029E3612DFFD229045
:109F6500246BE0FF902469E0FD3395E0FCA3E0FB62
:0F9F75003395E0FAC3EB9DFDEA9CFC12DAF22271
:10D59C009024647409F012C51A12C51A1292FA1268
:10D5AC00C271902464EFF0901CA8E07004A3E064B6
:10D5BC0001701220110512C9D28010901CA7E070C6
:10D5CC000AD20F8006C2A9C211D2A9200F0890243A
:10D5DC0064E0FFB40204D29080FEEFB408BB02DF1B
:01D5EC00FD41
:1077A10090244B7409F012DFFD7BFF7AAB79A87F3F
:1077B1000212CFDE7AAB79B51279ABE4FF12DDC4E8
:1077C10090244CEEF0A3EFF07F0112DDC49024541D
:1077D1001279E7902458EEF0A3EFF07BFF7AAB79B2
:1077E100D77F0212CFDE7AAB79EC1279AB7FF47ED0
:1077F1000112DE9C7F0112DDC49024561279E790BC
:10780100245A12C9A57D017F0112DA58127997E431
:10781100FD1279C190244E12C9A5E4FD7F0112DA4F
:107821005812C9AA7D017F0212DA587FF47E011233
:10783100DE9CE4FF12DDC4902450EEF0A3EFF012C1
:1078410079977D011279C190245212C9A5E4FD7F77
:107851000312DA587AAB79FF90244C12C97F7F0169
:1078610012D2B57AAC791590244E12C97F7F0212DB
:10787100D2B57BFF7AAC792B90245012C9817F035A
:1078810012D2B57BFF7AAC794190245212C9811290
:1078910079D390245412C9E59013ED122045901329
:1078A100F17401F090245612C9B19013ED12C95C24
:1078B10012156212C9BAE4FFFE7D807C4512176081
:1078C10090140E1220459014127401F090245A1253
:1078D100C9E512186A90142F1220459014337401CF
:1078E100F090245212C9B17F487E617D057C43121C
:1078F100156290134812204590134C7401F09024A6
:107901004E12C96812C9C37BCD7ACC793478421240
:10791100C98E90245C12204590245012C96812C966
:10792100C37B147AAE7907784112C98E9024601214
:1079310020457BFF7AAC796D7F0112D2B57BFF7A4E
:10794100AC797390245C12C95C12C9DF7F0212D238
:10795100B57BFF7AAC798990246012C95C12C9DFCA
:107961007F0312D2B57BFF7AAC799F90134812C97D
:107971005C12C9DF1279D3129E15E4FFFEFDFC9063
:10798100166912C974FBC3121F1E600990166D742B
:1079910001F012DDE6227B017A24794AE4FD7F02BF
:1079A10012DA587B017A24794A227BFF7F0312CFB6
:1079B100DE7BFF7AAB79CB7F0512CFDE12D59C221D
:1079C1007F0312DA587FF47E0112DE9CE4FF12DDA0
:1079D100C4227F0412D2B57BFF7AAC79577F05129E
:1079E100CFDE12D59C22EEF0A3EFF07F0212DDC4B0
:0179F1002273
:10A4A100537465702536750044697363686172671A
:10A4B100652025372E3466202573006C62006B679A
:10A4C100004164642025372E3466202573202573CE
:10A4D100004469736368617267652025352E3166B2
:10A4E1002025730070736900626172004164642009
:10A4F10025352E3166202573202573004469736349
:10A50100682E20746F2025352E3166202573004179
:10A51100646420746F2025352E3166202573202533
:10A52100730050726573737572653A2025362E314A
:10A5310066202573007D2025362E3166205C20257E
:10A54100362E316620257300536F6C76696E670075
:10A551005068617365202020203100506861736567
:10A561002020202032004E6F20736F6C7574696F4C
:10A571006E2E005468657265206973206E6F7420B9
:10A58100656E6F75676800676173657320746F200E
:10A591006D616B650064657369726564206D6978CE
:10A5A100747572652E0000000000000000000000BC
:10A5B100000000000000000000000000000000009A
:10A5C100000000000000000000000000000000008A
:06A5D10000000000000084
:106271009025171220459019B8E0FCA3E0FDA3E09A
:10628100FEA3E0FF229024D1E0F8A3E0F9A3E0FA15
:10629100A3E0FBE4FFFEFD7C401215629024BAE00E
:1062A100FBA3E0FAA3E0F9121FF51216579024BAE6
:1062B100E0FBA3E0FAA3E0F9121F7F9024BAE0FB10
:1062C100A3E0FAA3E0F9121F2F9024E7E0F8A3E07E
:1062D100F9A3E0FAA3E0FB22F09024AFE0F9A3E0F8
:1062E100FAA3E09024BAC9F0A3EAF0A3E9F090245C
:1062F100B2E0F9A3E0FAA3E09024BDC9F0A3EAF06B
:10630100A3E9F09024A9E0FBA3E0FAA3E0F922902D
:106311002547E0FBA3E0FAA3E02408F9E43AFA9068
:106321002561E075F004A4F58285F08322122045F1
:106331009024B5E0FFA3E0F9A3E0FAA3E0902511D2
:10634100C9F0A3EAF0A3E9F0A37401F0A37424F067
:1063510074F8A3F0A37401F0A32290251BEBF0A322
:10636100EAF0A3E92290257D122045902581740150
:10637100F0A3229024C9E075F018A4244CF582E41E
:106381003427F58322121566A804A905AA06AB07CE
:1063910022902547E0FBA3E0FAA3E02408F9E43AC0
:1063A100FA22121760902561E025E025E02462F5CC
:1063B10082E43425F583122045902561E004F0E064
:1063C10064042290253BE025E025E0241EF582E4CB
:1063D1003425F5832278D17C247B017A2479C17D0F
:1063E100017E007F10021C23E025E025E024C1F599
:1063F10082E43424F58322EF25E025E024AFF58201
:10640100E43424F58322121657E4FBFA797A7844AE
:106411001217609024D80220457F917E0F7D687C01
:1064210041229024CAE025E025E024B9F582E43434
:1064310024F5832290248AE075F018A42448F5827B
:10644100E43427F5832212156290255D122045E47C
:10645100FFFEFD22EC4D4E4F7BFF229025937401F0
:10646100F0A3229024CBE0FF04F022F58312204513
:106471009024D5E004F022121F2F9024E71220452A
:106481009024C0E09024F3F09024E122902596021C
:1064910020459024C0E025E025E024D1F582E434B4
:1064A10024F58322121F2FE4FBFAF9F80217FD905D
:1064B100259A0220457424F0A374CCF07BFF227549
:1064C100F018A42450F582E43427F583229024D5D2
:1064D100E0FFD394032225E025E0248FF582E43404
:1064E10024F58322900004021F4FC2A9D211901CEF
:1064F100A77428F0D2A922121F2F9024EB2225E0A5
:1065010025E024ACF582E43427227F897E187D0DB5
:106511007C409024D8227B0A7AD77923783C0217D1
:10652100FD7425F0A37472F090253F227425F0A329
:10653100744DF090255D227425F0A37455F09025DB
:106541003F227B017A2479F89025082290251712A1
:1065510020459019FA227F9A7E997C3F90249F22B0
:105C2D0090253C12635EF0A3122045902547126328
:105C3D00071264A56003025D417B0190259304F07A
:105C4D00A312652212627A12648D90254312627A34
:105C5D001264B090253C126307125F446003025F2B
:105C6D002C9025471263071264E59025721262CDC0
:105C7D00126447FC90255D1262CD1217FD60025033
:105C8D0003025E14126392C00390253F12627A12D2
:105C9D00636612652D12627AD003125F4C600302A7
:105CAD005F2CE4902561F0126310121F4F90254D6B
:105CBD001262CD121657C004C005C006C00790254C
:105CCD003C126307126320121F4F9025431262CDC1
:105CDD00121657D003D002D001D000121566C004A1
:105CED00C005C006C00790254D12627A902543125B
:105CFD0062CD126386D007D006D005D0041263A3FF
:105D0D0070A512645C12653812627A12648D90254A
:105D1D004D12627A9025431262CD125F2D600302FF
:105D2D005F2C9025471263071264E590255512628A
:105D3D00CD025F0B12645C12652212627A12648DC1
:105D4D0090254312627A1264B090253C12630712BB
:105D5D005F446003025F2C126392C003C002C00156
:105D6D009025471263091264E5C004C005C006C042
:105D7D0007902547A3A3E0121F2F1263667425F029
:105D8D00A37451F0D007D006D005D004D001D002B5
:105D9D00D003125F4C6003025F2C902547126307FE
:105DAD001264E5121FF5121657C004C005C006C0D7
:105DBD000790257212627A90253F1262CD12165706
:105DCD00D003D002D001D000121566C004C005C0AA
:105DDD0006C007902547126307121F2F90253F120B
:105DED0062CD126386D007D006D005D0041217609D
:105DFD009025721262CD126447FC90255D1262CD22
:105E0D001217FD6002500E90254A12630712208270
:105E1D000000000022126392C00390253F12627AA7
:105E2D0012636612652D12627AD00312BC8590271B
:105E3D00BCE06003025F2CE4902561F01263101248
:105E4D001F4F90254D1262CD121657C004C005C0CC
:105E5D0006C00790253C126307126320121F4F9056
:105E6D0025431262CD121657D003D002D001D000B7
:105E7D00121566C004C005C006C00790254D1262FC
:105E8D007A9025431262CD126386D007D006D005D5
:105E9D00D0041263A370A512645C12653812627A85
:105EAD0012648D90254D12627A9025431262CD12A7
:105EBD005F2D706B126392C003C002C00112645C4F
:105ECD007425F0A37459F0902547126309121F2F02
:105EDD0012648D90254D1262CDA312627A12156255
:105EED001264B0D001D002D00312C6579027BCE087
:105EFD00702D9025591262CD90255512627A121788
:105F0D006090254D1262CD12165790254D122045E9
:105F1D0090254D12627A90254A126307121F7F2237
:105F2D0012156690259A1220457B017A2579621209
:105F3D00C6579027BCE02212C6579027BCE022120C
:075F4D00BC859027BCE02297
:1080660090250DEFF0A312635EF090251A122051B1
:1080760000000000E490253BF090253BE0FBD39404
:1080860003501AEB25E025E012637C12627AEB12AC
:1080960063C812204590253BE004F080DC9027441D
:1080A60012627A90252E12204590252E12627A129F
:1080B60063667425F0A3741AF090274812627A7BDF
:1080C600017A25791E12BC859027BCE060030282E6
:1080D6008690251A12627A90250E126307121FF5F2
:1080E60012165790251A12204590251A12627A9078
:1080F6002511126307121F7F90253A7401F090250F
:108106000DE0FF90253AE0D39F400302824A902576
:108116001A12627A90254312204590253AE075F0AE
:1081260018A42444F9742735F0FA9025477401F011
:10813600A3EAF0E91263537425F0A37432F0902594
:108146002E12627A7B017A25791E125C2D9027BC4D
:10815600E0600302828690250E12630790253A128C
:108166006323121F4F9025321262CD1216579025A7
:108176003612644DFC9025361262CD1217FD70162C
:1081860090251112630790253A12632312209C0052
:10819600000000028241E490253BF090253A1263EC
:1081A60077C083C08290253BE0D082D08375F004EF
:1081B6001220C012627A9025361262CD121657C06E
:1081C60004C005C006C0071263C412627A90251A5D
:1081D6001262CD121657D003D002D001D00012156C
:1081E60066C004C005C006C00790253612627A90A4
:1081F600251A1262CD126386D007D006D005D004A8
:108206001217601263C412204590253B1263BD709D
:108216008A90251A12627A9025361262CD12156658
:1082260090251A12204590253612627A9025111251
:10823600630790253A126323121F9990253AE004AA
:10824600F0028104E490253BF090253BE0FFD394B7
:1082560003501EEF1263C812627A90251412630748
:1082660090253B126323121F9990253BE004F08072
:10827600D890251A12627A902517126307121F7F6B
:0182860022D5
:10C04E0090250D12635EF0A31220459027A4126274
:10C05E007A1263667425F0A37418F09027A8126202
:10C06E007A7B017A2779AC12BC859027BCE06006FA
:10C07E00E4FFFEFDFC22902514122051000000006A
:10C08E00E490251CF09025141262CDC000C001C0B2
:10C09E0002C00390250D12630790251C1263231214
:10C0AE001F4F9025101262CD121657C004C005C046
:10C0BE0006C00790251CE01264FFF58312627A9089
:10C0CE0025181262CD121657D003D002D001D0001F
:10C0DE0012156212E04CD003D002D001D00012151E
:10C0EE006690251412204590251CE004F0E0D394B0
:0AC0FE0003409290251412627A228A
:106561009024B5EFF0A312635EF090250C7409F04E
:10657100E4FB9024B5E0FFEBD39F500EEB1263EAEE
:106581001220513DCCCCCD0B80E89024C11220517A
:106591003F8000009024E11220513DCCCCCD9024CD
:1065A100EF12205160AD78ECE49024E5F0A3F09077
:1065B10024E6E004F070069024E5E004F07BFF7A25
:1065C100A479A19024E5E0FFA3E0902517CFF0A3E3
:1065D100EFF07F0312D2B512C51A1292FA12C271EC
:1065E10090250CEFF0901CA8E07004A3E06401700A
:1065F100122011051264EB8010901CA7E0700AD2E2
:106601000F8006C2A9C211D2A9200F0790250CE064
:10661100B4020B9024BD1263077401021CB19024D3
:10662100E712205160AD78EC9024EB12205100006C
:1066310000009024F412205100000000E49024F3A3
:10664100F09024B9E09024C0F09024B5E0FF9024AC
:10665100C0E0FED39F4003026799EE1263EA126223
:106661007A9024E11262CD121566E4FBFA79807802
:106671003F1217FD50030266F71263D6126493C0EE
:1066810083C08212627A9024E11262CD121566D023
:1066910082D08312632E1268379027BCE060030218
:1066A100683612654312627A12C04E9024BA1263A0
:1066B10007121F7F9027BCE06003026836126286D2
:1066C1001217FD601440129024BA12630712647805
:1066D10012627A9024F41220459024BA12630712B0
:1066E10064F81262CD1217FD500C9024BA126307A0
:1066F1001264F81220459024C01263E912627A9064
:1067010024E11262CD1217FD600540030267901269
:1067110063D6126493C083C08212627A9024E1121C
:1067210062CD121562D082D08312632E1268379027
:1067310027BCE0600302683612654312627A12C018
:106741004E9024BA126307121F7F9027BCE06003AA
:106751000268361262861217FD601740159024BA3E
:1067610012630712647812627A12186A9024F41282
:1067710020459024BA1263071264F81262CD1217F1
:10678100FD500C9024BA1263071264F81220459050
:1067910024C0E004F002664A9024F31263E9C08346
:1067A100C08212627A9024F41262CD121566D082F0
:1067B100D0831220459024EB12627AA31262CD128B
:1067C10017FD600250169024E112627A7433FBFACD
:1067D100F9783F1216579024E11220459024EB12CC
:1067E100627AA31220457F0A7ED77D237C3C9024C8
:1067F100EB1262CD1217FD602940277FBD7E377DE8
:10680100867C359024E11262CD1217FD4014D3909D
:1068110024E6E094E89024E5E06480948350030248
:1068210065B01263317425F0A37408F07B017A24FA
:1068310079D1128066227425F0A37408F07B017A65
:076841002479D112806622C8
:10359C009024A8EFF0A312635EF09024B512205192
:1035AC00000000009024CB7401F0E49027BCF09054
:1035BC0024CAF09024CAE0FFD394035013EF126492
:1035CC0027122051000000009024CAE004F080E390
:1035DC0090274812627A9024AD12204512DFFD909C
:1035EC00274412627A1263667424F0A374DCF090A0
:1035FC00274812627A7B017A27794C12BC85E490B9
:10360C0024C9F09024A8E0FF9024C9E0D39F400384
:10361C00023AEA9024A91263079024C91263231278
:10362C001F4F1264A840030236C3E49024CAF090E2
:10363C0024A91263079024C9126323121F4F12632B
:10364C0074C083C0829024CAE0D082D08375F00409
:10365C001220C01262CD121657C004C005C006C09D
:10366C000712642312627A9024B51262CD12165797
:10367C00D003D002D001D000121566C004C005C022
:10368C0006C0079024A91263079024C91263231261
:10369C001F4F9024B51262CD126386D007D006D08E
:1036AC0005D0041217601264231220459024CA120C
:1036BC0063BD600302363B9024B512627A9024A954
:1036CC001263079024C912632312201512156690F9
:1036DC0024B5122045E49027BCF09024AD12627AF8
:1036EC00A312644DFC9024B51262CD1217FD700C20
:1036FC009024AD12205100000000802512645C74EF
:10370C0024F0A374ADF090274412627A12648D9069
:10371C0024B512627A1264B07B017A2479B912C68C
:10372C005712637412627AC004C005C006C0077BCE
:10373C00017A2479CC9024C9E01264C012627A9088
:10374C0024F3122045D007D006D005D00412B3E3E1
:10375C0090193DE0640260030238569024C9E07071
:10376C007B7B017A27794C12D11BC004C005C006A3
:10377C00C0079024A9126307121F2F9024DC126239
:10378C00CD121562D003D002D001D0001264079084
:10379C0024ACE07003023AE1126464C0079019FA99
:1037AC0012627AEC4D4E4F600B12650B1262CD1209
:1037BC00165780069024D812627A12654D12627ADE
:1037CC0012645560067AA479BC80047AA479BF127D
:1037DC00635BF07BFF7AA479A902390C9024C9E0D1
:1037EC0075F018A4244CF9742735F0FA7B0112D12A
:1037FC001B9024A91263079024C91263231220156D
:10380C00126407126464C0079019FA12627AEC4DC4
:10381C004E4F600B12650B1262CD1216578006903C
:10382C0024D812627A12654D12627A1264556006BF
:10383C007AA479BC80047AA479BF12635B126354B6
:10384C001264B67AA479C202390C90193DE0640175
:10385C0060030239149024B11262CD9024AD12622F
:10386C007A1215627B007A5079C3784712641190F2
:10387C0024C9E0704A9024ACE07003023AE112646F
:10388C0064C007126277EC4D4E4F600E12641A90B2
:10389C0024D81262CD12165780069024D812627A60
:1038AC0012627112645560067AA479E580047AA4D8
:1038BC0079E912635BF07BFF7AA479D202390C129E
:1038CC006464C007126277EC4D4E4F600E12641A9E
:1038DC009024D81262CD12165780069024D812620A
:1038EC007A12627112645560067AA479E580047AC2
:1038FC00A479E912635B1263541264B67AA479ED6D
:10390C00D00712D2B5023AE17B007A5079C37847DE
:10391C009024AD12627A1264119024C9E0704A901E
:10392C0024ACE070030239BB126464C007126277E6
:10393C00EC4D4E4F600E12641A9024D81262CD12C8
:10394C00165780069024D812627A1262711264554E
:10395C0060067AA479E580047AA479E912635BF0B5
:10396C007BFF7AA479FD0239B6126464C007126237
:10397C0077EC4D4E4F600E12641A9024D81262CD23
:10398C0012165780069024D812627A126271126451
:10399C005560067AA479E580047AA479E912635B10
:1039AC001263541264B67AA57910D00712D2B512EC
:1039BC00E077EF64096003023AE11200077F327E80
:1039CC000012DE9C12DC369024E012204512CA82D2
:1039DC00AC06AD07EC1218809024E812644D7CC73D
:1039EC009024E81262CD1217FD703B126277EC4DF9
:1039FC004E4F601012DC367B917A0F796878411249
:103A0C001657800312DC3612627112645560067A06
:103A1C00A479E580047AA479E912635BF07BFF7AE0
:103A2C00A57923023AD99024E812627AE4FBFA7958
:103A3C008078411217609024E812204512DEE8903D
:103A4C0024F41220459024E812627A9024F012207B
:103A5C00459024F81220513E570A3D9024FC122028
:103A6C0051000000009024E012627A12D68A902451
:103A7C00E4126274EC4D4E4F600E12641A9024E006
:103A8C001262CD12165780069024E012627A1262EE
:103A9C0071EC4D4E4F600E12641A9024E41262CDFC
:103AAC0012165780069024E412627A90251B12623B
:103ABC007412645560067AA479E580047AA479E9D5
:103ACC0090251F12635EF07BFF7AA579367F051275
:0F3ADC00D2B51200069024C9E004F002360F2282
:10C5B9009024A8EFF0A312635EF07BFF7AA5794976
:10C5C9007F0112D2B57AA5795112C6479024B97460
:10C5D900011262D91265619024B2126307121C49D3
:10C5E90070309027BCE0702A9024AF126307121FA5
:10C5F9002F126517501C7AA5795C12C647E490245E
:10C60900B91262D91265619024AC126307740112E0
:10C619001CB19027BCE070251263041264A5401D6B
:10C62900126304121F2F7BAC7AC5792778B71217CA
:10C63900FD500A12630412208200000000227BFFD1
:0EC649007F0212D2B512C51A9024A8E0FF227B
:10ACB400902490EFF0E49024A1F09024A67409F07D
:10ACC400E4A3F09027BCF012DFFD12C51A90249083
:10ACD400E0FF9024AC7401F0A37424F0A374A712D1
:10ACE40063547424F0A374A21263547424F0A37400
:10ACF400A1F07B017A24799112C5B99024A1E06076
:10AD04000302ADBC9027BCE0600512ADBD80397F65
:10AD14000A7ED77D237C3C9024A21262CD1217FDBB
:10AD2400602C402A12ADBD12D2B57BFF7AA579748E
:10AD34007F0312D2B57BFF7AA579887F0412D2B53E
:10AD44007BFF7AA579967F0512D2B502D90D200F23
:10AD540067902490E0FF7B017A2479919024A7E006
:10AD64009024ACF012359C12C51A1292FA12C271D8
:10AD74009024A6EFF0901CA8E07004A3E064017096
:10AD8400122011051264EB8010901CA7E0700AD207
:10AD94000F8006C2A9C211D2A99024A6E024FE60A5
:10ADA4001724FA60130470A690193DE004F0E0D370
:10ADB4009402409AE4F080962212DFFD7BFF7AA58C
:05ADC40079677F012208
:105F5400902489EFF0788F7C247BFF7AA579A712AF
:105F640063E09024A31220510000000078AF7C2449
:105F74007D017BFF7AA579B71263E278BF7C247D2B
:105F8400017BFF7AA579C71263E29024CF122051D6
:105F940000000000E49024D3F0A3F09027BCF0901C
:105FA400248AF0902489E0FFA3E0FED39F400302FB
:105FB4006201EE12643912627A12651740030261BB
:105FC400F890248AE0FB12637812627A90248F128C
:105FD4002045EB1264C012627A90249312204590FB
:105FE400248AE0FB75F018A42454F582E43427F5E0
:105FF4008312627A902497122045EB75F018A4243A
:1060040058F582E43427F58312627A90249B122097
:106014004512643512627AC004C005C006C00790F8
:10602400257D1220513A83126F12636C7424F0A3FD
:10603400749FF07B017A24798FD007D006D005D0E5
:106044000412BC859027BCE060030262149024CF44
:1060540012627A1264351262CD1215669024CF1240
:1060640020457D991265571262CD1216579024ABC4
:106074001220457D191265571262CD1216579024CD
:10608400A71220459024D3E475F001121D43FED3DA
:10609400E5F09464EE64809480400B9027A812206D
:1060A4005140E00000229024AB12627A9024A7129F
:1060B40062CD121566E4FBFAF97840121760902459
:1060C4009F122045E49024D5F01264CE5052EF1272
:1060D40064D712627A90249F1262CD1216579024CC
:1060E400D5E01263F91262CD121566C004C005C072
:1060F40006C00790249F12627AA31262CD126386AF
:10610400D007D006D005D0041217609024D5E0251E
:10611400E025E024BFF582E4342412646C0260CDEF
:1061240012645C7424F0A3748BF0A31220513A839C
:10613400126F90249F12627AA31262CD1215661216
:1061440064B07B017A2479BF12C6579027BCE06003
:10615400030262149024CF12627A90248B1262CDCF
:106164001217FD90249F600A400812627A9024ABB3
:10617400800612627A9024A712204590248B126222
:10618400CD9024CF12627A12156212E027E4FBFA52
:1061940079C878421217FD5003026088E49024D530
:1061A400F01264CE50391263F8C083C0821262CDFB
:1061B400C000C001C002C0039024D5E01264D7120D
:1061C400627A90249F1262CD121657D003D002D067
:1061D40001D000121566D082D08312646E80C29002
:1061E40024A312627A90249F1262CD121566902421
:1061F400A312204590248AE004F0025FA77FBD7EAD
:10620400377D867C359024A31262CD1217FD500B86
:106214009027A81220510000000022E49024D5F019
:106224001264CE501C1263F8C083C08212627A904A
:1062340024A31262CD121760D082D08312646E80C0
:10624400DFE49024D5F09024D5E0FBD394035010E0
:10625400EB1263F912627AEB1264FF12646C80E64B
:0D6264009024CF12627A9027A812204522C4
:101525005027BD41FFFD8B4080155141E01B7142A5
:101535001FCAC15027DD431AC51F40A6666642FC77
:1015450080004316DC295027CD4A9B078048609CC4
:09155500004A4EE8C04A958940A5
:10BD4900E0FCA3E0FDA3E0FEA3E0FF902579E0F885
:10BD5900A3E0F9A3E0FAA3E0FB1216577BD37A0715
:10BD69007905784112176090258CE0F8A3E0F9A3D2
:10BD7900E0FAA3E0FB2290258412204590259374D4
:10BD890001F0A37425F0A37488F090257DE0FCA34D
:10BD9900E0FDA3E0FEA3E0FF902596122045902543
:10BDA90084E0FCA3E0FDA3E0FEA3E0FF2290259A36
:10BDB900122045902576E0FBA3E0FAA3E0F9227A68
:10BDC900691216579025B0E025E025E022EBF0A393
:10BDD900EAF0A3E9F0229025B0E075F004A4F58219
:10BDE90085F083227F337E937D887C439016602281
:10BDF90024DDF582E43427F5832224CDF582E43469
:04BE090027F5832274
:10DD570012A868C004C005C006C0079025C1E0FC32
:10DD6700A3E0FDEC121880D003D002D001D000123E
:06DD7700165712C7C92275
:10D11B009024EC12BDD69024F01220510000000098
:10D12B00E49024EFF09024F012BD73C000C001C056
:10D13B0002C0039024EC12BDBFA312BDE2121F4F1D
:10D14B009024EFE025E025E024BDF582E43427F5BB
:10D15B008312BD73121657D003D002D001D0001228
:10D16B0015669024F01220459024EFE004F0E0B413
:09D17B0004B39024F012BDAA22B5
:1097D4009025A212BDD69025B112205100000000A0
:1097E4009025B51220510000000012BDED12BD738A
:1097F4001215669025B91220459025B07401F09099
:1098040025B112BD73C000C001C002C00312BDCD9A
:1098140012BDF912BDAA9025C1E4F0A37402F0129E
:10982400DD577B5C79EC784112BDC812BE0312BDD2
:10983400731217609025A212BDBF12BDDF1220154E
:10984400121657D003D002D001D00012156690250D
:10985400B11220459025B512BD73C000C001C002ED
:10986400C00312BDCD12BDF912BDAA7B8C79387824
:109874003F12BDC812BE0312BD731217609025A219
:1098840012BDBF12BDDF122015121657D003D0022D
:10989400D001D0001215669025B51220459025B050
:1098A400E004F0E0C3940450030298039025B1123D
:1098B400BDAA12E04C9025B11220459025A812BDF6
:1098C400AAA312BD731217609025A81220459025F3
:1098D400B912BDAA12C324A804A905AA06AB07900D
:1098E40025B112BDAA121760C004C005C006C00786
:1098F4009025B512BDAA9025A812BD73121566A8AD
:1099040004A905AA06AB07D007D006D005D00412D7
:1099140017609025A812BD73121760C004C005C05B
:1099240006C0079025B512BD739025A812BDAA12D2
:109934001562C004C005C006C0077FD37E077D053D
:109944007C419025B912BD73121657D003D002D0B2
:1099540001D000121760D003D002D001D00012153C
:0A996400629025A512BDBF021F7F0F
:10C6570090259012BDD6E4FFFEFDFC90259A12BDF1
:10C66700731217FD700E90259312BDBF1220820022
:10C677000000002290163F12BDAAEC4D4E4F6032CB
:10C68700902593E0F9A3E0FAA3E09025A5C912BD90
:10C69700D790259612BDAA9025A812204590259AD5
:10C6A70012BDAA9025AC12204590259012BDBF025D
:10C6B70097D412BDED12BD7312156690259E1220F8
:10C6C700457FD37E077D057C4190259A12BD731265
:10C6D700165790259E12BD7312165790259612BDB8
:0EC6E7007312176090259312BDBF121F7F22A1
:10BC850090257612BDD6A312204512BDED12BD73C7
:10BC950012156690258C122045E4FFFE7D807C3FC1
:10BCA50090257912BD731217FD500E90258112BD96
:10BCB500BF122082000000002290163F12BDAAECA0
:10BCC5004D4E4F90257D606C12BD4912176012BD17
:10BCD5007F12BDB612C65790258412BD73C000C031
:10BCE50001C002C003A312BD7390257912BDAA122B
:10BCF5001760D003D002D001D00012165712BD7FB5
:10BD050012BDB612C65790258412BD73C000C0017E
:10BD1500C002C003A312BD7390257912BDAA1217E4
:10BD250060D003D002D001D000121657902584129E
:10BD3500BDA4800612BD4912176090258112BDBFB2
:04BD4500121F7F2228
:10DA8D007C40E0F8A3E0F9A3E0FAA3E0FB227840A4
:10DA9D00E0FCA3E0FDA3E0FEA3E0FF021760EBF0C6
:10DAAD00A3EAF0A3E9F0021F2FE0FBA3E0FAA3E045
:04DABD00F9021F7FCC
:10DCB5009024C6122045E4FFFE7D107C419024C6C9
:10DCC50012DA8F121657E4FBFA79A0784012176022
:0ADCD500E4FBFAF97842121566220A
:10D8C9009024C21220459024BF12DAAB12DCB59025
:10D8D90024C212DA8F1217FD6029E4FFFEFD7CC213
:10D8E9009024C212DA8F121566E4FBFA79A0784007
:10D8F900121657E4FBFA791078411217609024BF89
:04D9090012DAB62256
:10DF2B009024C61220457F487EF97D519024C6125D
:06DF3B00DA8D12165722D8
:10DBDC009024C21220459024BF12DAAB12DF2B9096
:10DBEC0024C212DA8F1217FD60127B487AF9795130
:0DDBFC009024C212DA9B9024BF12DAB622E8
:10DEB8009024C61220457F917E0F7D687C41902476
:08DEC800C612DA8F1216572270
:10DB23009024C21220459024BF12DAAB12DEB890C3
:10DB330024C212DA8F1217FD60147B917A0F796871
:0FDB430078419024C212DA9D9024BF12DAB622E4
:10DED0009024C61220457F507E187D747C42902489
:08DEE000C612DA8F1216572258
:10DB52009024C21220459024BF12DAAB12DED0907C
:10DB620024C212DA8F1217FD60147B507A1879746E
:0FDB720078429024C212DA9D9024BF12DAB622B4
:10DF41009024C61220457F897E187D0D9024C6122B
:06DF5100DA8D12165722C2
:10DC09009024C21220459024BF12DAAB12DF419052
:10DC190024C212DA8F1217FD60127B897A18790DE6
:0DDC29009024C212DA9B9024BF12DAB622BA
:108A4600C2B4128B27C2AFD2B4128B17A2B492D57E
:108A5600D2AF128B27A2D522C2AF7E08C2B4128B28
:108A6600001392B4128B1CD2B4128B17DEEED2AF67
:108A760022C2AF7E08C2B4128AFCD2B4128B05A2FF
:108A8600B413128B1CDEEED2AF128AE222C2B512EA
:108A96008B27C2AFD2B5128B17A2B592D5D2AF1221
:108AA6008B27A2D5D2AF22C2AF7E08C2B5128B00E9
:108AB6001392B5128B1CD2B5128B17DEEED2AF22F3
:108AC600C2AF7E08C2B5128AFCD2B5128B05A2B51A
:108AD60013128B1CDEEED2AF128AE222C0E07F08B0
:108AE60065F013E5F05002641813F5F0D0E003C00A
:108AF600E0DFEDD0E022000000227F10DFFE227FC3
:108B060013DFFE00227F15DFFE00227F22DFFE003C
:108B1600227F47DFFE227F7EDFFE00227FB6DFFE5A
:108B2600227F00DFFEDFFEDFFE7F96DFFE00227F74
:108B360000DFFEDFFEDFFEDFFEDFFEDFFEDFFE7FA5
:108B46002EDFFE227E237F00DFFEDEFA7FC8DFFEF9
:108B56000022128B4A128B4A22128B58128B5822F1
:108B6600128B5F128B5F2254074418232323D2975C
:108B76007F05339297C296D296DFF7C296D296C2F7
:108B860096D29674007F04C296D296A29533DFF7EA
:108B9600F5F07F08C296D296A29533DFF722D292DD
:108BA600128B00C291128B00C292128B0022C291CC
:108BB600128B00D292128B00D291128B00227E0869
:108BC600339291128B00D292128B00C292128B00BA
:108BD600DEEED291128B00D292128B00A291C2923B
:108BE600128B00227E0892D5D292128B00A291336C
:108BF600C292128B00DEF1A2D59291128B00D29214
:0E8C0600128B00C292128B00D291128B0022B0
:10155F00021925E86480F8E933E83360110460F07C
:10156F00ED33EC337009E8FCE9FDEAFEEBFF2204F2
:10157F0060DED3EB9FEA9EE99DE8C2E78CF0C2F7ED
:10158F0095F0400CE8CCF8E9CDF9EACEFAEBCFFBB9
:10159F001218F085D0F05804700320D5B3E804700A
:1015AF00075002B2D502192F92D5EC0460F7E4CCA4
:1015BF00C0E0C398F8603B94186008400DD0E0FB82
:1015CF00021907E4FBFAC9FC8028E830E406E4C9F5
:1015DF00FBE4CAFCE830E305E4C9CACBFCE85407D6
:1015EF006010F8C3E913F9EA13FAEB13FBEC13FCE1
:1015FF00D8F130F52FC3E49CFCEF9BFFEE9AFEED84
:10160F0099FDD0E0FBEF4E4D4C701222DB03021917
:10161F002CEC2CFCEF33FFEE33FEED33FDED30E71A
:10162F00EB021907EF2BFFEE3AFEED39FDD0E0FB91
:10163F0050130BBB000302192FED13FDEE13FEEF3A
:08164F0013FFEC13FC02190764
:10165700EC4D6011E8497017ED33EC3304600DE48D
:10166700FCFFFEFD22E933E8330470F80219251266
:1016770018F058046009E4CC248150062850090268
:10168700192F28400302192CC0E0EB4A7044B98097
:1016970006D0E0FB02191BEF4E701CBD8008EBFF64
:1016A700EAFEE9FD80EBE98DF0A4FEE5F0021740C4
:1016B700E9CDF9EAFEEBFFEF89F0A4FCE5F0CE896E
:1016C700F0A42EFFE435F0CD89F0A42DFEE435F02B
:1016D7008067EF4E7005BD80D780C3EF8BF0A4AC59
:1016E700F0EE8BF0A42CFCE435F0F8EF8AF0A42C94
:1016F700E5F038FCE433CB8DF0A42CFCE5F03BF8A7
:10170700EE8AF0A42CFCE5F038F8E433CF89F0A496
:101717002CFCE5F038CF3400CE89F0A42FFFE5F09C
:101727003EFEE433C98DF0A42EFEE5F039CD8AF0F4
:10173700A42FFFE5F03EFEE43DFD33D0E0FB50076C
:101747000BBB000F02192FEC2CFCEF33FFEE33FE1F
:06175700ED33FD0219074D
:10175D0002192FEC5D046005E85904700302192588
:10176D001218F0580460F6EC4860F2EC7004FDFEBF
:10177D00FF22C860DB2481C85009C398600250065F
:10178D0002192C9850CAF582E9294B4A7005AB8293
:10179D0002191B75F0007C1A7880C3EF9BEE9AED51
:1017AD0099400DC3EF9BFFEE9AFEED99FDE842F0D7
:1017BD00DC23ACF0D0E0FFD0E0FED0E0FDAB82202A
:1017CD00E7101BEB60BAEC2CFCEF33FFEE33FEEDB4
:1017DD0033FD021907E803F830E705C0F075F00096
:1017ED00EF2FFFEE33FEED33FD40B830E7C280AA98
:1017FD0074F8CC6480CCC86480C8F582046043C39F
:10180D00EB9FF5F0EA9E42F0E99D42F0E89C45F031
:10181D0060305018E5825FFFE582F42B5582FB5056
:10182D00210ABA001D09B90019088016E5825BFB73
:10183D00E582F42F5582FF50090EBE00050DBD0047
:10184D00010CC3EB9FF5F0EA9E42F0E99D42F0E8F2
:0D185D009C45F06007CC4820E701B3EC2269
:10186A00ED33EC33600A047003BD8004ECB2E7FC8C
:01187A00224B
:10187B0075F020800E75F010800575F0087D007EE8
:10188B00007F003392D530D503121EFAEC33401093
:10189B00EF33FFEE33FEED33FDEC33FCD5F0ED22F1
:0E18AB00E5F0247EA2D513CC92E7CDCEFF222D
:1018B900EDD2E7CD33EC3392D524814006E4FFFE27
:1018C900FDFC22FCE4CFCECDCC24E0501174FF8086
:1018D900EDC3CC13CCCD13CDCE13CECF13CF047023
:0718E900F030D5DE021EFA0B
:103AEB00E5082495F582E43425F583E0050822905A
:103AFB002592300803902595E475F0011220CC0235
:103B0B001C492001E97F2ED2018018EF540F24901D
:103B1B00D43440D4FF30050BEF24BFB41A0050034C
:103B2B002461FFE50960021509050CE50C7002051F
:103B3B000B30080E902592E475F0011220CCEF02A9
:103B4B001CB102DD307403D2088003E4C208F5080F
:103B5B009025921220E3E4F509F50BF50CE50960CD
:103B6B00077F20123B2E80F5750AFFC202C201C2ED
:103B7B0003C204C206C207C209123AFAFF700D3023
:103B8B0008057F00123B3FAF0CAE0B22B4255FC282
:103B9B00D5C205123AFAFF24D0B40A00501A75F0B8
:103BAB000A780930D50508B6FF0106C6A426F6200B
:103BBB00D5047002D20480D924CFB41A00EF50047C
:103BCB00C2E5D205023E31D20280C6D20180C0D2FC
:103BDB000380BCD2D580BAD20680B47F20123B2E94
:103BEB002003077401B5090040F1123AEBFF123BB9
:103BFB002E023B68D209D2078095123AEBFB123AA0
:103C0B00EBFA123AEBF94A4B7006792F7A3F7BFFAE
:103C1B0020032EE509602A7E008E82758300121C1C
:103C2B006260060EEE650A70F0C2D5EBC0E0EAC02A
:103C3B00E0E9C0E0EE123E92D0E0F9D0E0FAD0E03D
:103C4B00FB121C49FF60AAEBC0E0EAC0E0E9C0E050
:103C5B00123B2ED0E02401F9D0E03400FAD0E0FB87
:103C6B00E50A0460DCD50AD98087D20380A2123E14
:103C7B007460F7E50A700104121954A90A600DE586
:103C8B000A600914F50A123F1CEF60F3EA30E702F1
:103C9B00F404C3995079EAF4250A0430E701E404EB
:103CAB00F50A800D123E7460C1EA050A250A121945
:103CBB0054EA9025C1F030E701E4250A04D50A0443
:103CCB0020060114123E92E4C0E0123F1C9025C165
:103CDB00E0601320E70714F0123B16802204F0D0AB
:103CEB00E014C0E07F00123B16E50A6007123B0DA3
:103CFB00150A800B300603123B0DD0E0023B68D057
:103D0B00E00480C4123E74609EE50A0412195490BC
:103D1B0025C1EAF0E50A2006026001042404123EE4
:013D2B009205
:103D2C0074FF04C0E0123F1C123B16E50A20060289
:103D3C006003123B0DD0E0B50AE87F45123B2090A2
:103D4C0025C1E07F2B30E7047F2DF404C0E0123B4B
:103D5C002ED0E075F00A84C0F0123B17D0E0123B75
:103D6C0017023B68791080027908C207C2098008E3
:103D7C00D2D5790A8004790AC2D5E50A047002F515
:103D8C000AE4FAFDFEFF123AEBFC7B082002131248
:103D9C003AEBFD7B1030010A123AEBFE123AEBFFC4
:103DAC007B20EC3382D592D55013C3E43001069FAF
:103DBC00FFE49EFEE42002039DFDE49CFCE4CBF8B2
:103DCC00C202EC700CCFCECDCCE824F8F870F380A6
:103DDC0017C3EF33FFEE33FEED33FDEC33FCEB3367
:103DEC00FB994002FB0FD8E9EB300205F8D0E0C498
:103DFC0048B202C0E00AEC4D4E4F78207B0070C2F6
:103E0C00EAB50A0040BCC0E0123E94D0F0D0E020ED
:103E1C000204C4C0E0C4B202C0F0123B17D0F0D50B
:103E2C00F0EB023B681221953C05533D70583BD694
:103E3C004C3BD2423D744F3D7C443D7C493BEB4373
:103E4C003D82553CAF463D0F453C79473F4F503B7B
:103E5C00DA2D3BDE2E3C012B3BE2233BFF203F388F
:103E6C002A3B9A4800003BF9E50AB4FF03750A06A1
:103E7C00123AEBFC123AEBFD123AEBFE123AEBFF64
:103E8C009025BA021991790AA2D52004143006099A
:103E9C00B910020404B9080104A2D520070250018C
:103EAC00042003689203B509005034C0E07F203031
:103EBC0004197F30A20372077206500F123EEBC238
:103ECC0003C207C206C2097F30800F300603E9C067
:103EDC00E0123B2E300603D0E0F9D0E0B509CC302F
:103EEC0006177F30B9100C123B2E7F583005077F18
:103EFC00788003B90803123B2E3003057F2D023B5B
:103F0C002E7F202009F87F2B2007F322920380CFED
:103F1C007F00B40700500B24BAF582E43425F583F6
:103F2C00E0FF22286E756C6C2900D202123AEB303D
:103F3C0002F8C202780930D50108F6023B9A2D50DE
:103F4C00434958123AEB2403B405004001E4903F76
:103F5C004A93123B1F743A123B1FD2047509040298
:023F6C003D70A6
:0DE02700ED33EC3360065004EC6480FC2205
:10C7910033DA929E35B16011377FE5FE3921848904
:10C7A1003AAEC3FF3C1D955B3D6358473E75FDF0B6
:10C7B1003F3172183F800000C2D502192F0219259E
:10C7C100BD80FA50F302192CED33EC330460F17B98
:10C7D1003B7AAA79B8783F121657ED33EC3392D5EC
:10C7E100247B5011A2D570DB500BED448024045002
:10C7F10004A2D580CEEFFBEEFAEDF9ECF81218B9F0
:10C80100EFF582F404FC121885121566C08290C7F8
:10C81100917409121AA5ED33CC33D0F092D525F0DD
:0AC82100A2D57001C313CC13FD2251
:10A834003E9248DA3ECCCCCD3F2AAAAB4000000081
:10A844003F8000003F9837F03FB504F33FD744FC06
:10A854003E3172173EB172173F0515913EDE5BD94A
:10A86400D2008002C200EDD2E7F8CD33EC3304709D
:10A874000BBD800592D502192F02192540FBD31474
:10A8840060F2F5F07C3FEE7A00C39496C8948B4056
:10A89400230AC89469C8941A401A0AC89468C894C8
:10A8A4001F40110AC8945AC89425400805F07A003C
:10A8B400CDC2E7CDC0F09025C3122045EA2323C0C2
:10A8C400E02444F582E434A8F583121FE5121566EA
:10A8D400ECC0E0EDC0E0EEC0E0EFC0E0121FC990B4
:10A8E40025C3121FD9121562D0E0FBD0E0FAD0E0E4
:10A8F400F9D0E0B2E7F81217609025C31220459012
:10A90400A8347403121A969025C3121FD91216572D
:10A91400D0E0600F2450F582E434A8F583121FE5DB
:10A924001215669025C3122045D0E0C3947FFDE440
:10A934009400FC1218807B187A727931783F1216D1
:10A94400579025C3121FD912156630000B7BD97A94
:09A954005B79DE783E12165722F1
:10C3200002192522EDA2E7D2E7F9EC3340F260F3DF
:10C33000B4FF08ED547F70E802192FF82481C2E0A1
:10C34000C0E0F40428FAC313FCED92E7FD9025BD8C
:10C35000122045EEA2E7E9BA7F02C313340094002D
:10C36000FA75F091A4E5F013F494FE8AF0A433E595
:10C37000F033248CD313FDE492E7FE7F007C3F75FD
:10C380008302ECC0E0F8EDC0E0F9EEC0E0FAEFC0E7
:10C39000E0FB8583F09025BD121FBD85F083121749
:10C3A00060D0E0FBD0E0FAD0E0F9D0E0F8121566FA
:10C3B000ED6480FD30E7011CD583C7ED33CC33F845
:0CC3C000D0E0A2E71328C313CC13FD2229
:109F8400902476122045E4FFFE7D807C3F90247669
:109F9400E0F8A3E0F9A3E0FAA3E0FB1217FD7006D2
:109FA40090247602A0DE902476E0FCA3E0FDA3E0FA
:109FB400FEA3E0FF12193AFBA3E0FCA3E0FDA3E03B
:109FC400FEA3E0FF12193AFFB40108E4FFFE7D800E
:109FD4007C3F22EF64046029EB64046024EBB40149
:109FE40030E4FFFEFDFC90247AE0F8A3E0F9A3E05E
:109FF400FAA3E0FB1217FD60084006E4FFFEFDFC37
:10A004002290247A122051FFFFFFFF90247A02A0AD
:10A01400DEE490247EF0A3F0FFFEFDFC902476E0C5
:10A02400F8A3E0F9A3E0FAA3E0FB1217FD505F9058
:10A03400247AE0FCA3E0FDA3E0FEA3E0FF1218B93C
:10A0440090247EEEF0A3EFF0FDCCEECCEC12188061
:10A05400C8ECC8C9EDC9CAEECACBEFCB90247AE0EC
:10A06400FCA3E0FDA3E0FEA3E0FF121562E4FBFA0B
:10A07400F9F81217FD708A902476E0FCA3E0FDA3A2
:10A08400E0FEA3E0FF12186A902476122045902483
:10A0940076E0FCA3E0FDA3E0FEA3E0FF12A8689035
:10A0A400247AE0F8A3E0F9A3E0FAA3E0FB12165740
:10A0B40012C7C990247A12204590247FE030E0171B
:10A0C40090247AE0FCA3E0FDA3E0FEA3E0FF1218D5
:10A0D4006A90247A12204590247AE0FCA3E0FDA340
:06A0E400E0FEA3E0FF22F4
:10D6D70090258CE0FFA3E0FEA3E0CF902595F0A373
:10D6E700EEF0A3EFF090258FE0CBF0A3E0CAF0A314
:10D6F700E0C9F07F22902598AD82AC83121C498D3A
:10D70700828C83F0A309E970010ADFEC90258FE092
:0AD71700FBA3E0FAA3E0F9023B5087
:1018F000E9D2E7C933E833F892D5EDD2E7CD33EC3E
:0719000033FC5002B2D522B6
:10190700EC30E7100FBF000C0EBE00080DBD000441
:101917000BEB6014A2D5EB13FCED92E7FD2274FFED
:10192700FCFDFEFF22E480F8A2D574FF13FC7D8046
:03193700E480EF5A
:10193A00ED33EC33601004700FED547F70057402C0
:0A194A0092E2227404220422E42237
:10195400F920E73624F950037907E4F42402FBE57F
:1019640082158270021583DBF6E024FB501BE960CC
:1019740014E4F0E582158270021583E004F0B40AE1
:0D19840008E4F0D9EE7401F00A22C2D52269
:10199100ED33EC3392D5FA602AB4FF33EDC2E77B25
:1019A100FF60067A1979B6E4227A1979BF20D50445
:1019B1007A1979BA224E614E002B494E46002D49C3
:1019C1004E4600E47A08F0A3DAFC7B00740722C0DB
:1019D10083C082ECC0E0EDC0E0EEC0E0EFC0E0EA21
:1019E10075F010A4CAABF075F04DA42BFBE435F0F3
:1019F100FCEA2410FAEB34C5FBEC34D9FCEDC2E768
:101A0100FF75F056A4F42411C5F0F434C58FF0A489
:101A11002AE5F03BE43CF020E714121B13D0E0FF71
:101A2100D0E0FED0E0FDD0E0FC1217608014F40499
:101A3100121B13D0E0FFD0E0FED0E0FDD0E0FC129D
:101A41001657D082D083E0FAEDD2E7CD33EC3324C0
:101A510082FBE4C3CF33CFCE33CECD33CD33DBF3F3
:101A61007B0775F00A846004F0A31B0AE5F0F0A37C
:101A71008FF0740AA4FFACF08EF0740AA42CFEACB3
:101A8100F050010C8DF0740AA42CFDE435F0F0A3A4
:051A9100DBDE740722FA
:101A9600C0E0EFFBEEFAEDF9ECF8121657D0E0F5E0
:101AA600F0EFFBEEFAEDF9ECF8121FC9A3A3A3A31E
:101AB600E8C0E0E9C0E0EAC0E0EBC0E0C0F0121622
:101AC60057121FE5A3A3A3A3121566D0F0D0E0FB1F
:0D1AD600D0E0FAD0E0F9D0E0F8D5F0D4224D
:101AE3003F8000004120000042C80000447A00000B
:101AF300461C400047C35000497424004B1896808D
:101B03004CBEBC205A0E1BCA6753C21C749DC5AE83
:101B1300FB60065407601C2323121B41EB543860FF
:101B230009121B2D121B3C121657ECF8EDF9EEFAB5
:101B3300EFCB22EB121B3C80F1543803241C901A88
:101B4300E3FE93FC0EEE93FD0EEE930ECE93FF2277
:0300000002CBA090
:0CCBA000787FE4F6D8FD75812302CBE716
:101B5300E709F608DFFA8046E709F208DFFA803E74
:101B630088828C83E709F0A3DFFA8032E309F60861
:101B7300DFFA8078E309F208DFFA807088828C83C9
:101B8300E309F0A3DFFA806489828A83E0A3F6087D
:101B9300DFFA805889828A83E0A3F208DFFA804C57
:101BA30080D280FA80C680D4806980F2803380102E
:101BB30080A680EA809A80A880DA80E280CA803397
:101BC30089828A83ECFAE493A3C8C582C8CCC5830F
:101BD300CCF0A3C8C582C8CCC583CCDFE9DEE780DF
:101BE3000D89828A83E493A3F608DFF9ECFAA9F05E
:101BF300EDFB2289828A83ECFAE0A3C8C582C8CCB4
:101C0300C583CCF0A3C8C582C8CCC583CCDFEADECC
:101C1300E880DB89828A83E493A3F208DFF980CC2E
:101C230088F0EF60010E4E60C388F0ED2402B40427
:101C33000050B9F582EB2402B4040050AF232345CE
:061C43008223901BA37335
:101C4900BB010689828A83E0225002E722BBFE0299
:091C5900E32289828A83E49322CC
:101C6200BB010CE58229F582E5833AF583E0225037
:101C720006E92582F8E622BBFE06E92582F8E22281
:0D1C8200E58229F582E5833AF583E493229B
:101C8F00BB010989828A83F8E028F022500327F7E5
:101C9F0022BBFE05F8E328F3228A838982F8E493B6
:021CAF002822E9
:101CB100BB010689828A83F0225002F722BBFE0112
:021CC100F3220C
:101CC300F8BB010DE58229F582E5833AF583E8F057
:101CD300225006E92582C8F622BBFE05E92582C803
:021CE300F222EB
:101CE500EF8DF0A4A8F0CF8CF0A428CE8DF0A42E13
:021CF500FE22CD
:101CF700C2D5EC30E709B2D5E4C39DFDE49CFCEE08
:101D070030E715B2D5E4C39FFFE49EFE1221E7C377
:101D1700E49DFDE49CFC80031221E730D507C3E472
:061D27009FFFE49EFE2276
:101D2D00C5F0F8A3E028F0C5F0F8E5821582700241
:061D3D001583E038F022DE
:101D4300A3F8E0C5F025F0F0E58215827002158353
:061D5300E0C838F0E822B0
:101D5900BB0110E58229F582E5833AF583E0F5F0C8
:101D6900A3E0225009E92582F886F008E622BBFEA5
:101D79000AE92582F8E2F5F008E222E5832AF583EB
:081D8900E993F5F0A3E99322B0
:101D9100BB010A89828A83F0E5F0A3F0225006F79D
:0F1DA10009A7F01922BBFE06F3E5F009F319229A
:101DB000F8BB0111E58229F582E5833AF583E8F065
:101DC000E5F0A3F0225009E92582C8F608A6F02222
:0D1DD000BBFE09E92582C8F2E5F008F22209
:101DDD00E88FF0A4CC8BF0A42CFCE98EF0A42CFCA5
:101DED008AF0EDA42CFCEA8EF0A4CDA8F08BF0A423
:101DFD002DCC3825F0FDE98FF0A42CCD35F0FCEB82
:101E0D008EF0A4FEA9F0EB8FF0A4CFC5F02ECD3946
:0F1E1D00FEE43CFCEAA42DCE35F0FDE43CFC22B3
:101E2C0075F008758200EF2FFFEE33FECD33CDCC6D
:101E3C0033CCC58233C5829BED9AEC99E5829840F0
:101E4C000CF582EE9BFEED9AFDEC99FC0FD5F0D6CD
:101E5C00E4CEFBE4CDFAE4CCF9A88222B800C1B9F7
:101E6C000059BA002DEC8BF084CFCECDFCE5F0CB35
:101E7C00F97818EF2FFFEE33FEED33FDEC33FCEB6E
:101E8C0033FB10D703994004EB99FB0FD8E5E4F929
:101E9C00FA227818EF2FFFEE33FEED33FDEC33FC16
:101EAC00C933C910D7059BE99A4007EC9BFCE99A0A
:101EBC00F90FD8E0E4C9FAE4CCFB2275F010EF2F4F
:101ECC00FFEE33FEED33FDCC33CCC833C810D7074F
:101EDC009BEC9AE899400AED9BFDEC9AFCE899F88A
:0E1EEC000FD5F0DAE4CDFBE4CCFAE4C8F9221D
:0E1EFA00C3E49FFFE49EFEE49DFDE49CFC22F9
:101F0800EB9FF5F0EA9E42F0E99D42F0EC6480C850
:061F180064809845F022F0
:101F1E00EB9FF5F0EA9E42F0E99D42F0E89C45F019
:011F2E002290
:101F2F00BB010789828A83021FBD5005E9F802228F
:101F3F003CBBFE05E9F802224889828A83021FC949
:101F4F00BB010DE58229F582E5833AF583021FBDBA
:101F5F005007E92582F802223CBBFE07E92582F8EB
:101F6F00022248E58229F582E5833AF583021FC9EB
:101F7F00BB010789828A830220455005E9F80222B6
:0A1F8F006EBBFE05E9F802227A227B
:101F9900BB010DE58229F582E5833AF583022045E7
:101FA9005007E92582F802226EBBFE07E92582F86F
:041FB90002227A2264
:0C1FBD00E0FCA3E0FDA3E0FEA3E0FF2297
:101FC900E493FC740193FD740293FE740393FF225E
:0C1FD900E0F8A3E0F9A3E0FAA3E0FB228B
:101FE500E493F8740193F9740293FA740393FB2252
:101FF500BB010789828A83021FD95005E9F80222AD
:1020050054BBFE05E9F802226189828A83021FE535
:10201500BB010DE58229F582E5833AF583021FD9D7
:102025005007E92582F8022254BBFE07E92582F80C
:10203500022261E58229F582E5833AF583021FE5EF
:0C204500ECF0A3EDF0A3EEF0A3EFF0220E
:10205100A8828583F0D083D0821220681220681272
:102061002068122068E473E493A3C583C5F0C58397
:10207100C8C582C8F0A3C583C5F0C583C8C582C8D9
:01208100223C
:10208200BB010789828A830220515005E9F80222A6
:0A20920086BBFE05E9F802229F223A
:10209C00BB010DE58229F582E5833AF583022051D7
:1020AC005007E92582F8022286BBFE07E92582F853
:0420BC0002229F223B
:0C20C000A42582F582E5F03583F583222B
:1020CC00F8E0FBA3A3E0F925F0F0E582158270029D
:0720DC001583E0FA38F02241
:0920E300EBF0A3EAF0A3E9F022FE
:1020EC00BB010789828A830222CA5005E9F80222C1
:1020FC00B8BBFE05E9F80222D389828A830222E565
:10210C00BB010DE58229F582E5833AF5830222CAEB
:10211C005007E92582F80222B8BBFE07E92582F8B0
:10212C000222D3E58229F582E5833AF5830222E582
:10213C00BB0120E58229F582E5833AF583D0F0D006
:10214C00E0F8D0E0F9D0E0FAD0E0FBE8C0E0C0F075
:10215C000220E35018E92582F8D083D082D0E0F930
:10216C00D0E0FAD0E0FBC082C0830222C1BBFE18D3
:10217C00E92582F8D083D082D0E0F9D0E0FAD0E023
:09218C00FBC082C0830222DC22A8
:10219500D083D082F8E4937012740193700DA3A3D9
:1021A50093F8740193F5828883E4737402936860ED
:0621B500EFA3A3A380DFED
:10DD3000EFB40A07740D12DD3B740A309811A899EC
:10DD4000B8130CC2983098FDA899C298B811F63053
:07DD500099FDC299F599222B
:10DFCD00C3EE6480948040028007C3E49FFFE49E0B
:02DFDD00FE2222
:10DF6C00E4FFFE121C49600C0FEF70010E09E97002
:05DF7C00F20A80EF2213
:1021BB00EF4E6012EF60010EEDBB010B89828A833B
:1021CB00F0A3DFFCDEFA2289F05007F709DFFCA948
:0C21DB00F022BBFEFCF309DFFCA9F0229F
:10CBAC0002C3CCE493A3F8E493A34003F68001F210
:10CBBC0008DFF48029E493A3F85407240CC8C3338A
:10CBCC00C4540F4420C8834004F456800146F6DF59
:10CBDC00E4800B0102040810204080900026E47EC3
:10CBEC00019360BCA3FF543F30E509541FFEE4934E
:10CBFC00A360010ECF54C025E060A840B8E493A315
:10CC0C00FAE493A3F8E493A3C8C582C8CAC583CA3F
:10CC1C00F0A3C8C582C8CAC583CADFE9DEE780BEF7
:01155E00008C
:1021E700BC000BBE0029EF8DF084FFADF022E4CCDC
:1021F700F875F008EF2FFFEE33FEEC33FCEE9DECA5
:10220700984005FCEE9DFE0FD5F0E9E4CEFD22EDEA
:10221700F8F5F0EE8420D21CFEADF075F008EF2F34
:10222700FFED33FD4007985006D5F0F222C398FD25
:052237000FD5F0EA22C2
:0C223C00E6FC08E6FD08E6FE08E6FF22CE
:0C224800E2FC08E2FD08E2FE08E2FF22D2
:0D225400E6FB08E6F908E6FA08E6CBF822FA
:0D226100E2FB08E2F908E2FA08E2CBF822FD
:0C226E00ECF608EDF608EEF608EFF6229C
:0C227A00ECF208EDF208EEF208EFF222A0
:10228600D083D082E493F608740193F6087402931F
:09229600F608740393F674047356
:10229F00D083D082E493F208740193F2087402930E
:0922AF00F208740393F274047345
:0922B800E6FB08E6FA08E6F9224B
:0922C100EBF608EAF608E9F62242
:0922CA00E0FBA3E0FAA3E0F92215
:0922D300E2FB08E2FA08E2F9223C
:0922DC00EBF208EAF208E9F22233
:0C22E500E493FB740193FA740293F92255
:00000001FF
